:020000040800F2
:10000000D84A022021030008E18400082D65000879
:1000100005840008F13900086DEE000800000000BA
:10002000000000000000000000000000C5DA000829
:10003000B152000800000000F3300008D58C000821
:100040003B0300083B0300083B0300083B03000898
:100050003B0300083B0300083B0300083B03000888
:100060003B0300083B0300083B0300083B03000878
:100070003B0300083B0300083B0300083B03000868
:100080003B0300083B0300083B030008A93C0008B1
:10009000853B00083B0300083B0300088D53000824
:1000A0003B0300083B0300083B0300083B03000838
:1000B0003B03000891E00008D1E000083B03000882
:1000C0003B0300083B0300083B0300083B03000818
:1000D0003B03000879E40008E5E500085DE7000857
:1000E0003B0300083B0300083B0300083B030008F8
:1000F0003B0300083B0300083B0300083B030008E8
:100100003B0300083B03000811E100083B03000823
:1001100089E200083B0300083B03000855E10008A2
:100120003B0300083B0300083B0300083B030008B7
:100130003B0300083B0300083B0300085540000850
:10014000BD3E00083B0300083B0300083B030008DA
:100150003B0300083B0300083B0300084DE900088F
:100160003B0300083B0300083B0300083B03000877
:100170003B0300083B0300083B0300083B03000867
:100180003B0300083B03000800F002F800F0B6F85B
:100190000AA090E8000C82448344AAF10107DA45E2
:1001A00001D100F0ABF8AFF2090EBAE80F0013F07E
:1001B000010F18BFFB1A43F001031847F87E010036
:1001C000187F010010F8013B0A4413F0030408BF34
:1001D00010F8014B1D1108BF10F8015B641E05D01B
:1001E00010F8016B641E01F8016BF9D1002D15D0D8
:1001F00010F8014B03F00C030C2BA1EB04040ABF15
:1002000010F8013BA4EB8314A4EB032405F10103D4
:1002100014F8016B5B1E01F8016BF9D5914238BFF0
:1002200010F8013BD1D3704700230024002500269D
:10023000103A28BF78C1FBD8520728BF30C148BF49
:100240000B6070476E2900F01685702900F09F81C1
:10025000662917F06D83652917F06A83672917F0FF
:100260006783612917F0668303681B0A28BF41F082
:100270008001692900F01081642900F00D81752941
:1002800000F00A816F2900F00E86782900F06B815A
:10029000E92900F0A985E42900F0A685F52900F0F8
:1002A000A385EF2900F00B86F82900F06A81036826
:1002B000DB0928BF41F08001632900F0188573290C
:1002C00000F01D85E32901F05D85F32901F06285C9
:1002D000002070471FB517F01EFB01F069F90400FC
:1002E0000020002116F060FC401C6060002000210E
:1002F00016F070FCE0601FBD10B510BD01F0BCFF32
:100300001146FFF7E7FF13F0D3FE02F045FA03B4FE
:10031000FFF7F2FF03BC11F00DF9000040BA70477F
:100320000948804709480047FEE7FEE7FEE7FEE789
:10033000FEE7FEE7FEE7FEE7FEE7FEE704480549C5
:10034000034A054B7047000029E0000889010008B6
:10035000D83B0220D84A0220D83B022072B6704710
:1003600062B67047EFF3108072B6704780F3108862
:10037000704730BF704720BF7047B0FA80F07047B9
:1003800090FAA0F0B0FA80F0704790FAA0F07047B1
:100390001CB50C46064B7B4469460090204600F095
:1003A00084FC04460020694600F092FC20461CBDF7
:1003B000370900000FB4044910B503AA029800F0F1
:1003C000A3FC10BC5DF814FB381100200FB41CB561
:1003D000084B06AA7B4469460090059800F065FC2E
:1003E00004460020694600F073FC20461CBC5DF802
:1003F00014FB0000F908000070B504468569006828
:10040000C10601D5302600E02026C00707D070BD08
:10041000D4E9012130469047206A401C20626D1EBD
:10042000F6D570BD70B5044685690078C00707D160
:1004300070BDD4E9012120209047206A401C206231
:100440006D1EF6D570BD70B50C460546012A05D067
:100450002878800600D5EA69002302E0012305E040
:100460005B1C934202D2E05C0028F9D1A869E6182F
:10047000C01AA861286A184428622846FFF7BCFF02
:1004800004E0D5E9012114F8010B9047B442F8D3F8
:100490002846FFF7C7FF70BD2DE9F041064600244E
:1004A00010687529314616A510D000F079FB002898
:1004B00002DA404213A507E031688A0701D512A588
:1004C00002E0490704D511A5012401E000F071FB09
:1004D00000210A2206F1240709E0B0FBF2FCB0FB80
:1004E000F2F302FB1C00303078541846491C0028F7
:1004F000F3D123462A463046BDE8F04100F062BB06
:10050000000000002D0000002B0000002000000073
:10051000F0B40D460188090502D5214C7C4402E067
:100520001F4C7C440E34002100F1240608E002F048
:100530000F071209E75D42EA03721B097754491C51
:1005400052EA0307F3D102780023120704D5702D75
:1005500006D009B1022311342246F0BC00F032BBB0
:1005600001231034F8E770B504460D4621461068A3
:1005700000F01FFB024629462046BDE870400023DC
:10058000C6E7D21D22F00703D3E90023C0E70368C2
:10059000126843F0200303600823C3610023B7E718
:1005A000B87501002DE9F05F894604464FF0000A56
:1005B000DFF874B1FB44C0F820A02046E16888470A
:1005C000002874D0252806D0D4E901219047206A5C
:1005D000401C2062F1E700265F462046E16888471C
:1005E0002028054607DB312D05D2781910F8200C9C
:1005F00008B10643F1E7B00701D526F00406C4F8B8
:100600001CA00027C4F818A02A2D09D0284610F0F5
:100610008AFF38B304EB8708303DC8F8185019E05A
:1006200059F8041B204604EB87029161E168884772
:10063000012F054618D1E069002820DA26F02006AF
:100640001DE0D8F8180000EB800005EB40003038C2
:10065000C8F818002046E1688847054610F063FF97
:100660000028EED1012F0AD02E2D08D12046E168B6
:1006700088477F1C0546022F46F02006C4DBA06990
:10068000002803DA404246F00106A061F00701D0DD
:1006900026F010066C2D0BD0682D09D04C2D39D0CA
:1006A0006A2D35D0742D35D07A2D33D016E038E050
:1006B000E1682F4620468847B842054609D16C2F8D
:1006C00026D04FF48060E1680643204688470546FF
:1006D00004E06C2F1AD04FF4807006430DB3A5F1DF
:1006E0004100192802D8203546F400664A462946BA
:1006F000204626604E46FFF7A5FD80B101280BD0AD
:10070000F61D26F0070000F1080956E74020E4E74F
:100710008020D8E70020D6E706F104094DE72846F7
:1007200052E7206ABDE8F09F487501000FB400B59C
:100730008DB010A9099000910B904FF0FF300A90F6
:1007400000200C90064878440690064878446A4693
:1007500007900F9909A800F04DFE0DB05DF814FB4D
:10076000CB0C0000E30C00002DE9FF5F1D464FF0AD
:10077000FF3B91464FF000085F46D5E90146A96965
:1007800001987F1C8847296A824688470028F6D14D
:10079000BAF1FF3F0CD0002E24F4C06419DD6006CE
:1007A00014D5BAF12B0F09D0BAF12D0F0ED103E0F9
:1007B000584604B0BDE8F09F44F48064A9690198EC
:1007C0007F1C8847761E8246002E02DDBAF1300F6C
:1007D00003D0B9F1000F26D032E0A969761E019846
:1007E0007F1C44F400748847002E824605DDBAF170
:1007F000780F06D0BAF1580F03D0B9F1000F10D01E
:100800001EE0B9F1000F02D0B9F1100F18D1A9699B
:10081000761E01987F1C24F40074884782461020BD
:1008200002E0082000E00A20814609E0A96908FBEF
:100830000908761E01987F1C44F40074884782469C
:10084000002E05DD4946504600F044FB0028EDDA55
:10085000E96901988847A00502D46FF00100A8E774
:10086000E00725D1600613D5600502D5C8F1000068
:1008700000E0404629680A1D2A600968220501D562
:10088000087015E0220701D5088011E008600FE02C
:100890002868011D29600068210502D580F80080C4
:1008A00006E0210702D5A0F8008001E0C0F8008032
:1008B00038467EE770B5064600F056F904680546EE
:1008C00030460A22002100F014FE2C6070BD2DE994
:1008D000F05F93460F4680460446002600F044F938
:1008E000D0F80090824614F8015B2DB100F034F985
:1008F0000068405DC007F6D12B2D02D02D2D1AD0F7
:10090000641E0021CAF800105A463946204600F0FD
:10091000A1FD014627B13868A04201D1C7F8008087
:10092000DAF80000022809D0CAF80090700505D551
:100930004842BDE8F09F46F48066E2E70846F8E7E3
:10094000014A00F00FBE0000CC29002040EA01035C
:10095000024630B59B0710D14FF0013400E008C2C9
:1009600008C91D1B9D4315EAC41FF8D013F0FF01F1
:1009700002F8011B0DD01B0AF8E711F8013B002B10
:1009800002F8013B05D011F8013B002B02F8013BB6
:10099000F3D130BD2DE9F0410E460546002400E0BC
:1009A000641C285D00F0EFF80746305D00F0EBF8BE
:1009B000381A02D1295D0029F2D1BDE8F08110B5C5
:1009C000431C02E010F8011B71B18107FAD14FF00E
:1009D000013202C88C1A8C4314EAC211F9D0C01A31
:1009E0000A0603D0C01E10BDC01A10BD0A0401D0F3
:1009F000801E10BD0902FCD0401E10BD421E12F820
:100A0000013F002BFBD111F8013B002B02F8013B09
:100A1000F9D17047032A40F2308010F0030C00F047
:100A2000158011F8013BBCF1020F624498BF11F828
:100A300001CB00F8013B38BF11F8013BA2F10402E1
:100A400098BF00F801CB38BF00F8013B11F0030359
:100A500000F02580083AC0F0088051F8043B083ABD
:100A600051F804CBA0E80810F5E7121D5CBF51F85F
:100A7000043B40F8043BAFF30080D20724BF11F8D9
:100A8000013B11F801CB48BF11F8012B24BF00F83E
:100A9000013B00F801CB48BF00F8012B704710B5AF
:100AA000203AC0F00B80B1E81850203AA0E8185066
:100AB000B1E81850A0E81850BFF4F5AF5FEA027C27
:100AC00024BFB1E81850A0E8185044BF18C918C096
:100AD000BDE810405FEA827C24BF51F8043B40F837
:100AE000043B08BF7047D20728BF31F8023B48BF1C
:100AF00011F8012B28BF20F8023B48BF00F8012B5A
:100B000070474FF0000200B51346944696462039D0
:100B100022BFA0E80C50A0E80C50B1F12001BFF4B6
:100B2000F7AF090728BFA0E80C5048BF0CC05DF81C
:100B300004EB890028BF40F8042B08BF704748BF6A
:100B400020F8022B11F0804F18BF00F8012B7047DE
:100B5000704770477047000010B500F029FD001D78
:100B600010BD00BF4560010000487047783B02207F
:100B700010B5FFF7F9FF006810BD10B50446FFF788
:100B8000F3FF046010BD10B50446FFF7E5FF0068F1
:100B9000005DC00602D504F1200010BD204610BD46
:100BA00009684A0501D540B27047C905FCD500B2B5
:100BB000704709684A0501D5C0B27047C905FCD520
:100BC00080B270472DE9F0470D469946924604469B
:100BD00000F124080168880604D5E06921F01001BD
:100BE000216000E00120A84201DD471B00E0002752
:100BF000A1697A1902EB0900081AA0612078C006E1
:100C000002D42046FFF7F8FB002608E0D4E90121D2
:100C10001AF806009047206A401C761C20624E4558
:100C2000F4DB2078C0060AD52046FFF7E5FB06E096
:100C3000D4E9012130209047206A401C2062381EF0
:100C4000A7F10107F4DC07E0D4E9012118F8050059
:100C50009047206A401C2062281EA5F10105F3DCA4
:100C60002046FFF7DFFB2078000602D50220BDE812
:100C7000F0870120FBE711680268006A530501D57F
:100C800008700AE0D30501D5088006E0130603D5F5
:100C9000C217C1E9000200E00860012070470000AF
:100CA00001694A1C02610878704700B58FB0CDE930
:100CB00001310021059105497944CDE90310114620
:100CC0006846FFF76FFC0FB000BD0000E5FFFFFFB7
:100CD0000A6802F8010B0A60704710B5436913B146
:100CE000AFF3008001E0FFF7AEFB012010BD1278EA
:100CF00000F124010A7000224A700122EDE7116818
:100D00004FF0FF32E9E70000074B70B50D467B441A
:100D1000FFF7CBFF0446284601F06CFA10B14FF004
:100D2000FF3070BD204670BD6F2001002DE9FF5FD0
:100D300015468A460446DFF8AC80F8440027D8E917
:100D400000103E46CDE9001010E03AF816106A4651
:100D500002A801F053FA411C07D02178890603D577
:100D6000E269391891420DD80744761C2078800634
:100D700002D5E069B84205DDAE42E6DB3AF816007E
:100D80000028E2D1A069C01BA0612046FFF734FB18
:100D9000D8E90010CDE90010002017E03AF818104B
:100DA0006A4602A801F02AFAB0F1FF3F81460BD053
:100DB00000250DF1080B05E0D4E901211BF8050021
:100DC00090476D1C4D45F7D308F10100B0428046B5
:100DD000E4DB206A384420622046FFF723FBBDE8AD
:100DE000FF9F0000626E01002DE9F0418046D21D98
:100DF00022F007020025D2E90002F52915A614D039
:100E0000011E72F1000106DA0023D0EB030063EB50
:100E1000020211A608E0D8F800108B0701D50FA632
:100E200002E0490701D50EA601251146002408F16C
:100E3000240704E000F0C0FB30323A55641C50EA4D
:100E40000102F7D12B46324621464046BDE8F0412B
:100E5000FFF7B8BE000000002D0000002B000000CE
:100E60002000000030B4002100F1240408E002F06A
:100E70000705D208303542EA4372DB086554491C45
:100E800052EA0305F3D10468002310A2250707D511
:100E9000A40600D421B1C46901230DA2641EC4615B
:100EA00030BCFFF78FBE10B5044621461068FFF72F
:100EB00080FE02462046BDE810400023D2E7D21D46
:100EC00022F00701D1E90023CCE700000000000078
:100ED000300000003A2800D2303820F02002412AA9
:100EE00001D3A2F13700884201D34FF0FF307047A1
:100EF0002DE9FF4F06468BB00878FF2806D0491C25
:100F00002D2805D000244FF0000908E000200CE057
:100F10000124F8E709EB8903491C00EB4309087831
:100F2000FF28F7D114B1C9F10000814610780025DF
:100F30002C46AA4629462D2801D02B2804D1521C24
:100F40002D2813D0002082468B461078FF280FD022
:100F50004FF0000C0A21521CA5FB017804FB018113
:100F600005FB0C11C5194BEB0104EEE70120EAE784
:100F7000002108464FF00000BAF1000F02D000EB4C
:100F800080004008C0F38157012F01DD4FF0FF378B
:100F90000E9955EA040009EB01080BD04FF0020945
:100FA00018F5FA7F16DA4FEACA70002F706008DD74
:100FB000012007E04FEACA70C6E900B00FB0BDE8F3
:100FC000F08F00203060FFF7CFFDC0F800901821AF
:100FD000084616E0B8F5FA7F18DD002F02DAF74868
:100FE000784401E0F6487844D0E90010C6E90010E2
:100FF00040EACA707060FFF7B7FDC0F80090142196
:1010000008460FB0BDE8F04F16F08FBC002108462F
:101010004FF00000B8F10001099002DAC7F10002B8
:1010200000E03A4601DAC8F1000106A801F070F8C4
:1010300006AB93E8070003AB83E8070044F23E00E9
:101040005BEA04010090584604D144F21E012C468C
:101050005D460091210C0904014306D10099240446
:1010600044EA15442D041039009104F07F410143F6
:1010700006D10099240244EA15642D020839009132
:1010800004F07041014306D10099240144EA15742B
:101090002D01091F009104F04041014306D1009940
:1010A000A40044EA9574AD00891E009104F000414B
:1010B000084304D100986D196441401E00904FF020
:1010C00001033A466846B8F1000FCDE9014503A98E
:1010D00002DD01F0BCFE01E001F08FFEBAF1000F6D
:1010E00004460D4601D084F00044002108464FF02C
:1010F0000000099940F2FF77484010F00C0F07D12B
:1011000024F00040284303D0C4F30A50B84212D15F
:10111000FFF72AFDC0F80090C4F30A50B8420AD184
:10112000A8487844D0E90010C6E9001004F0004156
:101130000843706042E7C6E900543FE72DE9FF4FDE
:101140001F464FF0000A4FF0FF38454691B0D7E9EF
:101150000146CDF83CA000F02BFAC0680168405C65
:101160001090B96912986D1C8847396A8146884782
:101170000028F6D1B9F1FF3F0AD0002E24F4D06444
:1011800011DDB9F12B0F08D0B9F12D0F0BD102E011
:10119000404615B013E744F48064B96912986D1C99
:1011A0008847761E8146600504A901D52D2000E000
:1011B0002B20002E01F1010B0DF130088DF81000ED
:1011C0003FDDB9F1690F08D0B9F1490F05D0B9F188
:1011D0006E0F02D0B9F14E0F1CD13B4601A800950D
:1011E00080E85002DDE912126FF0020016F008FCF0
:1011F000C11CCED10EE0B96912986D1C884781469A
:101200001398761E44F4007405600F98401C002E5D
:101210000F9016DDB9F1300FEDD0B9F1780F02D093
:10122000B9F1580F0DD10F9801280AD13B46CDE9ED
:101230000054DDE91212001F029616F0DFFBC11CFC
:10124000A7D1109989453ED144F0800406E0139956
:10125000681CAAF1010A44F400740860B9696D1CA5
:101260001298761E884730288146F0D02BE01099DE
:10127000894505D1200603D4761E44F0800418E089
:10128000484610F050F908B3761E0DF123018B4546
:1012900044F4007408D2A9F130000BF8010B2006C9
:1012A00007D5AAF1010003E0200602D40AF10100EB
:1012B0008246A00502D51399681C0860B969129886
:1012C0006D1C88478146002ED1DC53E0002E51DD95
:1012D000B9F1650F02D0B9F1450F4BD1A00549D541
:1012E000B9696D1C1298761E24F440748847002E4C
:1012F00081460CDD2B2804D0B9F12D0F07D144F421
:101300008074B96912986D1C8847761E8146E00585
:1013100001D52D2100E02B2108F8011BCDF800801C
:1013200021E0761E0DF13901884544F400740CD299
:10133000A9F1300010F0FF0088F8000002D10099F8
:10134000884509D908F1010806E0E00501D51E48E5
:1013500001E042F20F708246B96912986D1C88470D
:10136000814613980560002E04DD484610F0DBF836
:101370000028D6D1F96912988847FF2053468BF888
:10138000000088F8000000200A900B9004AA0CA925
:101390000AA8FFF7ADFDA00502D46FF00100F8E642
:1013A00014F0240F12D0E0071CD13868DDE90A12CE
:1013B000031D3B600068C0E9001213E0F8700100F3
:1013C000EA700100AE6F0100F1D8FFFF0AA968467C
:1013D00010F096F8E00705D13868009A011D3960D1
:1013E000006802602846D4E6026811441378016060
:1013F00018467047D16005497944516104497944E0
:10140000116200211161114600F0C8BCEDFFFFFF21
:1014100041020000426842B1016811F8013B23B16A
:10142000521EC0E90012184670470121C160881E93
:10143000704742685AB1C368016843B983688B42F8
:1014400005D0491E521CC0E90012002070474FF021
:10145000FF3070472DE9F05F824615468B46002726
:101460000AF10104B9460078302801D09DB113E09B
:1014700014F8010B0127782803D0582801D045B172
:101480000AE00DB1102D07D1002714F8010B10252B
:1014900002E0082500E00A250026B0460EE005FB24
:1014A000080005FB06F101271FFA80F801EB104642
:1014B000B6F5803F00D3B94614F8010B2946FFF773
:1014C00009FD0028EBDABBF1000F05D00FB1641E57
:1014D00000E05446CBF80040B9F1000F06D0FFF70A
:1014E00043FB02210160C81EBDE8F09F48EA0640A8
:1014F000FAE72DE9F04791460F468046044600265C
:1015000014F8015B2DB1FFF727FB0068405DC007B1
:10151000F6D12B2D02D02D2D18D0641E4A46394607
:101520002046FFF797FF27B13968A14201D1C7F8DC
:1015300000804FF0020471050BD54042002803DD06
:10154000FFF712FB0460A007BDE8F08746F4806651
:10155000E4E70028F8DAFFF707FB04606FF00040CB
:10156000F2E700002DE9F04115460E46040002D1D5
:101570002C6804B90BA4204600F070FE04442078C7
:1015800070B127463146384600F058FE04442078B2
:1015900010B1002004F8010B38462C60BDE8F08142
:1015A0000027F9E70000000000487047783B022060
:1015B00000487047983B022030B5B0F10A024FEA6C
:1015C000900E71F100034EEA817EB0EB0E0061EBEC
:1015D00091014FEA101E4EEA017E10EB0E0041EB26
:1015E00011114FEA102E4EEA016E10EB0E0041EB86
:1015F00011214FEA104E4EEA014E10EB0E0041EB66
:101600001141401841F100014FEAD00040EA417019
:101610004FEAD10110EB80054FEA810444EA90744F
:1016200044EB01046D1944EB0404521BA3414FF039
:10163000000348BF0A3200D530BD401C41F1000113
:1016400030BD10B50446FFF787FA0068005D00F072
:10165000010010BD70472DE9FF4F0C461E464FF0AC
:10166000FF378BB0D2E90001DDF860800A908A462E
:10167000C1F30A5505B93D46002108464FF0000068
:10168000BAF1000F00F4400005DA00EB80004FF4DF
:10169000400101EA50004FEA9059B9F1010F00DD15
:1016A000B9460A9850EA4A000ED044F61050A5F206
:1016B000FF3545432F14B8F1000F1ED07542291E87
:1016C0001EDDC9F100021CE0B8F1010F4FF000006F
:1016D00001D0302103E0F24305E02154401CB04228
:1016E000FBDB30460022002121540B99C1F8088011
:1016F000C1E900200FB0BDE8F08FBD1B6D1CDEE717
:101700004A4600DA694206A800F002FD06AB93E8FB
:10171000070003AB83E8070050460A9901F099F8E7
:101720008DE80700A0F500501F3800900398002DA9
:101730000ADD42F21F014A460844002303A9039030
:10174000684601F045FB09E0A0F500504A461F3805
:10175000002303A90390684601F064FB8DE80700AD
:101760000004000C03D04FF0FF30410800E01046A9
:10177000B8F1000F03D00022009215461EE0751E3E
:1017800005D4FFF719FF303262556D1EF9D5B34607
:101790000122084302D000227F1C04E02078302878
:1017A00001D100227F1E002A099784D01DE0112D4F
:1017B00007DAFFF701FF303262556D1C50EA010273
:1017C000F5D1084302D00098C8B10EE00021681E90
:1017D00005E0235C625C63542254401E491C814234
:1017E000F7DBAB46A81B401E0990002004F80B0055
:1017F0000B98099AC0F80880C0E9002B7AE71126F7
:101800004FF0000857E72DE9F04F88460446D21DF7
:1018100022F0070191B0D1E90001CDE90A010EF0F3
:101820000BF802460B98C00F01D02D2007E020686E
:10183000810701D52B2002E0202101EAC000032A04
:10184000099001D0072A05DB03464146204600F0F7
:1018500039FD0BE12078800601D5E06900E0062023
:10186000B8F1650F814606D0B8F1660F18D0B8F10F
:10187000670F70D131E00020B9F1110F009001DB4A
:10188000112301E009F101030AAA01A90CA8FFF73D
:10189000E2FEDDE90C70002609F10105834647E010
:1018A00001204B4600904FF000470AAA01A90CA85E
:1018B000FFF7D1FEDDE90DB00C995D46002610B9A9
:1018C00009F101000D18B9EB050003D4C0F1FF3692
:1018D00009F10105A5EB09002BE0B9F1010F01DACF
:1018E0004FF001090020B9F1110F0090484601DDC9
:1018F000112300E003460AAA01A90CA8FFF7ABFEDA
:10190000DDE90C704D4600268346207800070AD496
:10191000AB4500DA5D4601A8012D04DD411911F83F
:10192000011C302907D04F4502DA17F1040F04DA01
:10193000012082460FE06D1EEEE7002F02DCED1B5A
:101940003E4403E0781CA84200DD7D1CB81B00F17A
:10195000010A4FF000472078000703D4AA4501DBB5
:101960004FF0FF3A0021B7F1004F0DF143088DF819
:10197000431024D002202B23002F01DA7F422D2395
:101980000A21021EA0F1010000DC5FB197FBF1FC0F
:1019900097FBF1F201FB1C7C17460CF1300C08F8A8
:1019A00001CDEEE7A8F1010003702188090501D5FA
:1019B000452100E06521A0F1010800F8011C09980B
:1019C0000FA9A1EB0807FF1D00B10120411901EB90
:1019D000EA70A1693844081A401EA0612078C00648
:1019E00002D42046FEF708FD099828B1D4E9012168
:1019F0009047206A401C20622078C00622D52046ED
:101A0000FEF7FAFC1EE0002E04DBB34502DD01A860
:101A1000805D00E03020D4E901219047206A401C1D
:101A20002062761CAAF101005FEA000A0AD1FFF7E2
:101A3000BFFDC0680168405CD4E901219047206A7D
:101A4000401C2062281EA5F10105DCDC07E0D4E97A
:101A5000012118F8010B9047206A401C2062381EB3
:101A6000A7F10107F3DC2046FEF7DCFC032011B0F0
:101A700041E600002DE9F04F04460D46D21D22F04C
:101A8000070089B0D0E90097484639460DF0D4FEEA
:101A90000246F80F01D02D2307E02068810701D509
:101AA0002B2302E0202101EAC0038DF820300BB186
:101AB000012000E00020032A824601D0072A04DB2F
:101AC0002946204600F0FEFB3FE12078800601D445
:101AD0000D2500E0E569C7F30A560D2D49DA00210E
:101AE0004FEA175B08464FF00000002F00F440005B
:101AF00007DA00EB80004FF4400100EBD07001EA00
:101B000060008115012901DD4FF0FF3100224FEA0D
:101B1000850CBCF1180F06D31346ACF118004FF03A
:101B20008052C24003E04FF4801323FA0CF30CF10F
:101B30000C0CBCF1200F04D3ACF1200C09FA0CF012
:101B400001E007FA0CF000294FF0004801DD18B958
:101B50000FE00ED140450CD319EB02095F4121B9CA
:101B6000404502D19F4329EA0209BBEB175F00D031
:101B7000761C2088000502D57B48784402E07A482C
:101B80007844193808AA302302F80A30037C0AF195
:101B90000101002E0AF1020A53546A4602DC4FF09A
:101BA000300101E04FF031014FF001088DF80010D5
:101BB00002D0A6F2FF3603E059EA470100D06B4E8F
:101BC000002D02DC2178090704D54FF002082E21F0
:101BD0008DF80110C44600210BE0C7F303433F0119
:101BE000C35C491C6D1E02F80830052908F1010884
:101BF00001DA002DF1DC00210CE000EB1973491C27
:101C00001B786D1E082902F808304FEA091908F1FF
:101C1000010801DA002DF0DC21688B0602D516E000
:101C2000A8F10108E04505DD02EB080313F8013CCB
:101C3000302BF5D0B8F1000F09DD02EB080313F8E3
:101C4000013C2E2B03D1090701D4A8F10108002D76
:101C500005DD3E2102F808106D1E08F10108407CE8
:101C6000002E02F8080008F1010804DA2D2076425F
:101C700002F8080002E02B2002F808000A214FF4C5
:101C80007A70864208F101080BDB96FBF0F33033E3
:101C900002F8083096FBF0F308F1010800FB136628
:101CA00001E0642E0CDB642096FBF0F3303302F885
:101CB000083096FBF0F308F1010800FB136601E021
:101CC0000A2E06DB96FBF1F0303002F8080008F12E
:101CD000010896FBF1F001FB1060303002F80800BB
:101CE000A16908F1010808EB050202EB0A00081AD5
:101CF000A0612078C00602D42046FEF77DFB216A51
:101D000008AE01EB0A00206204E0D4E9012116F8D4
:101D1000010B9047BAF1010AF7D22078C00602D52C
:101D20002046FEF769FB6E4609E016F8010B3E28D7
:101D30000FD0D4E901219047206A401C2062B8F1FD
:101D40000108F2D22046FEF76DFB09B00320BDE882
:101D5000F08F206A2844206203E0D4E9012130207A
:101D600090476D1EEBD3F8E7C561010002FCFFFF51
:101D700010B5436913B1AFF3008001E0FEF7D6FF61
:101D8000012010BD128800F1240182840022C28447
:101D90000122EDE711684FF0FF32E9E72DE9F34F3B
:101DA0004FF0000A0C4656468DB001200C9001F110
:101DB0000C000B9062690B9801219047051E2DD0F5
:101DC000252D2CD0216A8847C0B162690B9801216A
:101DD0009047216A88470028F7D16269411E0B9815
:101DE000904700E0761CA1690D988847216A8847D2
:101DF0000028F7D1E1690D988847DBE7A1690D98C4
:101E00008847A842074601D1761CD3E7E1690D98BF
:101E100088477F1C02D1BAF1000F6FD06BE1626975
:101E20000B9800273D46394690472A2804D162691D
:101E30000B98012190470125DFF8D08262690B9849
:101E400001219047A0F130010A290AD24745E5DC7B
:101E500007EB870100EB4107303FDFD445F0100569
:101E6000ECE7E90601D46FF000476C280AD04C2853
:101E700014D0682815D06A280DD074281CD07A2870
:101E80001AD01DE062690B98012190476C2802D09E
:101E900045F0040514E045F002050DE045F020058D
:101EA0000AE062690B9801219047682802D045F04A
:101EB000080505E045F4006562690B98012190472B
:101EC000C4E9015765283DD019DC58287AD00CDCCC
:101ED000452837D004DC252826D041289ED131E082
:101EE00046282FD0472899D12CE05B2877D061284D
:101EF00028D063287CD0642823D15AE0F6E06F28EC
:101F000048D008DC66281DD067281BD0692821D05E
:101F10006E2816D127E0702845D0732868D0752820
:101F200047D078280DD14DE0A1690D988847252824
:101F300005463FF469AFE1690D9888476D1C3FF491
:101F40006AAFD8E00D9923466A466FF0010015F09C
:101F500053FDC5E045F0400023464FF000026060AD
:101F6000A80736D43EE0E8077FF447AF2068011D9C
:101F700021600068290501D506701BE7290701D5F6
:101F8000068017E7A90703D5F117C0E9006111E73B
:101F900006600FE745F0400023464FF008026060FE
:101FA000A80716D41EE040F60E0125EA0100606085
:101FB00016E045F0400023464FF00A026060A80793
:101FC00007D40FE045F040006060A80708D523461D
:101FD00010220D996FF00100AFF3008080E007E060
:101FE000102223460D996FF00100FEF7BDFB77E04C
:101FF0004FF0000963284F46C8464B46CB4602D0F7
:102000005B2806D038E0E80601D40120A060012753
:1020100032E06269D4F80CB00B98012190475E2839
:1020200007D14FF0010949466269D4F80CB00B980A
:102030009047216939B900210A4603AB43F82120B2
:10204000491C0829FADBD8B3216949B308F1010812
:1020500062690B98012190475D28F4D1B9F1000F16
:1020600009D0002003A951F82020D24341F82020B4
:10207000401C0828F7DB03AB2069002820794FEAD1
:1020800040701ED05B462246CDF80080CDE9019716
:102090000D9900286FF0010020DAAFF300801FE0F7
:1020A000C11703AA00EBD1614B1121F01F0102EB14
:1020B0008302411A13680120884003431360C7E775
:1020C00019E00D99224600286FF00100009702DA0E
:1020D000AFF3008004E0AFF3008001E0AFF30080D5
:1020E00000280ADA401C06D10C9820B14FF0FF30CE
:1020F0000FB0BDE8F08F5046FAE7E90701D10AF1C9
:10210000010A064400200C9054E60000CCCCCC0C14
:102110002DE9F047814616468AB0354878440DC807
:102120008DE80D0032487844801C03AC0DC884E86B
:102130000D0041F69B300844372190FBF1F290FBF3
:10214000F1F5A5F1800501FB12041B3C02D56442A8
:10215000012000E00020DFF898A080460027FA4424
:10216000AAF1BE0A0EE0E0070AD03246684607EB45
:10217000470101230AEB810100F054FE8DE80700BE
:1021800064107F1C002CEED1194F7F44AE3F19E044
:10219000E80715D007EB04100DF1180A90E80E00BF
:1021A0008AE80E00C068F04201D1981908903246C2
:1021B000012306A903A800F035FE03AB83E807005E
:1021C0006D10641C002DE3D14FF0010332466946C7
:1021D000B8F1000F03A802D000F0FAFD01E000F012
:1021E00021FEC9E90001C9F808200AB0BDE8F0875E
:1021F000B45C0100007B00F08000704770B51646AB
:102200000C460546FEF7A8FC036893F80101012877
:1022100006D0FF2C0FD8185D68B101202C7070BD5E
:10222000D3F807013246214603F207130344284638
:10223000BDE8704018474FF0FF3070BD30B5034621
:102240001D781DB10A4603E0AC4201D1181A30BD19
:1022500012F8014B002CF7D15B1CF1E730B50346B7
:102260001D783DB10A4612F8014B1CB1AC42FAD1BF
:102270005B1CF5E7181A30BD7546FFF795F9AE46B9
:1022800005006946534620F00700854618B020B582
:10229000FEF754F8BDE820404FF000064FF000076D
:1022A0004FF000084FF0000B21F00701AC46ACE8FE
:1022B000C009ACE8C009ACE8C009ACE8C0098D466B
:1022C000704700002DE9F0411F46044603260168CF
:1022D000072A01F4006004DB08B116A505E016A585
:1022E00003E008B115A500E015A521F0100020605D
:1022F000A069C01EA0610FB1401EA0612046FEF77C
:102300007BF84FB1D4E9012138469047206A401C40
:102310002062C01C206206E0206AFAE7D4E90121AD
:1023200015F8010B9047761EF8D22046FEF77AF892
:10233000BDE8F0814E414E006E616E00494E460090
:10234000696E66002DE9FF4F1F464FF03C0987B0CC
:102350004FF00042DDE9141001F10108DDF858A04A
:1023600002EA40500390002005908346054604464B
:102370000490B969461E08988847AAF1010A02909C
:10238000BAF1000F3BDD02982E2815D01021FEF780
:10239000A1FD00282EDB4FF0010B0599014317D05A
:1023A000B9F1000F0BDB4A46C11700F03FFA0543B5
:1023B0000C43A9F1040905E0012004900BE008B1E9
:1023C00045F0010501200590049820B9361D02E072
:1023D000049800B1361FB969089808F101088847C8
:1023E000BBF1000FAAF1010A0290C9D00999C1F806
:1023F0000080C5E70298702808D0502806D0F969F7
:1024000008988847BBF1000F14D04FE000200290DD
:102410000120BBF1000F049009D0B969089808F1B8
:1024200001088847AAF10109B9F1000F07DCF96931
:10243000089888476FF001000BB0BDE8F08F2B289B
:1024400004D02D280CD14FF0FF300490B9690898C2
:1024500008F101088847A9F10109B9F1000FE6DD8B
:10246000411CE4D00A21FEF735FD0028DFDB02998C
:1024700008F1010801EB810100EB41000290B9690C
:10248000089888470A21FEF725FD099AA9F1010954
:10249000B9F1000FC2F8008001DD0028E7DAF96920
:1024A000089888470499029800FB016655EA0400E1
:1024B00004D004F04041090002D006E0039898E0FF
:1024C000A40044EA9574AD00B61E04F00041080073
:1024D00002D16D196441761E159810F0240F03D0B7
:1024E0004FF00B095C4803E04FF028096FF07D00C6
:1024F0008246564507DAAAEB06018944B9F1410F35
:1025000001DD4FF0410901200021A9F1010200F095
:102510008DF9024628400B462140084301D0012195
:1025200000E00021501E029143F1FF31284021407C
:10253000084301D0012000E000200299834651EABF
:102540000B014FD0002108464FF00000039900F422
:10255000400039B100EB80004FF4400100EBD07037
:1025600001EA60008015012802DD4FF0FF3000E035
:1025700013D0401C36D0029860B3BBF1000F0CD1D1
:102580004A460120002100F051F92840214008432B
:1025900001D0012000E00020E0B101204A460021E6
:1025A00000F044F9034640190A4661412D1A8C4156
:1025B00011D3B9F1400F09DD159810F0240F02D0A6
:1025C000AAF1340603E0AAF1170600E0761C002504
:1025D0004FF0004406E05B1E42F1FF3220EA0305A3
:1025E00021EA0204CAF10100B04206DA1B4903984D
:1025F00008430190002000900EE0039AC4F3D32119
:10260000E80A0A43164940EA44500A433146CDE9F4
:10261000000268460EF07DFF159810F0240F0BD0D5
:102620001598C00715D13868DDE90012031D3B601D
:102630000068C0E900120CE002A869460EF060FFD5
:102640001598C00705D13868029A011D39600068E5
:1026500002604046F0E6000002FCFFFF0000F07F51
:102660000000F03F2DE9FF4F92461D4685B04FF028
:102670000041DDE9124BDDE914727F1E01EA4B5087
:10268000414940F0FF4940EA0108002122F02000C2
:102690004928049102D04E2828D04CE03BA00126C6
:1026A00007C88DE80700A9690698641C88477F1E43
:1026B000014606D41DF8060018B121F02001814220
:1026C0000BD0E96906988847032E34D0082E32D003
:1026D0006FF0010009B0BDE8F08F761C032E01D029
:1026E000082EE0D1601CCAF80000DCE7A969069852
:1026F000641C88477F1E2AD420F02000412826D160
:10270000A9690698641C88477F1E20D420F0200009
:102710004E281CD1A9690698641C88477F1E48F47E
:10272000002849F48009CAF8004001D4282806D0BE
:10273000E969069888475FEACB7012D022E0A96960
:102740000698641C88477F1E01D4002803DAE969D3
:1027500006988847BCE72928F1D1641CCAF80040D4
:10276000E9E71BF0240F07D028680499031D2B60AC
:102770000068C0E9001805E02868021D2A600068AA
:10278000C0F800902046A5E70000F07F494E46497A
:102790004E4954590000000010B50446AFF30080C4
:1027A0002046BDE81040FDF7B2BD00004FF0013CEF
:1027B00050F8042B51F8043B9A4221D1A2EB0C03B0
:1027C000934313EACC1317D150F8042B51F8043B70
:1027D0009A4215D1A2EB0C03934313EACC130BD10D
:1027E00050F8042B51F8043B9A4209D1A2EB0C0398
:1027F000934313EACC13DBD04FF00000704700BFC7
:10280000D01A01BAB1FA81F101F0180122FA01F0EF
:10281000CB40C1F12001DBB2C0B2C01A2CFA01F3E7
:10282000D11A914311EAC311E6D17047B2F12003E6
:102830000AD5C2F1200301FA02F120FA03F300FAEB
:1028400002F041EA0301704700FA03F14FF0000083
:1028500070475FEA400C08BF91F0000F4FEA8C23ED
:102860004FEAC12243EA51514FEA1C5018BF00F50C
:10287000F0404FEA300018BF41F000415FEA6C5C65
:1028800000F02980BCF1FF3F08BF40F08040704756
:10289000130C06BF12044FF0100C4FF0000C130E77
:1028A00004BF12020CF1080C130F04BF12010CF14B
:1028B000040C930F04BF92000CF1020CD30F04BF61
:1028C00052000CF1010C11464FF00002A0F11F0064
:1028D000A0EB0C00704711F0004F08BF704731F0BB
:1028E00000413FF4D5AF0B0C06BF09044FF0100CAC
:1028F0004FF0000C0B0E04BF09020CF1080C0B0F7B
:1029000004BF09010CF1040C8B0F04BF89000CF10A
:10291000020CCB0F04BF49000CF1010CCCF12003D9
:10292000A0EB0C0022FA03F302FA0CF241EA0301D5
:1029300000F10100704720F07F4C80EA030023F093
:102940007F47ACEB070303F57C5300F0004003F135
:10295000FF032DE980494FEA154B09B44FEA1443B0
:1029600025EA0B4E24EA03480FF2042606EB132750
:1029700049083E785FEA320203FB0667C7F50007A5
:1029800007FB06F64FEA54374FEAD64606F1020631
:1029900007FB066CCCF1005C4FEA1C472CEA074CA5
:1029A00007FB06F40CFB06F504EB15464FEA9616FA
:1029B00034BF00204FF000404FEAD13706FB07FC40
:1029C0004FEA1C4C0CFB0BF7D21B03FB0CF761EB23
:1029D00007010CFB0EF7B0EB074072EB17420CFB44
:1029E00008F734BFA2EB0742B2EB074261EB174195
:1029F0004FEA0C444FEA910706FB07FC4FEA1C4CD8
:102A00000CFB0BF7B0EBC74072EB573203FB0CF734
:102A100034BFA2EBC742B2EBC74261EB57310CFBAC
:102A20000EF7B0EBC70072EB57720CFB08F734BF20
:102A3000A2EBC702B2EBC70261EB5771039F4FEAEB
:102A4000816141EA921104EBCC044FEAD1374FEA9D
:102A5000826206FB07FC42EA90124FEA80604FEA6E
:102A60001C4C0CFB0BF7D21B03FB0CF761EB0701B3
:102A70000CFB0EF7B0EB074072EB17420CFB08F7AC
:102A800034BFA2EB0742B2EB074261EB17414FEABA
:102A90008C554FEA910704EB9C2406FB07FC4FEA98
:102AA0001C4C0CFB0BF7B0EBC74072EB573203FB2F
:102AB0000CF734BFA2EBC742B2EBC74261EB573110
:102AC0000CFB0EF7B0EBC70072EB57720CFB08F76C
:102AD00034BFA2EBC702B2EBC70261EB577115EB33
:102AE0004C254FEA816141EA92114FEA82624FEA36
:102AF000D13742EA901206FB07FC44F100044FEA8A
:102B000080604FEA1C4C0CFB0BF7D21B03FB0CF74D
:102B100061EB07010CFB0EF7B0EB074072EB1742BD
:102B20000CFB08F734BFA2EB0742B2EB074261EBA4
:102B3000174115EB1C154FEA813141EA92414FEAEA
:102B4000823242EA90424FEA80304FEA0C7644F1FA
:102B5000000448EA03434EEA0B484FF0000EB2EB84
:102B6000080C71EB030724BF624639464EEB0E0E8C
:102B70004FF0000B0018524149414BEB0B0BB2EBED
:102B8000080C71EB03077BF1000B24BF624639464A
:102B90004EEB0E0E4FF0000B0018524149414BEB2B
:102BA0000B0BB2EB080C71EB03077BF1000B24BF9E
:102BB000624639464EEB0E0E51EA020718BF46F048
:102BC000010616EB0E7655F1000254F1000103D513
:102BD000BDE88901BDE80088BDE88901BDE800487D
:102BE000B619524141EB0101A3F101037047808006
:102BF0007F7E7D7C7B7A7978777676757473727157
:102C000071706F6E6E6D6C6C6B6A6A69686867660E
:102C100066656464636362616160605F5F5E5E5DA0
:102C20005D5C5C5B5B5A5A59595858575756565514
:102C300055555454535352525251515050504F4F76
:102C40004F4E4E4D4D4D4C4C4C4B4B4B4A4A4A49C6
:102C50004949484848474747474646464545454409
:102C600044444443434343424242424141410000C1
:102C700046EA0646A3F570534FEA164646EA425620
:102C80004FEAD22242EA415210B54FEAD121A3F1D4
:102C9000010300F02FF820F0004000F1020C00F0DA
:102CA000004701EB00501146BCF5006F40EA0700F9
:102CB00000D210BDBAF1000F0AD01CB503B44FF01A
:102CC00004004FF004014FF000000FBCBDE81040BD
:102CD0004FF00001BBF1010FB9BF04484FF0FF31C5
:102CE0000348002140EA070010BD00BFFFFFEF7F4F
:102CF0000000F07F002B9C4630D477002BD01CB511
:102D00004FEA370703B44FF010004FF01001BAF14B
:102D1000000F06D0BCF1000FDCBF40F0080040F00F
:102D200008014FF000000FBCBDE810400BF1010B93
:102D3000BBF1010F08BF5FEA170722BF12F10102C2
:102D400011F101014FF0004143F1000300F0004098
:102D500043EA00007047F9D35708D0E746EA064631
:102D600013F1400F4FEA16461FDD13F1200FDFBFAE
:102D700016430A46002120335B42BED0C3F1200730
:102D800046EA064602FA07F74FEA164646EA0706FB
:102D9000C3F1200722FA03F201FA07F721FA03F13F
:102DA0004FF0000342EA0702A7E746EA020646EAB6
:102DB00006464FEA164646EA0106BCBF46EA064604
:102DC000360C4FF000034FF000024FF0000194E783
:102DD0002DE9804C9A46934670B491E8380007C8B4
:102DE00031EA400C48BF34EA430C03D5FFF7A3FD9A
:102DF000FFF780FFF0BCBDE8008C2DE9804C9A46BF
:102E0000934670B491E8380007C831EA400C48BFD7
:102E100034EA430C03D5FFF78EFDFFF729FFF0BC22
:102E2000BDE8008C2DE9804C9A46934670B491E839
:102E3000380007C810F0804F08BF13F0804F03D14F
:102E400000F01AF8FFF756FFF0BCBDE8008C2DE942
:102E5000804C9A46934670B491E8380007C810F049
:102E6000804F08BF13F0804F03D100F005F8FFF743
:102E7000FFFEF0BCBDE8008C20F07F4780EA030035
:102E800023F07F4C07EB0C03A3F57C5300F00040CC
:102E9000A3F1FE0392F0000F00F0B38095F0000F55
:102EA00000F077802DE901494FEA11404FEA1446BE
:102EB00021EA004800FB06FC24EA064708FB06F668
:102EC00007FB08F800FB07F718EB06484CEB164C1D
:102ED0004FEA124B18EB07484FEA15464CEB1740E8
:102EE00022EA0B4E0BFB06FC25EA06470EFB06F614
:102EF00007FB0EFE0BFB07F71EEB064E4CEB164CCA
:102F00004FF000061EEB074E4CEB174B18EB0B086F
:102F100040F1000018EB0E0B58EB000840F10000E8
:102F20008F1A4FF000013CBFC943661B14BFB5EBBD
:102F3000040C00213CBFC943F61B4FEA17444EEA7C
:102F40008E0E27EA04454FEA1C4704FB07622CEA71
:102F5000074C05FB07F70CFB05F604FB0CFC16EB16
:102F6000074642EB174216EB0C4642EB1C421BEBAA
:102F7000060658EB0202414146EA9E0601D5BDE82D
:102F80000189B619524141EB0101A3F10103BDE8EA
:102F900001894FEA14454FEA114724EA054621EA20
:102FA000074C05FB07F406FB07F70CFB06F105FBD6
:102FB0000CFC11EB074144EB17444FEA124711EBAD
:102FC0000C4144EB1C4422EA074C05FB07F206FBCC
:102FD00007F70CFB06F605FB0CFC16EB074642EB6D
:102FE000174216EB0C4642EB1C456A1854F10001DF
:102FF00048BF7047B619524141EB0101A3F10103EB
:10300000704795F0000F37D04FEA11424FEA14474E
:1030100021EA024624EA074C02FB07F106FB07F708
:103020000CFB06F402FB0CFC14EB074441EB1741CC
:103030004FEA154714EB0C4441EB1C4125EA074CC1
:1030400002FB07F506FB07F70CFB06F602FB0CFC80
:1030500016EB074645EB174516EB0C4645EB1C42B5
:10306000121951F1000148BF7047B619524141EBA6
:103070000101A3F1010370474FEA14454FEA1147DC
:1030800024EA054621EA074C05FB07F106FB07F792
:103090000CFB06F24FF0000605FB0CFC12EB07429E
:1030A00041EB174112EB0C4251EB1C4148BF7047FA
:1030B000921841EB0101A3F10103704721484FF041
:1030C000FF010170002080F309881F48016881F327
:1030D00008881E484FF08051016062B6FEE71B4829
:1030E0004FF080510160704718484FF080510160E7
:1030F000704772B6EFF3098050B11EF0100F08BF91
:1031000020ED108A734620E9F80F1149096808601C
:1031100000B5104880475DF804EB0F480F490A7866
:1031200002700B480E490A6802601068B0E8F80F98
:103130009E461EF0100F08BFB0EC108A80F309887D
:1031400062B6704722ED00E0F007002004ED00E0D9
:10315000E8070020D18B0008D2070020D307002009
:10316000EC07002000B52DED048B8DB0824890F85F
:10317000250020B90121084606F09EFB10E0C8207A
:1031800005F0F6F97D4908700846007820B1012164
:10319000084606F091FB03E00021012006F08CFBBD
:1031A0007748007980BB012076490870012108200A
:1031B00006F082FB0020744948707449744810F08E
:1031C00049F84FF47A71022003F03EFA01206C496D
:1031D0004872084690F88D0060B103F07FFD6848A2
:1031E000B0F8A80000F4807008B904F0BBFF11F03B
:1031F000D9FDBDE00EF0ACFD11F0F6FD0EF0EEFFD6
:1032000000205F49C862B3E0FFE75E48007830B154
:103210000021082006F050FB00205A49087009F0F0
:10322000C7FC5749D1F8A8000EF086F9B8B1544848
:1032300024300EF07FFF11F0B5FD514991ED000AE9
:10324000BDEEC00A10EE100A10F01CFE00EE100ACF
:10325000B8EEC00A4A4880ED000A0EF019FC484852
:10326000D0F8A800B0F5007F04D04548D0F8A800F9
:10327000402803D111F096FD0EF06AFD404890F809
:10328000BA0078B33C48406840F2CA31884203D063
:1032900039484068E63028B9374800684CF6406144
:1032A000884210D03448006844F67C41884205D0FA
:1032B0003148006845F22211884207D12E48406803
:1032C0003449884202D104F05FFC01E003F0F0FED3
:1032D0002B48B0F8A80000F4807008B904F042FF51
:1032E00011F060FD2C4801680068401C2A4A1060FB
:1032F00032293DDD0020114608601F4890ED030A89
:1033000010EE101A084614F095FA41EC180B1A4802
:1033100090ED020A10EE101A084614F08BFA41ECF8
:10332000190B8DED0A8B8DED089B154890F8240044
:103330001349897F124AD2F8A820184B5B69CDE95E
:103340000332CDE90510154890ED010ABDEEC00A23
:10335000007C0B49897CCDE900108DED020A0848FC
:1033600090F8BB3090F8BD200D4901200BF0B6FC61
:103370000DB0BDEC048B00BDD432012058030020F9
:103380005439022059030020408901202C3B02209F
:10339000783A0220BAF5FFFF5C0300206833012071
:1033A000EC7D01080246642A04D101232C4880F8F0
:1033B0008F3003E000232A4880F88F30752A04D12B
:1033C0000123274880F88E3003E00023244880F84A
:1033D0008E30652A03D0642A01D0752A01D10020DD
:1033E0007047662A03D1612901D10320F8E7662AD4
:1033F00003D1632901D10420F2E7662A03D16D29A4
:1034000001D10120ECE7622A03D1612901D1052015
:10341000E6E7622A03D1632901D10620E0E7622AA8
:1034200003D16D2901D10220DAE7662A03D16C2984
:1034300001D10720D4E7622A03D16C2901D10920E8
:10344000CEE7662A03D1722901D10820C8E7622A93
:1034500003D1722901D10A20C2E70020C0E7000091
:103460005439022010B502460B460021002000BF4F
:1034700004E0545C0444A0B24C1CA1B29942F8DBB5
:1034800010BD000008B538E01C4890F8250018B1C0
:1034900001211B4806F070FA184890F8271090F8A0
:1034A0002700401E154A82F827000A2903DA002067
:1034B000114681F82500134890F8250018B1012124
:1034C000114809F091FA0F4890F8271090F827005A
:1034D000401E0C4A82F827000A2907DA002011460C
:1034E00081F825002C211046FDF70BFB0CF016F897
:1034F0006A460821022005F06DFBC5E7D4320120A1
:10350000AC2A012000330120242B012010B58AB001
:1035100004463E480078052817D109A80321002257
:103520000592CDE90621089010464FF480711922CA
:10353000374BCDE90132CDE9031002200023354A93
:1035400035A10090394805F095F909A8032100221A
:103550000592CDE90621089010464FF40061CC2277
:10356000334BCDE90132CDE903100A200023314A63
:1035700031A10090364805F07DF909A80721002205
:103580000592CDE90621089010464FF40061CC2247
:10359000304BCDE90132CDE90310042000232E4A3F
:1035A0002EA10090314805F065F909A803210022F9
:1035B0000592CDE90621089010464FF40061CC2217
:1035C0002B4BCDE90132CDE9031006200023294A17
:1035D00029A100902E4805F04DF903200021059106
:1035E000CDE90704069108464FF40061CC22294B2F
:1035F000CDE90132CDE9031005200023264A27A199
:1036000000902B4805F036F90AB010BD9801002053
:10361000382A002011370008417070205461736B04
:103620002046656564446F6700000000D0290020D3
:10363000A02E0020D5360008417070205461736BB5
:103640002045746865726E657420536572000000D1
:10365000382E0020D88F002085340008417070205B
:103660005461736B2043414E00000000708F0020B6
:10367000084F0020B5360008417070205461736B0C
:103680002045746865726E657420436C69000000A3
:10369000A04E002040B00020293700084170702063
:1036A0005461736B2053706565642043747200002D
:1036B000D8AF002008B509E00EF062F80449C1F85F
:1036C00004016A460821012005F084FAF4E70000AD
:1036D0005439022008B50AF0EDFB15E00EF062FF48
:1036E0000A48B0F8A80000F4005040B10AF0E2FB2C
:1036F0000020064908734FF4005009F073FC6A4635
:1037000008211E2005F066FAE8E70000543902207F
:1037100008B50EF05BF806E001F058FE6A4600219D
:103720000A2005F057FAF7E708B50AE00BF070FB3E
:103730000BF08CFF0BF080FB6A4608210A2005F095
:1037400049FAF3E710B52DED048B374890ED000AE8
:10375000B8EEC00A3548D0ED000AB4EE600AF1EECA
:1037600010FA5ED1304890ED010AB8EEC00A2F4839
:10377000D0ED010AB4EE600AF1EE10FA51D12C48F6
:10378000817F2C484068401E814225DB284890F804
:103790002400022820D1244890ED020A10EE101ACD
:1037A000084614F047F841EC190BB0EE490AF0EE68
:1037B000690A0CF039F9B0EE408AF0EE608A9FEDAC
:1037C0001E0B53EC102B51EC180B13F001FD28D2FB
:1037D0000120BDEC048B10BD134890ED020A10EEE1
:1037E000101A084614F026F841EC190BB0EE490AFD
:1037F000F0EE690A0CF018F9B0EE408AF0EE608A3B
:103800009FED0F0B53EC102B51EC180B13F0E0FC59
:1038100007D20748C27F0CA101200BF05FFA0120FC
:10382000D7E70020D5E70000D4320120183B022062
:10383000543902204089012000000000000014409B
:103840000000000000002E40D5FDB3A3B5BDB4EFCD
:10385000202025640D0A00001FB5684609F0F2F922
:10386000019804B010BD00002DE9F041FFF7F4FF0E
:10387000054614480068B5FBF0F42146481EB0F137
:10388000807F00D31BE0481E4FF0E02250615017AC
:103890000F22002807DA13071F0E0B4B00F00F064C
:1038A000361F9F5503E013071E0E084B1E5400BF22
:1038B00000204FF0E02290610720106100BFBDE8BA
:1038C000F0810000947A010818ED00E000E400E0C7
:1038D00038B50025404890F8360708283DD008DC68
:1038E00001280FD002280ED0032815D0042870D14B
:1038F00029E00B2830D020285BD0212849D0272868
:1039000067D13DE065E035480223012200210090A7
:10391000084601F065FC5CE03048032301220021E9
:103920000090084601F05CFC2D48D0F8A8102DA0AE
:1039300006F00EF8044606230022114600900120EE
:1039400001F04EFC45E025480423012200210090AF
:10395000084611F0DFFB3CE03BE01F48D0F8380799
:1039600010B1012802D100E000E000BF00BF1B48F9
:103970000823012202210090002011F0CBFB28E057
:1039800016482723012200210090084611F0C2FBAF
:103990001FE012482123012200210090084611F067
:1039A000B9FB124A51680C4AD2F838070EF088FC6D
:1039B0000FE00A482023012200210090084611F060
:1039C000A9FB0A4A5168044AD2F838070EF020FDD4
:1039D00000BF00BF38BD0000F81B0220A81D022058
:1039E00054390220253034780000000030230220B2
:1039F00000BFFEE730B58BB004460D4601210846F6
:103A000009F0F0F80121480609F0FCF84FF4C05025
:103A1000099002208DF8280000208DF82A0003204C
:103A20008DF8290001208DF82B0009A9534801F0D9
:103A3000DFFC09220B21514801F022FD09220C2153
:103A40004E4801F01DFD00208DF81E0001208DF86C
:103A50001F0000208DF820008DF821008DF8220035
:103A60008DF823008DF81A50052C45D2DFE804F0BC
:103A700003101D2A370000208DF81B0006208DF84A
:103A80001C0005208DF81D001E20ADF8180040E038
:103A900000208DF81B0006208DF81C0005208DF8F5
:103AA0001D001820ADF8180033E000208DF81B0031
:103AB00006208DF81C0005208DF81D000F20ADF8A4
:103AC000180026E000208DF81B0006208DF81C0051
:103AD00005208DF81D000C20ADF8180019E000201D
:103AE0008DF81B0006208DF81C0005208DF81D00A8
:103AF0000620ADF818000CE000208DF81B00062011
:103B00008DF81C0005208DF81D000620ADF818006A
:103B100000BF00BF06A91A4800F04DFC00208DF838
:103B200012008DF8130001208DF814000020ADF86C
:103B30000800ADF80A00ADF80C00ADF80E00ADF8C5
:103B4000100001208DF8150002A800F017FB0122DB
:103B500002210B4800F026FC14208DF804000120FF
:103B60008DF8050000208DF8060001208DF8070073
:103B700001A804F0B7FC00200BB030BD00000240EB
:103B80000064004030B585B00025002400BF00BFB0
:103B9000FCF7E8FB044600BF00BF04F075FD00BF62
:103BA00000BF2046FCF7E2FB00BF00BF022118481F
:103BB00000F068FB20B36A460021154800F085FC40
:103BC00040F281510098884202D1684602F008FF15
:103BD00040F282510098884202D1684609F00CFAFE
:103BE00040F283510098884202D1684602F0B4FF47
:103BF00040F284510098884202D1684609F0B8FA30
:103C000000200090019004F055FD05B030BD00008B
:103C1000006400402DE9F04786B007468846164606
:103C200099464FF0140A00250097122001900020B9
:103C30008DF808008DF809008DF80A6000BF05E0D6
:103C400018F805100DF10B0041556D1CB542F7D366
:103C50001DE06946134800F0B0FC0446042C0FD068
:103C600006E05046411E01F0FF0A012800DA05E097
:103C700021460C4800F034FD0028F2D000BF07E0D8
:103C80005046411E01F0FF0A012800DA00E0E0E79B
:103C900000BF05AA0821484604F09CFF002006B09A
:103CA000BDE8F0870064004010B5002400BF00BFED
:103CB000FCF758FB044600BF00BF04F0E5FC00BF62
:103CC00000BF2046FCF752FB00BF00BF0121154892
:103CD00000F000FA0121134800F0D4FA012804D1C1
:103CE0000121104800F0F6F914E001210D4800F020
:103CF000C9FA012804D101210A4800F0EBF909E0D2
:103D00000121084800F0BEFA012803D1012105482D
:103D100000F0E0F900220121024800F043FB04F02A
:103D2000C9FC10BD0064004030B58BB004460D46A0
:103D30000121022008F056FF01214FF0C06008F079
:103D400061FF6020099002208DF8280000208DF886
:103D50002A0003208DF8290001208DF82B0009A9E5
:103D6000544801F045FB09220521524801F088FB27
:103D7000092206214F4801F083FB00208DF81E0028
:103D800001208DF81F0000208DF820008DF8210003
:103D90008DF822008DF823008DF81A50052C45D29D
:103DA000DFE804F003101D2A370000208DF81B0007
:103DB00006208DF81C0005208DF81D001E20ADF892
:103DC000180040E000208DF81B0006208DF81C0034
:103DD00005208DF81D001820ADF8180033E00020F4
:103DE0008DF81B0006208DF81C0005208DF81D00A5
:103DF0000F20ADF8180026E000208DF81B000620EB
:103E00008DF81C0005208DF81D000C20ADF8180061
:103E100019E000208DF81B0006208DF81C000520FD
:103E20008DF81D000620ADF818000CE000208DF87C
:103E30001B0006208DF81C0005208DF81D000620B3
:103E4000ADF8180000BF00BF06A91B4800F0B3FA88
:103E50000E208DF8120000208DF8130001208DF83F
:103E600014000020ADF80800ADF80A00ADF80C0011
:103E7000ADF80E00ADF8100001208DF8150002A875
:103E800000F07CF9012202210B4800F08BFA40205F
:103E90008DF8040001208DF8050000208DF8060043
:103EA00001208DF8070001A804F01CFB00200BB0D6
:103EB00030BD0000000402400068004030B585B00D
:103EC0000025002400BF00BFFCF74CFA044600BFE9
:103ED00000BF04F0D9FB00BF00BF2046FCF746FA44
:103EE00000BF00BF0221344800F0CCF900285CD0AC
:103EF0006A460021304800F0E8FA0098B0F5007FEB
:103F000029D19DF80C009DF80B1040EA012000EE2D
:103F1000100AB8EEC00A294880ED3E0A9DF80E103E
:103F20009DF80D0041EA002001B22448A0F8FC10E1
:103F30009DF812109DF8110041EA00211F48A0F8D9
:103F40000211B0F8020140F6B831884203DD0021C9
:103F50001A4880F8FE1040F201210098884213D1DF
:103F60009DF812109DF8110041EA00211348A0F8B5
:103F7000001190F8FE0038B11048B0F80001801E22
:103F800081B20E48A0F8001140F202210098884248
:103F90000BD19DF80B10094880F8FF1090F8FF0036
:103FA00018B10021054880F8FE1000200090019013
:103FB00004F080FB05B030BD006800405439022099
:103FC0002DE9F04786B007468846164699464FF0D9
:103FD000140A002500971220019000208DF8080097
:103FE0008DF809008DF80A6000BF05E018F805108B
:103FF0000DF10B0041556D1CB542F7D31DE069462C
:10400000134800F0DAFA0446042C0FD006E05046BC
:10401000411E01F0FF0A012800DA05E021460C48A4
:1040200000F05EFB0028F2D000BF07E05046411EC2
:1040300001F0FF0A012800DA00E0E0E700BF05AA6E
:104040000821484604F0C6FD002006B0BDE8F08710
:104050000068004010B5002400BF00BFFCF782F9E3
:10406000044600BF00BF04F00FFB00BF00BF2046A6
:10407000FCF77CF900BF00BF0121154800F02AF8C9
:104080000121134800F0FEF8012804D10121104855
:1040900000F020F814E001210D4800F0F3F80128A9
:1040A00004D101210A4800F015F809E0012108486F
:1040B00000F0E8F8012803D10121054800F00AF8D2
:1040C00000220121024800F06DF904F0F3FA10BD5E
:1040D00000680040B1F5007F3AD00FDC202928D0DD
:1040E00006DC01291CD004291DD0082940D11DE07F
:1040F000402921D0B1F5807F3AD126E0B1F5004FBB
:1041000031D006DCB1F5806F25D0B1F5006F2FD12D
:1041100024E0B1F5803F12D0B1F5003F28D111E085
:10412000154A826025E00822C26022E01022C260A7
:104130001FE0082202611CE01022026119E008223F
:10414000426016E01022426013E00422426010E058
:10415000042242600DE0042242600AE000228261F3
:104160000422426005E0002282610422426000E0F5
:1041700000BF00BF704700000101010010B5002121
:10418000837A012202FA03F13D4A126842F00102E9
:104190003B4B1A603A4A1C3212688A43384B1C3334
:1041A0001A60027BCAB9364A0C3212688A43344B11
:1041B0000C331A604288C38842EA0343304A4032D3
:1041C000847A42F834300288838842EA03432C4AD6
:1041D0004032847A02EBC4025360027B012A19D177
:1041E000274A0C3212680A43254B0C331A60428866
:1041F000038842EA0343224A4032847A42F8343048
:10420000C288838842EA03431D4A4032847A02EB23
:10421000C4025360C27A3AB9194A121D12688A431D
:10422000174B1B1D1A6006E0154A121D12680A433F
:10423000134B1B1D1A60028932B9114A14321268DD
:104240008A430F4B14331A600289012A06D10C4AA3
:10425000143212680A430A4B14331A60427B012A53
:1042600006D1074A1C3212680A43054B1C331A60F8
:10427000034A126822F00102014B1A6010BD0000CF
:104280000066004070B504460D460026606928406F
:10429000002871D0B5F5807F5CD010DC082D35D0BA
:1042A00006DC012D20D0022D24D0042D72D127E070
:1042B000102D31D0202D35D0402D6BD138E0B5F503
:1042C000004F60D009DCB5F5007F49D0B5F5806FAF
:1042D0004CD0B5F5006F5DD14FE0B5F5803F2DD0E6
:1042E000B5F5003F56D12FE0A0682D4900F004FF3E
:1042F000064651E0E068032100F0FEFE06464BE072
:10430000E068082100F0F8FE064645E0E06810216C
:1043100000F0F2FE06463FE02069032100F0ECFECB
:10432000064639E02069082100F0E6FE064633E043
:104330002069102100F0E0FE06462DE060680821AB
:1043400000F0DAFE064627E06068102100F0D4FE97
:10435000064621E0A069012100F0CEFE06461BE0E2
:10436000A069022100F0C8FE064615E0A0690421FC
:1043700000F0C2FE06460FE00FE0A069702100F0D9
:10438000BBFE064608E06068042100F0B5FE064664
:1043900002E0FFE7002600BF00E00026304670BDC7
:1043A000010101001AB143690B43436102E0436913
:1043B0008B434361704730B50246002000231468E8
:1043C00024F002041460146844F00104146000E056
:1043D0005B1C546804F001041CB94FF6FF74A3423F
:1043E000F6D1546804F001040CB900206CE08C791B
:1043F000012C04D1146844F08004146003E01468B4
:1044000024F080041460CC79012C04D1146844F0A9
:104410004004146003E0146824F0400414600C7A33
:10442000012C04D1146844F02004146003E01468E3
:1044300024F0200414604C7A012C04D1146844F058
:104440001004146003E0146824F0100414608C7AE3
:10445000012C04D1146844F00804146003E01468CB
:1044600024F008041460CC7A012C04D1146844F0C0
:104470000404146003E0146824F0040414608C78CD
:10448000A407CD7844EA05640D7944EA05444D79E2
:1044900044EA05540D886D1E2C43D461146824F041
:1044A00001041460002300E05B1C546804F0010464
:1044B0001CB14FF6FF74A342F6D1546804F0010416
:1044C0000CB1002000E0012030BD10B500F5D8731C
:1044D00003EB01131B6803F004031372137A53B93F
:1044E00000F5D87303EB01131B6840F2FF7404EA74
:1044F0005353136009E000F5D87303EB01131B68F5
:104500006FF0604404EAD303536000F5D87303EB03
:1045100001131B6803F00203537200F5D87303EB19
:1045200001135B6803F00F03937200F5D87303EB7C
:1045300001135B681B0AD37400F5D87303EB0113F6
:104540009B68D37200F5D87303EB01139B681C0AB8
:10455000147300F5D87303EB01139B681C0C5473A0
:1045600000F5D87303EB01139B681B0E937300F5E2
:10457000D87303EB0113DB68D37300F5D87303EB37
:104580000113DB681C0A147400F5D87303EB0113E4
:10459000DB681C0C547400F5D87303EB0113DB6863
:1045A0001B0E937421B9C36843F02003C36003E07A
:1045B000036943F02003036110BD10B502460020DB
:1045C000936803F08063B3F1806F00D110E09368CB
:1045D00003F00063B3F1006F01D1012008E093689C
:1045E00003F08053B3F1805F01D1022000E004208A
:1045F000042874D002F5C07303EB00131B6803F0AA
:10460000010402F5C07303EB00131C600B7A7BB945
:104610004B7A0C8843EA445302F5C07404EB00144F
:104620002468234302F5C07404EB0014236010E0F7
:104630000B7A4C6843EAC4034C7A234302F5C074F6
:1046400004EB00142468234302F5C07404EB001447
:1046500023608B7A03F00F038B7202F5C07303EBB8
:1046600000135B6823F00F0402F5C07303EB001323
:104670005C6002F5C07303EB00135B688C7A234324
:1046800002F5C07404EB001463608B7B1C064B7B4B
:1046900044EA03440B7B44EA0323CC7A234302F528
:1046A000C07404EB0014A3608B7C1C064B7C44EAB2
:1046B00003440B7C44EA0323CC7B234302F5C07400
:1046C00004EB0014E36002F5C07303EB00131B68F6
:1046D00043F0010402F5C07303EB00131C6010BD2E
:1046E00010B50246002321B1012907D002290FD1BC
:1046F00009E090681D4C00EA04030BE090681C4C34
:1047000000EA040306E090681A4C00EA040301E0A2
:10471000002300BF00BF184C181BA34216D007DCB3
:1047200083B16FF08060184470B1022818D111E095
:10473000B0F5007F10D0114C204448B1B0F5003FD7
:104740000ED10BE002230DE000230BE0002309E073
:10475000002307E0012305E0012303E0012301E03A
:10476000002300BF00BFD8B210BD0000030000044A
:104770000003000800000310000100080001FFF71B
:1047800010B500F01FF800F019F810BD10B50024A6
:1047900000BF00BFFBF7E6FD044600BF00BF1021CD
:1047A000054803F031FE00BF00BF2046FBF7DEFDE9
:1047B00000BF00BF10BD000040D0002010B5FFF7C3
:1047C000E5FF10BD10B500200249086000F00AF8AE
:1047D00010BD0000C40700200149086070470000B8
:1047E000C407002010B5FFF737F8044608480068F2
:1047F00040F080700649086000200649486008467D
:10480000006840F0010008602046FFF7E5FF10BD9A
:10481000FCED00E0001000E001494868704700002E
:10482000001000E0F0EE400A9FED3D0AF4EEC00AF1
:10483000F1EE10FA05DD9FED3B0A30EEC00AF0EE16
:10484000400A9FED390AF4EEC00AF1EE10FA05D2E3
:104850009FED340A30EE800AF0EE400AB2EE040A10
:10486000F4EEC00AF1EE10FA0CD2BAEE040AF4EE3D
:10487000C00AF1EE10FA05DD9FED2C0A2C4880ED00
:10488000000A48E09FED2B0AF4EEC00AF1EE10FAA0
:104890000CD29FED290AF4EEC00AF1EE10FA05DD04
:1048A0009FED260A224880ED000A34E09FED240A9D
:1048B000F4EEC00AF1EE10FA06D29FED1B0AF4EEF8
:1048C000C00AF1EE10FA0DDA9FED1E0AF4EEC00AEE
:1048D000F1EE10FA0CDD9FED120AF4EEC00AF1EED3
:1048E00010FA05D89FED0E0A114880ED000A12E07B
:1048F0009FED150AF4EEC00AF1EE10FA0BD29FED0F
:10490000130AF4EEC00AF1EE10FA04DD9FED100A6E
:10491000074880ED000A064890ED000A7047000045
:10492000000034430000B443000034C30000000022
:104930004C1F00200000C8420000A0420000B4420A
:1049400000002AC300002A430000A0C20000C8C221
:104950000000B4C210B52DED0A8BB0EE408AF0EE27
:10496000608A38EE680A10EE101A084612F062FFEC
:1049700041EC1A0BB0EE4A0AF0EE6A0A0BF054F85A
:10498000B0EE409AF0EE609A9FED2A0B53EC102B9C
:1049900051EC190B12F056FD2DD238EE680A10EECC
:1049A000101A084612F046FF41EC1C0BB0EE4C0A00
:1049B000F0EE6C0A0BF038F8B0EE40BAF0EE60BAE8
:1049C0009FED1E0B53EC102B51EC1B0B12F048FE0D
:1049D00041EC1A0BB0EE4A0AF0EE6A0A0BF024F82A
:1049E000B0EE409AF0EE609A51EC190B12F014F907
:1049F0001449086018E038EE680A10EE101A0846EC
:104A000012F018FF41EC1A0BB0EE4A0AF0EE6A0AF7
:104A10000BF00AF8B0EE409AF0EE609A51EC190BE8
:104A200012F0FAF807490860064890ED000ABDEC5C
:104A30000A8B10BD000000000080664000000000EE
:104A400000807640481F002070B52DED108B8CB093
:104A5000F0EE409AB0EE60FAB0EE419AF0EE61FAF4
:104A600005460E461446BE4890F8270030B101288E
:104A70000AD0022812D0032824D119E094ED000AAC
:104A8000B84880ED000A1EE094ED000ADFEDB60A9A
:104A900030EE600AB34880ED000A14E094ED000A9D
:104AA000DFEDB20A30EE600AAE4880ED000A0AE09F
:104AB00094ED000ADFEDAC0A30EE200AA94880ED43
:104AC000000A00E000BF00BF1FEE900A12F0B2FE25
:104AD00041EC180B19EE100A12F0ACFE53EC182B37
:104AE000CDE900019DED000B51EC100B12F0ACFB79
:104AF00041EC1E0B9FED9E0B53EC102B12F07AF93C
:104B000041EC1C0B9748006812F094FE41EC1D0B21
:104B100053EC1C2B12F0B2F841EC1B0BB0EE4B0A1D
:104B2000F0EE6B0A0BF01CFE8DED020B1FEE100A6F
:104B300012F080FE41EC1B0B53EC182B12F084FB9F
:104B400041EC1A0B9DED020B53EC102B12F07CFB89
:104B5000CDE9060119EE100A12F06CFE53EC182B89
:104B6000CDE900019DED000B51EC100B12F06CFB38
:104B70009FED7F0B53EC102BCDE902019DED020B55
:104B800051EC100B12F036F941EC1C0B7548006823
:104B900012F050FE41EC1E0B53EC1C2B12F06EF881
:104BA00041EC1B0BB0EE4B0AF0EE6B0A0AF0D8FE9C
:104BB000B0EE40DAF0EE60DA19EE900A12F03AFE4A
:104BC00041EC1B0B53EC182B12F03EFB41EC1A0B83
:104BD00053EC1D2B12F038FBCDE904019DED060BC3
:104BE00053EC102B9DED040B51EC100B12F038FD23
:104BF000CDE90A0119EE100A12F01CFE41EC1C0B63
:104C000053EC182B12F020FB41EC1B0B9FED580BC3
:104C100053EC102B12F0EEF841EC1A0B51480068DF
:104C200012F008FE53EC1A2BCDE900019DED000BAC
:104C300051EC100B12F022F8CDE902019DED020BB0
:104C40000AF08EFEB0EE40DAF0EE60DA1FEE100AE7
:104C500012F0F0FD41EC1A0B53EC182B12F0F4FAA1
:104C600041EC1E0B53EC1D2B12F0EEFACDE90601C0
:104C700019EE100A12F0DEFD41EC1C0B53EC182B60
:104C800012F0E2FA41EC1E0B9FED390B53EC102BA6
:104C900012F0B0F841EC1B0B3248006812F0CAFD6C
:104CA00041EC1D0B53EC1B2B11F0E8FF41EC1A0BF0
:104CB000B0EE4A0AF0EE6A0A0BF052FD8DED020BDF
:104CC00019EE900A12F0B6FD41EC1A0B53EC182BBA
:104CD00012F0BAFACDE900019DED020B53EC102B56
:104CE0009DED000B51EC100B12F0AEFACDE9040172
:104CF0009DED060B53EC102B9DED040B51EC100BAE
:104D000011F0BCFFCDE9080195ED000A10EE101A74
:104D1000084612F08FFD41EC1B0B9DED0A0B53EC86
:104D2000102B11F0ABFF41EC1A0B11F075FF28604E
:104D300096ED000A10EE101A084612F07BFD41ECC9
:104D40001B0B9DED080B53EC102B11F097FF41EC62
:104D50001A0B11F061FF30600CB0BDEC108B70BD10
:104D60005439022034210020DA0FC93FDA0F4940BC
:104D70000000000000000040B0EE401ADFED111A04
:104D8000B0EE610A71EE601AB0EE610ADFED0E1A44
:104D9000B4EEE10AF1EE10FA05D8DFED0C1A70EE70
:104DA000211AB0EE610ADFED0A1AB4EEE10AF1EE63
:104DB00010FA05DBDFED051A70EE611AB0EE610A3C
:104DC0007047000000000000DA0F49C0DA0FC94048
:104DD000DA0F49402DED060BDFED2C0AB0EE600A2C
:104DE000DDED000AFDEEE00A10EE900ADDED030AAB
:104DF000FDEEE00A10EE901A88421BD1DDED040AA8
:104E00009DED011AF4EEC10AF1EE10FA04DDDFEDBA
:104E1000200AB0EE600A36E0DDED040A9DED011ACD
:104E2000F4EEC10AF1EE10FA2DD2DFED1A0AB0EE5F
:104E3000600A28E0DDED010AFDEEE00A10EE900ABE
:104E4000DDED040AFDEEE00A10EE901A88421AD158
:104E5000DDED030A9DED001AF4EEC10AF1EE10FA41
:104E600004DDDFED0A0AB0EE600A0CE0DDED030AB6
:104E70009DED001AF4EEC10AF1EE10FA03D2DFED57
:104E8000060AB0EE600A06B070470000000000009D
:104E9000DA0FC93FDA0FC9BFDA0F4940244890ED55
:104EA000000AB8EEC00A2348D0ED030A30EE200A0B
:104EB000214880ED000A1E4890ED010AB8EEC00AB4
:104EC0001C48D0ED010A30EE200A1B4880ED010A93
:104ED000174890ED060A1948D0ED100A30EE200A66
:104EE000154880ED020A90ED020ADFED150AB4EED6
:104EF000E00AF1EE10FA08DD90ED020ADFED110A8A
:104F000030EE600A80ED020A11E00B4890ED020AD3
:104F1000DFED0D0AB4EEE00AF1EE10FA07D290EDE3
:104F2000020ADFED080A30EE200A80ED020A70471F
:104F3000D4320120743A0220243B0220543902204A
:104F4000DA0F4940DA0FC940DA0F49C0F8B5044614
:104F50000E460020009000255D48007868B94FF4A7
:104F6000AF615C48FBF7CDFD00205B490870012074
:104F700057490870002059490880232C0FD101207F
:104F80005549087056480088401C55490880084615
:104F90000088012806D100205049088002E0002046
:104FA0004F4908804C480078052873D2DFE800F0AC
:104FB0000311043E050086E000BF4FF4AF61454891
:104FC000FBF79FFD012044490870002043490880F9
:104FD00000BF202C0CD041480088B0F5AF6F07DA35
:104FE0003E4801880088401C3C4A1080394844549F
:104FF0005A2C0DD13B480088401C3A49088008468D
:105000000088022803D10320334908700DE05AE0DC
:1050100000203449088031480088B0F5AF6F03DBC9
:1050200002202D49087000E04DE000BF2B4909889F
:105030000839284A88186A462BA1FBF777FB2748CE
:105040000088083801B22348FEF70CFA054600989C
:10505000854204D041F23421009888421BD14FF49C
:10506000AF612348FBF74DFD1A492148FBF76EFC61
:105070004FF4AF611748FBF744FD1D48FBF79FFC59
:105080001C49C1F8E0090020144908800420124995
:10509000087018E015E04FF4AF610E48FBF731FDE2
:1050A00000200E49088002200B490870232C07D1EC
:1050B0004FF4AF610748FBF724FD00200749088043
:1050C00001E000BFFEE700BF03480078F8BD000024
:1050D000F727002048C90120F8270020FA270020E0
:1050E000FE270020FC270020253034780000000037
:1050F00080960120481902200246002002EA01039E
:105100000BB1012000E000207047000070B50025C1
:1051100002212D4880F83417302180F836172B48AB
:1051200000F092FA0546002413E004EB8400284ABC
:1051300002EB80012748FBF72DFC05461DB92248EC
:1051400080F8344707E0022C01D1022070BD601CBA
:10515000C4B2032CE9DB00BF002414E004EB84009C
:105160001D4A02EB80011B482838FBF713FC05465B
:105170001DB9154880F8354707E0032C01D10320FD
:10518000E4E7601CC4B2042CE8DB00BF002416E096
:1051900004EB440000EBC400104A02EB40010D4850
:1051A0002830FBF7F7FB05461DB9074880F836475E
:1051B00007E0302C01D10720C8E7601CC4B2312CB5
:1051C000E6DB00BF0020C1E7F81B022048C9012030
:1051D000D022002010CF012070230020C023002007
:1051E0002DE9FE4F82460C4615461E460C9F4FF495
:1051F000FA611F48FBF785FC1E48B0F8440030B147
:105200001C48B0F844201CA11D48FBF7DFF806EB52
:10521000460000EBC6001B4901EB4000CDE900074A
:1052200005EB8500184901EB800304EB8400144969
:1052300001EB800215A10E48FBF7C8F80C48FBF7FC
:10524000BEFB0FFA80F949460948FEF70BF9804684
:10525000424614A102A8FBF7B9F802A90448FBF7DB
:10526000CDFB0120034981F82800BDE8FE8F000036
:105270008C290220543902202530345800000000C7
:1052800070230020C0230020D022002023232C2CB8
:1052900025732C2C25732C2C25732C2C25732C2C4E
:1052A00000000000253034782C2C5A5A00000000F1
:1052B0007047000010B52DED048B2848007828B108
:1052C00000202649087026480DF040FA244890ED49
:1052D000890A10EE101A084612F0ACFA41EC190BCC
:1052E0009FED200B53EC102B11F0AEFF41EC180B8F
:1052F00011F092FC1D490860194890ED8F0A10EEDC
:10530000101A084612F096FA41EC190B9FED180B93
:1053100053EC102B11F06EFD41EC180B11F07CFCDE
:1053200012494860144890F82500012809D1124814
:1053300090ED060A0846D0ED010A30EE600A80EDD5
:10534000020A0A4890ED010AD0ED020A30EE200A66
:1053500080ED010ABDEC048B10BD0000401600205A
:10536000FC2B0120514CDE0033DF913F5C330120E8
:105370006666666666A64C40D432012000BF011EF8
:10538000A0F1010290B2FAD17047000010B504A15B
:10539000012009F0A3FC4FF4807000F011F810BD5B
:1053A0003C2A2A2A2A2A2A2A2A2A2A2A2A2A2A2A4B
:1053B0002A2ABFAAC6F4B1A3B4E60D0A0000000071
:1053C0000149086070470000143C014010B50748CF
:1053D000006800F07F000549091D096801F07F01A0
:1053E000884202D27F2009F02BFE10BD002C004025
:1053F000F0B50A4600210023002400BF3DE001254E
:1054000005FA01F3156805EA03049C4234D10568E6
:105410004F000326BE40B543056015794E00B540E8
:105420000668354305601579012D02D01579022DE6
:1054300016D185684F000326BE40B5438560557977
:105440004E00B540866835438560456801268E402C
:10545000B5434560456896798E40B6B235434560A0
:10546000C5684F000326BE40B543C560D5794E00E0
:10547000B540C6683543C560491C1029BFD3F0BD8F
:10548000F0B5002300244D07ED0E02FA05F3CE100F
:1054900000F1200555F826504E07F70E0F26BE40A6
:1054A000B543CF1000F1200646F82750CE1000F18A
:1054B000200555F8265045EA0304CE1000F12005DA
:1054C00045F82640F0BD0246002013690B400BB1A1
:1054D000012000E00020704741837047018370473E
:1054E00000B52DED0A0BC5B09DED450ADDED480A6E
:1054F000B4EEE00AF1EE10FA04DD4FF0FF304F4950
:10550000086002E001204D4908609DED471ADDED7D
:10551000460A9DED450A68460DF0AEFD302269460B
:1055200030A8FBF7BCFADDED4D2A9DED4C2ADDEDF0
:105530004B1A9DED4A1ADDED490A9DED480A684671
:105540000DF022FE3022694624A8FBF7A8FA24A910
:1055500030A80DF05FFC8DED3F0ACDED400A8DEDDA
:10556000411ADDED412A9DED402ADDED3F1A9DED0A
:10557000471ADDED460A9DED450A08F023FE304846
:1055800080ED000A2F4890F82400082804D02D4808
:1055900090F824000A2810D12848012203682848DE
:1055A00090ED000A3FA924A80EF096F88DED420A6E
:1055B000CDED430A8DED441A19E0224890F82400FD
:1055C000072804D01F4890F8240009280FD11B4851
:1055D000002203681A4890ED000A3FA924A80EF0A3
:1055E0007BF88DED420ACDED430A8DED441A45AAB4
:1055F00030A968460EF05EFA3022694618A8FBF71B
:105600004EFA42AA24A968460EF054FA302269469E
:105610000CA8FBF744FA0CA918A80DF0FBFB8DEDC4
:105620003C0ACDED3D0A8DED3E1A9DED3C0ADDEDC7
:105630003D0A9DED3E1A4FB000BD00003021002014
:105640002C2100205439022070B50446002145F673
:10565000D81001512AA12B48FBF772F905464AE000
:1056600045F6D810005904282CD14FF4AF6141F20F
:1056700068002044FBF745FA2A4623A141F268005E
:105680002044FAF7A3FE45F6D811095901EB81022F
:1056900004F5AF6101EBC2001CA21BA1FAF796FE54
:1056A0004FF4AF6145F260402044FBF72AFA4FF413
:1056B000AF6241F26800211845F260402044FBF7D8
:1056C000EEF90CE045F6D811095901EB810204F519
:1056D000AF6101EBC2002A460BA1FAF777FE45F64F
:1056E000D8100059401C45F6D811085104A10020DB
:1056F000FBF726F90546002DB2D1002070BD000051
:105700002C2C000080960120257300003000000042
:105710002DE9F0418EB004460D461646342101A80D
:10572000FBF7EFF92846FBF74AF98046424629463F
:1057300001A8FBF76FF900202070314601A8FBF7A4
:10574000FFF8074611E02178C1EB0112611C01EB63
:1057500042003A4608A1FAF739FE2078401C207032
:1057600031460020FBF7ECF80746002FEBD1002074
:105770000EB0BDE8F081000025730000F0EE401A85
:10578000B4EEE01AF1EE10FA04DD30EEA10AF0EE0C
:10579000400A08E0B4EEE01AF1EE10FA03D230EE5F
:1057A000E10AF0EE400A30EEC10AB0EEC00AB4EEF3
:1057B000E10AF1EE10FA01D8F0EE410AB0EE600A0B
:1057C000704700002DE9F041054600240026002125
:1057D00045F6DC10415100BF0AE004EB840205F5F8
:1057E000AF5101EBC2002821FBF78BF9601C84B29A
:1057F000B4F5C87FF1DBE7A141F268002844FBF76C
:105800009FF8804610E006EB860205F5AF5101EBEC
:10581000C2004246E0A1FAF7D9FDDEA10020FBF765
:105820008FF88046701C86B2B8F1000FEBD1DBA177
:10583000DD48FBF7AFF878B900240BE004EB440136
:10584000C1EB4411D94A02EBC100E821FBF759F939
:10585000601C84B2B442F1DBD548C0F8786DCFA1AA
:10586000D148FBF797F800287DD1D24890F8BD00C9
:10587000012879D1CF4890F8A80000F080000028D6
:10588000F7D1CDA205F5AF51C848FFF741FFC74991
:105890000978491EC1EB0112C449491C01EB4200C1
:1058A000FBF708F8C5490860C248806F096888425C
:1058B00002D10020BDE8F0810CF090FCC0484660A9
:1058C00000242AE1BA48C0F87C6D04EB840305F596
:1058D000AF5202EBC30104EB4402C2EB4412B34BE0
:1058E00003EBC200B4A2FFF713FF002733E004EB81
:1058F0004401C1EB4411AD4A02EBC101491CC7EBA5
:10590000071201EB42000A220021FAF7E0FF04EB44
:105910004401C1EB4411A54A02EBC101D83141F861
:10592000270004EB4400C0EB4410114601EBC0001B
:10593000D83050F8270000EE100AB8EEC00AC4EBC9
:10594000C4019F480C3000EB810000EB870080ED24
:10595000000A781C87B2022FC9DB04EB4401C1EBBB
:105960004411924A01E0ECE011E102EBC101491C53
:1059700004EB4402C2EB44128C4B13F83220521E4B
:10598000C2EB021201EB4200FAF794FFC4EBC4022F
:105990008B490C3101EB8201886104EB4401C1EBBE
:1059A0004411824A02EBC101491C04EB4402C2EBE0
:1059B00044127E4B13F83220921EC2EB021201EB0E
:1059C0004200FAF777FFC1B2C4EBC4027C480C3046
:1059D00000EB8200017304EB4401C1EB4411734AF4
:1059E00002EBC101491C04EB4402C2EB44126F4BB1
:1059F00013F83220D21EC2EB021201EB4200FAF77A
:105A000059FFC4EBC4026E490C3101EB82010861FD
:105A100004EB4400C0EB4410644901EBC000401C9F
:105A200004EB4401C1EB4411604A12F83110491FE4
:105A3000C1EB011100EB410104EB4400C0EB441049
:105A400002EBC0000988A0F8D31004EB4400C0EBBF
:105A50004410114601EBC000401C04EB4401C1EBB3
:105A6000441112F83110091FC1EB011100EB410183
:105A700004EB4400C0EB441002EBC0000988A0F81E
:105A8000D51004EB4400C0EB4410114601EBC000FC
:105A900090F8D500702808D10121C4EBC402484811
:105AA0000C3000EB820001751BE004EB4400C0EBFE
:105AB00044103E4901EBC00090F8D500712808D190
:105AC0000221C4EBC4023E480C3000EB8200017599
:105AD00007E00021C4EBC40239480C3000EB82001F
:105AE000017504EB4402C2EB4412304B03EBC202DB
:105AF00092F8D51004EB4402C2EB441203EBC2024D
:105B000092F8D300FDF74EFCC4EBC4022C490C31D3
:105B100001EB8201C881601C84B2B442FFF6D2AEB0
:105B20000021244880F8BA1080F8BB1080F8BD101E
:105B30004FF4127007F056FA2148416A1D488167F8
:105B400025E0002421E01FA11748FAF723FF68B9D8
:105B500004EB840205F5AF5101EBC20010220021D5
:105B6000FAF7B5FE194941F824000CE004EB840271
:105B700005F5AF5101EBC2000A220021FAF7A7FE9A
:105B8000124941F82400601C84B2B442DBDB0020DF
:105B900090E600003A3A0000257300007365746CCB
:105BA000726F75740000000038CF0120F89B01204F
:105BB000F81B0220543902205F0000000428002056
:105BC000408901207365747469707300302302206A
:105BD00010B52DED068BFE48D0ED022A90ED012A7E
:105BE000D0ED001AFB4890ED021AD0ED010A90EDBD
:105BF000000AFFF7EFF8F84880ED090AF748007847
:105C000000287DD19FEDF60AF64880ED000A0020BD
:105C1000F5490870F54890ED010A10EE101A084693
:105C200011F008FE41EC190BB0EE490AF0EE690ADA
:105C300009F0FAFEB0EE408AF0EE608A9FEDEC0BC0
:105C400053EC102B51EC180B11F0C2FA74D2EA4845
:105C500090ED010A10EE101A084611F0EBFD41EC30
:105C6000190BB0EE490AF0EE690A09F0DDFEB0EE5C
:105C7000408AF0EE608A9FEDDE0B53EC102B51EC66
:105C8000180B11F0A5FAE1D2D34890ED091AF0EE05
:105C9000410ADA4890ED061AB0EE410AFFF76CF8B7
:105CA00010EE104A204611F0C5FD41EC1A0BB0EE83
:105CB0004A0AF0EE6A0A09F0B7FEB0EE409AF0EE3A
:105CC000609A9FEDCF0B53EC102B51EC190B11F098
:105CD000BBFA41EC180B10F09FFFC249086308465D
:105CE00090ED0C0ADFEDC80AB4EEE00AF1EE10FA0E
:105CF0000FDD90ED0C0ADFEDC50AB4EEE00A00E01E
:105D00001BE0F1EE10FA04D29FEDC10A80ED0C0AFF
:105D10000DE0B44890ED0C0ADFEDBE0AB4EEE00AE7
:105D2000F1EE10FA03DD9FEDBC0A80ED0C0A0120B4
:105D3000AA490870B94908700FE2A84800780128FC
:105D4000FAD1A84890F82400032804D0A54890F878
:105D50002400042832D1A04890ED091AF0EE410A3F
:105D6000AF4890ED021AB0EE410AFFF705F8AD48D2
:105D700080ED000A984890ED091AF0EE410AA84813
:105D800090ED021AB0EE410AFEF7F6FF10EE104A4F
:105D9000204611F04FFD41EC190BB0EE490AF0EE30
:105DA000690A09F041FEB0EE408AF0EE608A51ECDB
:105DB000180B10F031FF9C49086039E0864890EDDF
:105DC000091AF0EE410A964890ED021ADFED971A93
:105DD00031EE211AB0EE410AFEF7CEFF914880ED78
:105DE000000A7D4890ED091AF0EE410A8C4890EDCA
:105DF000021ADFED8E1A31EE211AB0EE410AFEF7DB
:105E0000BBFF10EE104A204611F014FD41EC190BB7
:105E1000B0EE490AF0EE690A09F006FEB0EE408ADB
:105E2000F0EE608A51EC180B10F0F6FE7E49086027
:105E30007B4890ED020A6B4880ED360A664890ED8B
:105E4000090A684880ED370A774890ED000A6548EE
:105E500080ED380A744890ED000ADFED750AB4EE63
:105E6000E00AF1EE10FA07DB90ED000ADFED700AB0
:105E700030EE600A80ED000A68480078E0B36A48B6
:105E8000006811F0D7FC41EC180B9FED6A0B53EC46
:105E9000102B11F0D7FA0AD85248B0F8520000EE91
:105EA000100AB8EE400A4F4880ED000A8EE05E48C6
:105EB000006811F0BFFC41EC180B9FED5E0B53EC3A
:105EC000102B11F085F927D2574890ED000ADFED2D
:105ED0005B0AB4EEE00AF1EE10FA1DDD4148B0F8BD
:105EE000520000EE100AB8EE400AB0EE402AF3EE7F
:105EF0000E1AB6EE001A00E026E0DFED500A4A481E
:105F000090ED000A0EF0E6F8BDEEC00AB8EEC00A49
:105F1000344880ED000A59E0434890ED000ADFED77
:105F2000470AB4EEE00AF1EE10FA4FD8444801787F
:105F30000078401C424A10700A2947DD002037498A
:105F400008701146087041E09FED250A254880ED54
:105F5000000A264890ED010A10EE101A084611F0CA
:105F600069FC41EC190BB0EE490AF0EE690A09F040
:105F70005BFDB0EE408AF0EE608A9FED1D0B53ECA6
:105F8000102B51EC180B11F023F91FD21A4890ED89
:105F9000010A10EE101A084611F04CFC41EC190BE6
:105FA000B0EE490AF0EE690A09F03EFDB0EE408A13
:105FB000F0EE608A9FED0E0B53EC102B51EC180B9A
:105FC00011F006F902D2012007490870154839E09E
:105FD000183B02200C3B0220743A0220541D002082
:105FE0000000000054390220551D00202C330120F0
:105FF000000000000000144044330120D43201208E
:106000006666666666A64C4000008C420000DC4274
:106010000000B4420000204300003443561D00201D
:10602000243B02204C1D0020481D0020DA0F49406F
:10603000DA0FC940000000000000E03F0AD7A33C8F
:106040005C1D002090ED000A474880ED000A47489B
:106050000078012863D11FED1E0A434880ED000A35
:106060001FED210A424880ED000A424890ED010AE6
:1060700010EE101A084611F0DDFB41EC190BB0EEE2
:10608000490AF0EE690A09F0CFFCB0EE408AF0EE62
:10609000608A1FED290B53EC102B51EC180B11F0FB
:1060A00097F855D2344890ED010A10EE101A0846C0
:1060B00011F0C0FB41EC190BB0EE490AF0EE690A91
:1060C00009F0B2FCB0EE408AF0EE608A1FED380BAA
:1060D00053EC102B51EC180B11F07AF838D22448FD
:1060E000D0F8040125490968401AB0F5FA7F34D97F
:1060F0001F4890F82400032804D01D4890F824007D
:1061000004280DD101211A48807F401EC0EBC00237
:106110001B4800EB8200C18100201A4908701CE076
:10612000134890F82400052804D0114890F8240062
:10613000062812D102210E48807F401EC0EBC0020B
:106140000F4800EB8200C18100200E49087004E076
:106150000748D0F8040109490860B7EE080A0FF0B3
:1061600023FFBDEC068B10BD501D0020551D0020E7
:10617000543902202C33012044330120581D0020C3
:106180004C890120541D002010B52DED068B31489F
:1061900090ED000A10EE101A084611F04BFB41EC8E
:1061A000190BB0EE490AF0EE690A09F03DFCB0EEB9
:1061B000408AF0EE608A9FED280B53EC102B51ECD7
:1061C000180B11F03FF90ED82548B0F9200000EE69
:1061D000100AB8EEC00A224880ED000AB6EE000AA6
:1061E0000FF0E2FE33E01B4890ED000A10EE101AAB
:1061F000084611F01FFB41EC1A0BB0EE4A0AF0EE14
:106200006A0A09F011FCB0EE409AF0EE609A51EC87
:10621000190B10F001FD08EE100A1148B0F920002A
:1062200000EE100AB8EEC00AB0EE402ADFED0D1AFB
:10623000B6EE001ADFED0C0AB0EE480A0DF04AFF88
:10624000074880ED000A9FED090A0FF0ADFEBDEC96
:10625000068B10BD743A0220000000000000E03FF1
:10626000543902200000C84200000000CDCC4C3E52
:1062700010B52DED0C8BA448D0ED022A90ED012A2B
:10628000D0ED001AA14890ED021AD0ED010A90ED70
:10629000000A07F097FFB0EE408A9FED9D0AB4EE2A
:1062A000C08AF1EE10FA2CDD9A4890ED030A10EE48
:1062B000101A084611F0BEFA41EC1D0BB0EE4D0A63
:1062C000F0EE6D0A09F0B0FBB0EE40BAF0EE60BA45
:1062D00018EE100A11F0AEFA41EC1C0B53EC1B2B1C
:1062E00011F0BEF941EC1A0B9FED8B0B53EC102B08
:1062F00011F0B6F941EC190B10F08EFC85490861DC
:1063000023E0844890ED030A10EE101A084611F0BD
:1063100091FA41EC1C0BB0EE4C0AF0EE6C0A09F05D
:1063200083FBB0EE40AAF0EE60AA18EE100A11F05E
:1063300081FA41EC1B0B53EC1A2B11F091F941EC53
:10634000190B10F069FC73490861754890F8240036
:10635000734991F8251088420AD17148B0F920009C
:1063600000EE100AB8EEC00A6D4880ED000ABAE0EF
:106370006B4890F8250007280ED0694890F8250052
:10638000082809D0664890F82500092804D06448F8
:1063900090F825000A2841D15E48D0ED040A6048F3
:1063A000B0F8480000EE100AB8EE400AF4EEC00A59
:1063B000F1EE10FA0ADB5A48B0F9200000EE100A9C
:1063C000B8EEC00A564880ED000A8CE05448B0F997
:1063D000200000EE900AF8EEE00AB0EE602A504885
:1063E000B0F9220000EE900AF8EEE00AF0EE601A32
:1063F0004B48B0F8480000EE900AF8EE600AB0EEA4
:10640000601A4448D0ED040AB0EE600ADFED450A98
:106410000DF060FE424880ED000A64E03D48D0ED9A
:10642000040A3F48B0F8480000EE100AB8EE400AEF
:10643000F4EEC00AF1EE10FA0ADB3948B0F9200098
:1064400000EE100AB8EEC00A354880ED000A4AE0B6
:106450003048D0ED040A3248B0F8480000EE100A87
:10646000B8EE400AF4EEC00AF1EE10FA31D829482D
:1064700090ED040AF3EE0E0AB4EEE00AF1EE10FA23
:1064800027DD2748B0F9200000EE900AF8EEE00A78
:10649000B0EE602A2248B0F8460000EE900AF8EE0E
:1064A000600AF0EE601A1E48B0F8480000EE900A4C
:1064B000F8EE600AB0EE601A1648D0ED040AB0EEAD
:1064C000600AF3EE0E0A0DF005FE154880ED000A95
:1064D00009E01348B0F8460000EE100AB8EE400A92
:1064E0000F4880ED000A104890ED010AB5EEC00A91
:1064F000F1EE10FA04D09FED0B0A094880ED000A76
:10650000BDEC0C8B10BD0000183B02200C3B0220A0
:1065100000401C46743A0220000000000000794050
:1065200054390220000000008833012070B531A5E5
:1065300000240BE0285D3A49888000BF3848008875
:1065400000F040000028F9D0601CC4B22A2CF1D31E
:106550004FE07F2008F074FD08F032FD31480078EC
:10656000401C3049087008460078012800DD70BDE5
:10657000002240F225512C4808F0D6FA002240F2C1
:106580002771294808F0D0FA002240F2255124480A
:1065900008F0CAFA002240F22771214808F0C4FA34
:1065A000002240F22551214808F0BEFA002240F2B4
:1065B00027711E4808F0B8FA002240F225511C4805
:1065C00008F0B2FA002240F22771194808F0ACFA3C
:1065D00000BFBFF34F8F1748006800F4E060164912
:1065E0000843001D13490860BFF34F8F00BF00BF71
:1065F000FEE7AEE70D0A456E74657220486172646D
:106600004661756C745F48616E646C65722C2053D2
:10661000797374656D2048616C742E0D0A0000005A
:1066200000100140AC07002000140140004400406D
:10663000004800400CED00E00000FA0510B50DF038
:10664000B7FB0DF0AFFA10BD704710B50446202C13
:1066500079D2DFE804F0101D2A3744515E6B798649
:1066600093A0ADBAC7D4F1FEEEEDECEBEAE9E8E7B2
:10667000E6E5E4E3E2E10021162003F01DF9002144
:10668000172003F019F90021182003F015F9A4E1EF
:106690000121162003F010F90021172003F00CF956
:1066A0000021182003F008F997E10021162003F0DB
:1066B00003F90121172003F0FFF80021182003F04F
:1066C000FBF88AE10021162003F0F6F800211720DC
:1066D00003F0F2F80121182003F0EEF87DE101212A
:1066E000162003F0E9F80121172003F0E5F8002156
:1066F000182003F0E1F870E10021162003F0DCF827
:106700000121172003F0D8F80021182003F0D4F855
:1067100063E10121162003F0CFF80021172003F0D8
:10672000CBF80021182003F0C7F856E1002116200D
:1067300003F0C2F80021172003F0BEF80021182052
:1067400003F0BAF849E147E10121162003F0B4F85B
:106750000121172003F0B0F80121182003F0ACF854
:106760003BE10121162003F0A7F80021172003F0D8
:10677000A3F80121182003F09FF82EE10021162034
:1067800003F09AF80121172003F096F80121182050
:1067900003F092F821E10121162003F08DF8012188
:1067A000172003F089F80121182003F085F814E17F
:1067B0000121162003F080F80121172003F07CF856
:1067C0000021182003F078F807E10021162003F0DB
:1067D00073F80021172003F06FF80121182003F04F
:1067E0006BF8FAE00121162003F066F8002117206B
:1067F00003F062F80121182003F05EF8EDE00021BB
:10680000162003F059F80121172003F055F8012153
:10681000182003F051F8E0E0D1E0C3E0B5E0A7E0D4
:1068200099E08BE07DE06FE061E053E045E037E028
:1068300029E01BE00DE0FFE70121162003F03CF802
:106840000121172003F038F80121182003F034F853
:10685000C3E00121162003F02FF80121172003F0D7
:106860002BF80021182003F027F8B6E000211620AD
:1068700003F022F80021172003F01EF80121182050
:1068800003F01AF8A9E00121162003F015F8002101
:10689000172003F011F80121182003F00DF89CE0F7
:1068A0000021162003F008F80121172003F004F856
:1068B0000121182003F000F88FE00121162002F0DA
:1068C000FBFF0121172002F0F7FF0121182002F041
:1068D000F3FF82E00121162002F0EEFF01211720D4
:1068E00002F0EAFF0021182002F0E6FF75E0002127
:1068F000162002F0E1FF0021172002F0DDFF012148
:10690000182002F0D9FF68E00121162002F0D4FF20
:106910000121172002F0D0FF0121182002F0CCFF46
:106920005BE00021162002F0C7FF0121172002F0D2
:10693000C3FF0121182002F0BFFF4EE00121162005
:1069400002F0BAFF0021172002F0B6FF0121182043
:1069500002F0B2FF41E00021162002F0ADFF00215D
:10696000172002F0A9FF0121182002F0A5FF34E052
:106970000121162002F0A0FF0121172002F09CFF48
:106980000021182002F098FF27E00021162002F0D5
:1069900093FF0121172002F08FFF0021182002F041
:1069A0008BFF1AE00121162002F086FF002117203C
:1069B00002F082FF0021182002F07EFF0DE000218E
:1069C000162002F079FF0021172002F075FF002148
:1069D000182002F071FF00E000BF00BF10BD0000F2
:1069E00010B52DED0C8B0446E07A602809D1207B90
:1069F000602806D1607B602803D1012048494861A6
:106A00001EE0E07A60280CD1207B402809D1607B11
:106A1000602806D1E07B062803D102204049486166
:106A20000EE0E07A60280BD1207B402808D1607B03
:106A3000602805D1E07B0F2802D103203849486146
:106A4000E07A432868D1207B6C2865D1607B602880
:106A500062D1A07C0206607C02EB0042207C02EB4B
:106A60000022E07B104400EE100AB8EEC00A10EEDF
:106A7000101A084610F0DEFE41EC1D0B9FED290BAD
:106A800053EC102B10F0B6F941EC1C0B9FED270BCB
:106A900053EC102B10F0D8FB41EC1B0B9FED250B9A
:106AA00053EC102B10F0D0FB41EC1A0B9FED230B95
:106AB00053EC102B10F09EF941EC190B9FED210BBC
:106AC00053EC102B10F096F941EC180B10F0A4F8D1
:106AD00013494860084690ED010A10EE101A084666
:106AE00010F0A8FE41EC190BB0EE490AF0EE690A6D
:106AF00008F09AFFB0EE408AF0EE608A9FED130B2B
:106B000053EC102B51EC180B10F062FB04D29FEDEC
:106B1000110A034880ED010ABDEC0C8B10BD00008A
:106B20002C330120666666666655A5C00C022B876D
:106B300016D9E63FCDCCCCCCCCCCF03F0000000049
:106B4000000000408716D9CEF753F13F0000000047
:106B5000000024400000000010B50446E07A6028E0
:106B60000CD1207B602809D1607B602806D10120F0
:106B70004249087042A108F0B1F826E0E07A6028A6
:106B800010D1207B40280DD1607B60280AD1E07BAA
:106B9000062807D10220394908703FA1012008F0DA
:106BA0009DF812E0E07A60280FD1207B40280CD1BC
:106BB000607B602809D1E07B0F2806D103202F4994
:106BC00008703BA1012008F089F8E07A432833D10E
:106BD000207B632830D1607B60282DD13A4890F823
:106BE000930020BBE17B207C41EA0021607C41EAEC
:106BF0000041A07C41EA0060344908600846006812
:106C000033490968401A00EE100AF8EEC00A9FEDF9
:106C1000311A80EE810A1948D0ED030A30EE200ABD
:106C200080ED030A294800682949086004E09FEDC7
:106C30002A0A124880ED030A207B01280ED1607BCE
:106C400026280BD1617C207C41EA00200B49088377
:106C5000E17CA07C41EA0021084841830748008B81
:106C600020B14FF4006006F0FDFF06E00348808B82
:106C700018B94FF4006006F0B5F910BD6833012073
:106C8000BED9C9FDC9E8D6C3CBD9B6C8C4A3CABD4D
:106C9000B3C9B9A60D0A0000BED9C9FDC9E8D6C35B
:106CA000CAB9C4DC3036B3C9B9A60D0A0000000069
:106CB000BED9C9FDC9E8D6C3CAB9C4DC3046B3C918
:106CC000B9A60D0A0000000054390220D4050020A6
:106CD000D005002000409C470000000010B52DEDBD
:106CE0000A8BE64890ED000AF0EE000A30EE200A2A
:106CF00010EE101A084610F09DFD41EC180BE0480C
:106D000090ED020A10EE101A084610F093FD41ECC7
:106D10001A0BB0EE4A0AF0EE6A0A08F085FEB0EEF1
:106D2000409AF0EE609A53EC182B51EC190B10F0CE
:106D30004FFA50D2D14890ED000AF0EE000A30EE42
:106D4000200A10EE101A084610F074FD41EC180BE2
:106D5000CB4890ED030A10EE101A084610F06AFDB9
:106D600041EC1A0BB0EE4A0AF0EE6A0A08F05CFE3B
:106D7000B0EE409AF0EE609A53EC182B51EC190BE0
:106D800010F026FA27D2BF480078012823D106F058
:106D90006BF80446022006F067F80440BCB10020FE
:106DA000B94988754FF4806006F01CF9802006F020
:106DB00019F94FF4007006F055FF0121B34880F82F
:106DC000BD10002180F8BA1080F88D1053E1072023
:106DD000AD4988754FE10020AA490870AC48007899
:106DE000012843D1A64890ED020AAA48D0ED000A36
:106DF000B4EEE00AF1EE10FA03DD0220A349C876F2
:106E000016E09F4890ED020AA248D0ED000AF1EE8C
:106E1000600AB4EEE00AF1EE10FA03D201209B49B9
:106E2000C87605E000209949C87602209849087084
:106E3000994890ED020A10EE101A084610F0FAFC7C
:106E400041EC1A0B9FED950B53EC102B10F0FCF955
:106E500041EC190B0FF0E0FE08EE100AB0EE480A04
:106E6000FDF7E0FC864880ED080A04E188480078D8
:106E7000022868D103208549C8769FED8A0A084612
:106E800080ED0C0A844890ED020A10EE101A0846B4
:106E900010F0D0FC41EC1C0B9FED800B53EC102B41
:106EA00010F0D2F941EC1B0B0FF0B6FE08EE100A01
:106EB000734890ED080AF0EE400AB0EE480AFDF77C
:106EC00049FDDFED780A30EE600A10EE104A2046E8
:106ED00010F0B0FC41EC1A0BB0EE4A0AF0EE6A0A70
:106EE00008F0A2FDB0EE409AF0EE609A9FED6E0BB6
:106EF00053EC102B51EC190B10F06AF9B5D20020AD
:106F00006249C876644890ED020A10EE101A0846ED
:106F100010F090FC41EC1A0B9FED600B53EC102B22
:106F200010F092F941EC190B0FF076FE08EE100A02
:106F3000B0EE480AFDF776FC514880ED080A0320C0
:106F40005349087097E052480078032826D14C48EE
:106F500090ED020A4F48D0ED000AB4EEE00AF1EEDF
:106F600010FA03DD02204949C87684E0444890EDD8
:106F7000020A4848D0ED000AF1EE600AB4EEE00AD9
:106F8000F1EE10FA03D201204049C87673E00020E8
:106F90003E49C87604203E4908706CE03C480078C1
:106FA000042868D13949C8769FED3E0A084680ED2D
:106FB0000C0A394890ED020A10EE101A084610F03B
:106FC00039FC41EC1C0B9FED350B53EC102B10F0F2
:106FD0003BF941EC1B0B0FF01FFE08EE100A28488E
:106FE00090ED080AF0EE400AB0EE480AFDF7B2FC58
:106FF000DFED2C0A30EE600A10EE104A204610F049
:1070000019FC41EC1A0BB0EE4A0AF0EE6A0A08F0DD
:107010000BFDB0EE409AF0EE609A9FED230B53EC1F
:10702000102B51EC190B10F0D3F824D20020174983
:10703000C876194890ED020A10EE101A084610F0B2
:10704000F9FB41EC1A0B9FED150B53EC102B10F0D4
:10705000FBF841EC190B0FF0DFFD08EE100AB0EE63
:10706000480AFDF7DFFB064880ED080A01200849C1
:10707000087004490870BDEC0A8B10BD141F002075
:10708000D43201201E1F00208833012054390220F1
:107090001D1F0020181F0020243B02206666666624
:1070A00066A64C400000B442000000000000E03F33
:1070B00000B58DB0FE48007800287CD0FD4880687F
:1070C000019010F0B7FB9FEDFC0B53EC102BCDE9BA
:1070D00002019DED020B51EC100B10F0B5F8CDE95B
:1070E00004019DED040B51EC100B0FF095FD069083
:1070F0009DED060AFDF796FB8DED070A079810F047
:1071000099FB9FEDED0B53EC102BCDE908019DEDA4
:10711000080B51EC100B0FF06DFECDE90A019DED4F
:107120000A0B51EC100B0FF077FDE5490860E148C0
:1071300090ED020A8DED0B0A0846D0ED000A9DED98
:107140000B0AFDF719FEDF4880ED000A006810F019
:1071500071FB9FEDDD0B53EC102BCDE90A019DED8A
:107160000A0B51EC100B10F06DF90AD2B3EE040AC1
:10717000D74880ED000ABBEE040AD64880ED000A2D
:1071800024E2D048006810F055FB9FEDD30B53EC80
:10719000102BCDE90A019DED0A0B51EC100B10F0FC
:1071A00017F80CD2BBEE040AC94880ED000AB3EE12
:1071B000040AC84800E020E080ED000A06E29FEDE6
:1071C000C80AC34880ED000A9FEDC50AC14880ED9A
:1071D000000A802005F006FF4FF4007006F042FD23
:1071E0000121C04880F8BD10002180F8BA1080F855
:1071F0008D100020AE490870E8E1BB48006810F02F
:1072000019FBCDE90A01B9488068059010F012FB1E
:10721000CDE906019DED060B08F006FC8DED080B8F
:107220009DED0A0B53EC102B9DED080B51EC100B50
:107230000FF0CEFF24D2AC48006810F0FBFACDE985
:107240000A01AA48C068059010F0F4FACDE90601D9
:107250009DED060B08F0E8FB8DED080B9DED0A0B8C
:1072600053EC102B9DED080B51EC100B0FF0B0FF01
:1072700006D29F480078012802D18D490870A5E107
:1072800000209B4908708B488068059010F0D2FA66
:107290009FED890B53EC102BCDE906019DED060BFC
:1072A00051EC100B0FF0D0FFCDE908019DED080B5C
:1072B00051EC100B0FF0B0FC0B909DED0B0AFDF79D
:1072C000B1FA8A4880ED080A8A480078B0BB87483E
:1072D00090ED020A8848D0ED000AB4EEE00AF1EE23
:1072E00010FA03DD02207F49C87602E001207D49C3
:1072F000C8768148006810F09DFACDE90A017B4804
:107300008068059010F096FACDE906019DED060B18
:1073100008F08AFB8DED080B9DED0A0B53EC102B4A
:107320009DED080B51EC100B0FF052FFA7D200207F
:107330006C49C87601206F49087047E1FFE76D4846
:107340000078012877D1694890ED030A6A48D0EDAA
:10735000000AB4EEE00AF1EE10FA05DB0320614901
:10736000C876664908701DE0604890ED030A6248DF
:10737000D0ED000AF1EE600AB4EEE00AF1EE10FA88
:1073800005D204205749C8765C4908700AE0554880
:10739000C07E38B900205349C8765649087001208C
:1073A0005349087043488068019010F043FA9FEDFC
:1073B000420B53EC102BCDE902019DED020B51EC79
:1073C000100B0FF041FFCDE904019DED040B51ECD2
:1073D000100B0FF021FC0690444890ED080A8DED4B
:1073E000050ADDED050A9DED060AFDF7B3FAF1EE9B
:1073F0000C0A30EE600A8DED070A079810F01AFAB1
:10740000CDE908019DED080B08F00EFB8DED0A0B90
:107410009FED3B0B53EC102B9DED0A0B51EC100B29
:107420000FF0D6FE89D200202E49C87602203149BD
:10743000087085E3FFE72F480078022870D12B48B9
:10744000C068019010F0F6F9CDE902019DED020B44
:1074500008F0EAFA8DED040B9FED2B0B53EC102B8B
:107460009DED040B51EC100B10F0FAF8CDE906017C
:107470009DED060B08F0D8FA8DED080B9FED240B5F
:1074800053EC102B9DED080B51EC100B0FF0DCFEB4
:10749000CDE90A019DED0A0B51EC100B0FF0BCFB7E
:1074A0001D490860084690ED000ADFED1C0A38E02F
:1074B0001C1F0020243B02206666666666A64C40C0
:1074C000841F0020881F00207B14AE47E17A843F90
:1074D0002C330120443301207B14AE47E17A84BF72
:1074E0000000000054390220141F0020D432012073
:1074F0000D1F00200C1F0020181F0020681F0020F7
:10750000000000000000E03F000000000000084014
:107510000000000000001840741F002000003442EA
:107520008EE0B4EEE00AF1EE10FA05D290ED000A1A
:10753000FE4880ED000A04E01FED080AFB4880EDDC
:10754000000A0220FA49C876FA48006810F072F979
:10755000CDE90A01F8488068059010F06BF9CDE993
:1075600006019DED060B08F05FFA8DED080B9DED11
:107570000A0B53EC102B9DED080B51EC100B0FF088
:1075800027FE24D2EB48006810F054F9CDE90A0137
:10759000E948C068059010F04DF9CDE906019DED70
:1075A000060B08F041FA8DED080B9DED0A0B53EC2C
:1075B000102B9DED080B51EC100B0FF009FE06D2BD
:1075C0000020DB49C8760320DC490870B8E2D948BE
:1075D000006810F02FF9CDE90A01D748C06805907E
:1075E00010F028F9CDE906019DED060B08F01CFA14
:1075F0008DED080B9DED0A0B53EC102B9DED080B48
:1076000051EC100B0FF0E4FD06D20020C849C876FB
:107610000320CA49087093E2C74890ED020AC348A4
:10762000D0ED000AF1EE600AB4EEE00AF1EE10FAD5
:10763000CCD20020BE49C8760320C04908707FE242
:10764000BE48007803287DD1BD480078032807D1C3
:107650000420B749C8760846C07EBA4908700AE0D7
:10766000B7480078042806D10320B149C8760846F7
:10767000C07EB4490870B4488068019010F0DAF810
:107680001FED730B53EC102BCDE902019DED020BA6
:1076900051EC100B0FF0D8FDCDE904019DED040B6A
:1076A00051EC100B0FF0B8FA0690A34890ED080AC1
:1076B0008DED050ADDED050A9DED060AFDF74AF997
:1076C0005FED790A30EE600A8DED070A079810F039
:1076D000B1F8CDE908019DED080B08F0A5F98DED95
:1076E0000A0B9FED9A0B53EC102B9DED0A0B51ECFE
:1076F000100B0FF06DFD05D29648007810B90120EF
:107700009449087090488068019010F093F81FED3C
:10771000960B53EC102BCDE902019DED020B51ECC1
:10772000100B0FF091FDCDE904019DED040B51EC20
:10773000100B0FF071FA06907F4890ED080A8DED5E
:10774000050A00E043E0DDED050A9DED060AFDF7C0
:1077500001F9F1EE0C0A30EE600A8DED070A079888
:1077600010F068F8CDE908019DED080B08F05CF910
:107770008DED0A0B9FED750B53EC102B9DED0A0B55
:1077800051EC100B0FF024FD20D272480078012834
:107790001CD100206F4908706549C87604206749EC
:1077A00008706548C068079010F044F8CDE90801FA
:1077B0009DED080B08F038F98DED0A0B9DED0A0BD5
:1077C00051EC100B0FF028FA63490860B8E15B48F0
:1077D000007804287DD1604890ED000AF2EE040A9A
:1077E000B4EEE00AF1EE10FA12DD01205049C8763D
:1077F000514890ED020A5FEDB70AB4EEE00AF1EEEF
:1078000010FAE3DD0020C87605204C49087097E1A6
:107810004948C068019010F00DF8CDE902019DEDD6
:10782000020B08F001F98DED040B1FEDC90B53ECB1
:10783000102B9DED040B51EC100B0FF011FFCDE957
:1078400006019DED060B08F0EFF88DED080B1FED1E
:10785000D00B53EC102B9DED080B51EC100B0FF0DF
:10786000F3FCCDE90A019DED0A0B51EC100B0FF072
:10787000D3F93A490860084690ED000A5FEDD90A4D
:10788000B4EEE00AF1EE10FA05D290ED000A3448A9
:1078900080ED000A04E01FEDDF0A314880ED000AA8
:1078A00001202349C876234800680FF0C3FFCDE9C3
:1078B0000A012148806805900FF0BCFFCDE9060160
:1078C0009DED060B08F0B0F88DED080B9DED0A0B51
:1078D00000E0A6E053EC102B9DED080B51EC100BD3
:1078E0000FF076FC41D2134800680FF0A3FFCDE9FA
:1078F0000A011148C06805900FF09CFFCDE9060110
:107900009DED060B08F090F88DED080B9DED0A0B30
:1079100053EC102B9DED080B51EC100B0FF058FCA5
:1079200023D200200249C87605201BE0781F0020E2
:1079300054390220181F0020D43201200C1F0020CF
:10794000681F0020691F0020243B02200000000067
:107950000000F03F701F00206C1F00207C1F0020E3
:10796000801F002077490870EAE0774800680FF030
:1079700061FFCDE90A017548C06805900FF05AFF14
:10798000CDE906019DED060B08F04EF88DED080BD4
:107990009DED0A0B53EC102B9DED080B51EC100BD9
:1079A0000FF016FC06D200206949C876052065490B
:1079B0000870C5E0644800680FF03CFFCDE90A019B
:1079C0006248806805900FF035FFCDE906019DED16
:1079D000060B08F029F88DED080B9DED0A0B53EC12
:1079E000102B9DED080B51EC100B0FF0F1FB06D2A4
:1079F00000205749C876052052490870A0E0534836
:107A000090ED020A5348D0ED000AB4EEE00AF1EE20
:107A100010FA05DD00204E49C87605204949087056
:107A20008EE04848007805287ED14B48007803282E
:107A300003D104204649C87606E047480078042868
:107A400002D103204249C8764448806801900FF073
:107A5000F1FE9FED430B53EC102BCDE902019DEDA0
:107A6000020B51EC100B0FF0EFFBCDE904019DED83
:107A7000040B51EC100B0FF0CFF80690334890ED4B
:107A8000080A8DED050ADDED050A9DED060AFCF7F5
:107A900061FFDFED350A30EE600A8DED070A0798C9
:107AA0000FF0C8FECDE908019DED080B07F0BCFF03
:107AB0008DED0A0B9FED2D0B53EC102B9DED0A0B5A
:107AC00051EC100B0FF084FB3AD200202049C8760D
:107AD0002848006807900FF0ADFECDE908019DED44
:107AE000080B07F0A1FF8DED0A0B9FED230B53EC64
:107AF000102B9DED0A0B51EC100B0FF069FB1FD200
:107B00001F48006807900FF095FECDE908019DED34
:107B1000080B07F089FF8DED0A0B9FED170B53EC57
:107B2000102B9DED0A0B00E00AE051EC100B0FF05A
:107B30004FFB05D20020034908700120114908704D
:107B40000DB000BD0C1F0020181F0020D4320120F2
:107B500054390220801F0020691F0020243B02208E
:107B60006666666666A64C400000000000000000E5
:107B7000000000402C3301200000000000001440F1
:107B8000443301200D1F002010B52DED0C8BFE4855
:107B9000007800287ED0FD4890ED020A10EE101A01
:107BA00008460FF047FE41EC1C0B9FEDF90B53EC20
:107BB000102B0FF049FB41EC1B0B0FF02DF808EEDA
:107BC000100AB0EE480AFCF72DFE10EE104A2046CF
:107BD0000FF030FE41EC1A0B9FEDED0B53EC102B28
:107BE0000FF008F941EC190B0FF016F8EA4908609C
:107BF000E648D0ED020AB0EE600A0846D0ED000A71
:107C0000FDF7BAF8E54880ED000A00680FF012FEB3
:107C100041EC180B9FEDE20B53EC102B0FF012FC14
:107C20000AD2B3EE040AE04880ED000ABBEE040A73
:107C3000DE4880ED000A83E2D84800680FF0FAFDC4
:107C400041EC180B9FEDDA0B53EC102B0FF0C0FA40
:107C50000AD2BBEE040AD44880ED000AB3EE040A4F
:107C6000D24880ED000A6BE29FEDD30ACE4880ED4A
:107C7000000A9FEDD10ACD4880ED000A802005F072
:107C8000B1F94FF4007005F0EDFF0121CB4880F809
:107C9000BD1000E008E0002180F8BA1080F88D10D7
:107CA0000020B94908704BE2C54800680FF0C2FDDA
:107CB00041EC180BC34890ED020A10EE101A08466A
:107CC0000FF0B8FD41EC1A0BB0EE4A0AF0EE6A0A6A
:107CD00007F0AAFEB0EE409AF0EE609A53EC182B33
:107CE00051EC190B0FF074FA2CD2B54800680FF064
:107CF000A1FD41EC180BB34890ED030AB248D0ED5A
:107D0000000A30EE200A10EE101A08460FF092FD1D
:107D100041EC1A0BB0EE4A0AF0EE6A0A07F084FE54
:107D2000B0EE409AF0EE609A53EC182B51EC190B20
:107D30000FF04EFA06D2A5480078012802D19249E8
:107D40000870FDE10020A1490870904890ED020AFA
:107D500010EE101A08460FF06DFD41EC1A0B9FED66
:107D60008C0B53EC102B0FF06FFA41EC190B0EF04B
:107D700053FF08EE100AB0EE480AFCF753FD914895
:107D800080ED080A9248007801287CD18D4890ED5A
:107D9000030A9048D0ED000AB4EEE00AF1EE10FAC2
:107DA00005DB03208549C8768B49087036E0854895
:107DB00090ED030A8748D0ED000AF1EE600AB4EEB8
:107DC000E00AF1EE10FA05D204207C49C876824917
:107DD000087023E07A4800680FF02CFD41EC180B86
:107DE000784890ED020A10EE101A08460FF022FDB6
:107DF00041EC1A0BB0EE4A0AF0EE6A0A07F014FEE4
:107E0000B0EE409AF0EE609A53EC182B51EC190B3F
:107E10000FF018FB02D804206D4908705B4890ED04
:107E2000020A10EE101A08460FF004FD41EC1C0B7C
:107E30009FED570B53EC102B0FF006FA41EC1B0B88
:107E40000EF0EAFE08EE100A5E4890ED080AF0EE29
:107E5000400AB0EE480AFCF77DFDF1EE0C0A30EE68
:107E6000600A10EE104A20460FF0E4FC41EC1A0BB9
:107E7000B0EE4A0AF0EE6A0A07F0D6FDB0EE409A7C
:107E8000F0EE609A00E045E09FED540B53EC102BB0
:107E900051EC190B0FF09CF93BD200204749C876F2
:107EA00002204B490870474890ED030A10EE101A63
:107EB00008460FF0BFFC41EC1A0BB0EE4A0AF0EE98
:107EC0006A0A07F0B1FDB0EE409AF0EE609A9FEDBD
:107ED000450B53EC102B51EC190B0FF0B5F941EC9D
:107EE000180B0EF099FE41490860084690ED000A13
:107EF000DFED3F0AB4EEE00AF1EE10FA03DD9FED8C
:107F00003C0A80ED000A2F4890ED020A394880EDC6
:107F1000000A15E12E48007802287BD12749C8764F
:107F2000324800680FF086FC41EC180B31480068BD
:107F30000FF080FC41EC1B0B224890ED020A10EE82
:107F4000101A08460FF076FC41EC1D0BB0EE4D0AFE
:107F5000F0EE6D0A07F068FDB0EE40CAF0EE60CAC0
:107F600053EC1B2B51EC1C0B0FF07AFB41EC1A0B62
:107F7000B0EE4A0AF0EE6A0A07F056FDB0EE409AFB
:107F8000F0EE609A38E045E00E1F0020243B02200E
:107F90006666666666A64C40601F0020641F00206F
:107FA0007B14AE47E17A743F2C3301204433012027
:107FB0007B14AE47E17A74BF000000005439022000
:107FC000141F0020D43201205C1F0020101F00204D
:107FD0000F1F0020181F0020501F0020000000006D
:107FE0000000E03F0000000000001440541F00208B
:107FF00000000C42581F002053EC182B51EC190BB9
:108000000FF020FA05D200204F49C87603204F49CF
:10801000087095E04D480078032852D14C4800780C
:10802000032803D104204849C87606E04848007870
:10803000042802D103204449C876464890ED020A3C
:1080400010EE101A08460FF0F5FB41EC1C0B1FED6B
:10805000300B53EC102B0FF0F7F841EC1B0B0EF02C
:10806000DBFD08EE100A3C4890ED080AF0EE400AED
:10807000B0EE480AFCF76EFC5FED310A30EE600AA4
:1080800010EE104A20460FF0D5FB41EC1A0BB0EE73
:108090004A0AF0EE6A0A07F0C7FCB0EE409AF0EE2A
:1080A000609A1FED320B53EC102B51EC190B0FF0B3
:1080B0008FF845D200202449C8760420234908704F
:1080C0003EE02248007804283AD1234890ED020A85
:1080D0002248D0ED000AB4EEE00AF1EE10FA03DD1A
:1080E00002201949C87602E001201749C8761B48CA
:1080F00000680FF09FFB41EC180B174890ED020A47
:1081000010EE101A08460FF095FB41EC1A0BB0EE7A
:108110004A0AF0EE6A0A07F087FCB0EE409AF0EEE9
:10812000609A53EC182B51EC190B0FF051F807D251
:1081300000200549C87601200449087008490870E4
:10814000BDEC0C8B10BD0000543902200F1F002025
:10815000501F0020243B0220D4320120181F002091
:10816000101F002010B52DED0A8B964890ED020AE5
:1081700010EE101A08460FF05DFB41EC1C0B9FED52
:10818000920B53EC102B0FF05FF841EC1B0B0EF031
:1081900043FD08EE100A8E4890ED080AF0EE400A02
:1081A000B0EE480AFCF7D6FBDFED8A0A30EE600A33
:1081B00010EE104A20460FF03DFB41EC1A0BB0EEDA
:1081C0004A0AF0EE6A0A07F02FFCB0EE409AF0EE91
:1081D000609A51EC190B0EF01FFD7F4908607F4833
:1081E000007800287DD17E4800780028FAD17D48AB
:1081F000C07E05280ED2DFE800F0030E19248300AC
:108200009FED790A794880ED000A9FED770A78485A
:1082100080ED000AD1E0B3EE0E0A744880ED000A4A
:10822000B3EE0E0A724880ED000AC6E0BBEE0E0AFD
:108230006E4880ED000ABBEE0E0A6D4880ED000A24
:10824000BBE0654890ED000ADFED6A0AB4EEE00A93
:10825000F1EE10FA15DD6348B0F85A00404200EE26
:10826000100AB8EEC00A614880ED000A5D48B0F817
:108270005A0000EE100AB8EE400A5D4880ED000A90
:108280003DE0554800680FF0D5FA41EC180B9FED22
:108290005A0B53EC102B0FF0D5F826D25148B0F8FA
:1082A0005A0000EE100AB8EE400AB0EE402AF3EE93
:1082B000041AB3EE0E1AF6EE000A474890ED000AD3
:1082C0000BF008FF4E4880ED000A90ED000AB1EE79
:1082D000400A464880ED000A494890ED000A4448AB
:1082E00000E06BE080ED000A09E09FED3F0A3F48A7
:1082F00080ED000A9FED3C0A3D4880ED000A5CE0FD
:10830000354890ED000ADFED3B0AB4EEE00AF1EEED
:1083100010FA15DD3348B0F85A0000EE100AB8EE36
:10832000400A324880ED000A2E48B0F85A00404218
:1083300000EE100AB8EEC00A2D4880ED000A3BE0BE
:10834000254800680FF076FA41EC180B9FED2A0BD8
:1083500053EC102B0FF076F824D22248B0F85A00D4
:1083600000EE100AB8EE400AB0EE402AF3EE041A0E
:10837000B3EE0E1AF6EE000A174890ED000A0BF065
:10838000A9FE1F4880ED000A90ED000A174880ED15
:10839000000A1B4890ED000AB1EE400A144880ED37
:1083A000000A09E09FED100A104880ED000A9FEDD9
:1083B0000E0A0F4880ED000A00BF00BFBDEC0A8B1B
:1083C00010BD0000243B02206666666666A64C402F
:1083D000D43201200000B4428C1F00200E1F002068
:1083E0001C1F002054390220000000002C33012003
:1083F0004433012000003442000000000000E03F50
:10840000901F002000BFFEE730B505460C4622460F
:108410000021284600F001F830BD2DE9F041034667
:108420000C4617460FB9BDE8F08103B9FBE70025FC
:10843000002202E02D022543521C042AFAD33846BA
:1084400003F0030C1946BCF1000F08D0624603E0AC
:1084500001F8014B401E521C08B1042AF8D30E4605
:1084600001E020C6001F0428FBD2314602E001F8DB
:10847000014B401E0028FAD100BFD4E770B5044676
:108480000D461448D0F8040113490968401AB0F5A4
:10849000FA7F1DD90F48D0F804010F4908600D4834
:1084A000C07A50B10D4844718571002308220146FD
:1084B00040F20A60FBF784FD0AE00848447100209E
:1084C000064988710023082240F20A60FBF778FD14
:1084D00070BD000054390220A01400209014002028
:1084E0007047000070B5002100230F22C4781CB330
:1084F000174C246804F4E064C4F5E064C4F3072175
:10850000C1F10404E3B20A4144789C40E1B28478AA
:10851000144021430C07210E0E4C05786155047858
:1085200004F01F050124AC4005786D11AD0005F184
:10853000E025C5F8004109E0047804F01F05012496
:10854000AC40054D0678761145F8264070BD000018
:108550000CED00E000E400E080E100E002490143AE
:10856000024A1160704700000000FA050CED00E0BF
:1085700001460B48D0F804010A4A1268801A884262
:108580000AD90748D0F80401064A10600648007866
:1085900080F00100044A1070034800787047000022
:1085A00054390220DC170020E01700207047704784
:1085B00070B5044600F054F800201E4908701E49AA
:1085C00008701E4908701E4908601E4908601E494F
:1085D00008701E4908701E4908701E48006858B18E
:1085E0001D48056845B11B48066803E0761E00205B
:1085F00028602D1D002EF9D100201849087000F0C8
:1086000001FD00F02FFD204600F0DCFD208800B1C8
:1086100070BD204600F096FB208800B1F8E72046A8
:1086200001F0EEF8208800B1F2E7FFF7BFFF00BFCE
:10863000EEE70000D0070020D1070020D50700207A
:10864000E8070020EC070020D2070020D307002015
:10865000D4070020647A0108607A0108DE07002050
:10866000064800680649096800EB81000549086072
:108670000846006820F0070008607047607A01082B
:10868000647A0108F007002008480078012800D02B
:10869000704707480078FA2800DBF9E704480078BB
:1086A000401C0349087000BFF2E70000D10700201A
:1086B000D007002010B5002429480078012800D0F8
:1086C00010BD00BFF7F74EFE044600BF25480078F6
:1086D00028B900BF2046F7F749FE00BFF0E7214860
:1086E0000078401E1F49087008460078002805DD04
:1086F00000BF2046F7F73AFE00BFE1E71A480078CE
:10870000002805DD00BF2046F7F730FE00BFD7E7A1
:1087100000F064FC154908700846007800EB400042
:10872000134951F8200013490860084600681249AF
:108730000968884205D100BF2046F7F717FE00BF41
:10874000BEE70E480068401C0C490860FAF7CCFCF4
:1087500000BF2046F7F70AFE00BF00BFB0E70000E9
:10876000D1070020D0070020D5070020D307002024
:1087700038D90020EC070020E8070020D8070020A7
:1087800010B500241A480078002800DD10BD1948F3
:108790000078002800DDF9E700BFF7F7E3FD0446A5
:1087A00000BF00F01BFC144908700846007800EB7D
:1087B0004000124951F8200011490860084600683D
:1087C00010490968884205D100BF2046F7F7CEFD61
:1087D00000BFDBE70C480068401C0B490860FAF753
:1087E0007EFC00BF2046F7F7C1FD00BF00BFCDE70C
:1087F000D0070020D5070020D307002038D900205B
:10880000EC070020E8070020D807002010B5044638
:1088100012480078E8B900F0E1FB114908700846F9
:108820000078104908700E48007800EB40000E49AF
:1088300051F820000D490860084600680C4908609E
:10884000012006490870FAF739FC43F69920208088
:1088500002E045F68A60208010BD0000D1070020AC
:10886000D3070020D207002038D90020EC070020D1
:10887000E80700202DE9FF4F85B0044691469A464F
:10888000DDF854B0199E139D0020029012980F2815
:1088900009D13F48844206D046F273211A980180DC
:1088A00009B0BDE8F08F204600F098FC00211A982E
:1088B000018006F0010088B106F0020070B1A84600
:1088C0000020049007E00020C8F8000008F1040828
:1088D0000498401C049004985845F4D3149805EB70
:1088E00080000390CDE900B62A4651464846039BD6
:1088F00000F006F98046C4F82890C4F82CA0069829
:108900002062129884F83700C4F800800398A060B1
:1089100017986065189860606562C4F838B0A687DB
:10892000002706E0002104F15C0040F82710781CC5
:10893000C7B2002FF6D0204600F030F800BF00BFCD
:10894000F7F710FD029000BF00BF94F8370000F069
:1089500065FB204600F0CEFB0E480088401C0D4908
:1089600008800D480078012807D000BF00BF02989A
:10897000F7F7FCFC00BF00BF92E700BF00BF029802
:10898000F7F7F4FC00BF00BFFFF7FAFE00BF87E770
:10899000D0D80020DC070020D107002070477047A6
:1089A0002DE9F0470746884614461D464FF000095A
:1089B0000CB10020206000BF00BFF7F7D3FC814658
:1089C00000BF00BF43480068406CD0B14148006818
:1089D000406C401E3F49096848643E480068466C48
:1089E0001CB13C480068006C206000BF00BF4846D6
:1089F000F7F7BCFC00BF00BF002028803046BDE870
:108A0000F08708F4004058B100BF00BF4846F7F7B0
:108A1000ADFC00BF00BF46F2B01028800020EEE79A
:108A20002D48007800280BDD00BF00BF4846F7F74F
:108A30009DFC00BF00BF46F6635028800020DEE7A3
:108A40003B4607220021084600F0B4F900BF00BFF2
:108A50004846F7F78BFC00BF00BFFFF791FE00BF51
:108A600000BFF7F77FFC814600BF00BF19480068D0
:108A700090F8350020B101280AD0032818D110E061
:108A80001CB114480068006C20600020288013E0AE
:108A90001CB110480068006C206046F2A9102880C4
:108AA0000AE00CB10020206047F2D920288003E0C2
:108AB00046F62E60288000BF00BF06480068466C5E
:108AC00000BF00BF4846F7F751FC00BF00BF30466B
:108AD00095E70000E8070020D50700202DE9F041C8
:108AE00005460E4614464FF00008234642463146DE
:108AF000284600F0C9FB07463846BDE8F081000073
:108B0000F0B50446DDE9055602EB850020F00700CC
:108B10004FF0807C071F3846C7F800C0071F384653
:108B20003C60DFF8A8C0071F3846C7F800C04FF008
:108B3000123C071F3846C7F800C04FF0033C071F20
:108B40003846C7F800C04FF0023C071F3846C7F848
:108B500000C0071F38463B60071F384639604FF09A
:108B6000113C071F3846C7F800C04FF0103C071FE4
:108B70003846C7F800C04FF0093C071F3846C7F811
:108B800000C04FF0083C071F3846C7F800C04FF040
:108B9000073C071F3846C7F800C04FF0063C071FC8
:108BA0003846C7F800C04FF0053C071F3846C7F8E5
:108BB00000C04FF0043C071F3846C7F800C06FF0F4
:108BC000020C071F3846C7F800C0F0BD65920008C8
:108BD000704700002DE9F04105460E461446002777
:108BE00026480078002804DD46F663502080BDE862
:108BF000F08136B1022E05D0042E0AD0082E09D1FC
:108C000001E000BF00BF1DB947F27E202080EEE7E3
:108C100004E003E045F625602080E8E700BF00BFE0
:108C200000BFF7F79FFB074600BF00BF01201449B4
:108C3000096881F836002346324629461048006804
:108C400000F018FC208838B100BF00BF3846F7F7A5
:108C50008DFB00BF00BFCAE70948006800F068FA52
:108C600000BF00BF3846F7F781FB00BF00BFFFF72A
:108C700087FD0020208000BFB9E70000D507002055
:108C8000E807002070B50446002600BF00BFF7F7D4
:108C900069FB064600BF00BF0648056800BF00BF6D
:108CA0003046F7F763FB00BF00BF00202080284656
:108CB00070BD0000E007002008B500F009F86A4622
:108CC00000210248FFF70AFF08BD0000F8D9002084
:108CD0007047000010B5002400BF00BFF7F742FB4B
:108CE000044600BF00BF08480078401C06490870D1
:108CF00000BF00BF2046F7F739FB00BF00BFFFF7FA
:108D0000DBFFFFF7D7FC10BDD0070020002400BF19
:108D100014E000BF00BFF7F725FB044600BF00BF0B
:108D200007480068401C0649086000BF00BF204695
:108D3000F7F71CFB00BF00BFFFF739FCE9E70000B5
:108D4000CC07002010B58AB0044600200E49086008
:108D50000B2000210591CDE90704069108460B4937
:108D600009680B4A12680B4B1B68CDE90132CDE94B
:108D700003100F200023084A08A100900C48FFF7B9
:108D800079FD0AB010BD0000CC0700203C7A010834
:108D9000387A0108347A01080D8D000875432F4F89
:108DA000532D4949492049646C65205461736B0017
:108DB000D0D800202DE9F04105460C4616461F4646
:108DC0001248006880F8346000201049096881F872
:108DD000350039460D48006800F0D8F96CB104F14F
:108DE0000808EC60012229460848006800F010F8E5
:108DF0002946404600F01FF806E0002003490968B4
:108E0000C887024909680863BDE8F081E8070020C7
:108E100010B5C287016300230AE000244C600C6097
:108E20000C614C610C83CC61886020315C1CA3B266
:108E30009342F2DB10BDF0B58E6896F83750078983
:108E40003FB90127078100274F600F600160416033
:108E500023E007897F1C0781026806E0946894F884
:108E60003770AF4200DD02E05268002AF6D100BF41
:108E700032B900274F6043680B60596041600CE0D5
:108E800017682FB9116000270F604A60016004E085
:108E900013680B604A6059601160F0BD2DE9F04124
:108EA0000446256BE68F0AE0D5F80C8008F1080728
:108EB0002946384600F00AF82035701E86B2002E8A
:108EC000F2DC0020E0872063BDE8F08110B5048962
:108ED000012C03D100240460446011E00C6824B923
:108EE0004A680024146002600AE04C6824B90B68E8
:108EF00000245C60436003E00B684A685A601360BA
:108F00000489641E048100244C600C6010BD2DE9AE
:108F1000F84306460C4617469846089D94F83600D6
:108F2000082842D2DFE800F00405080906072425D6
:108F300000BF00BF00BF39E000BF94F83400032831
:108F400007D143463A4621463046009500F031F8B5
:108F500000E0256416B12046FFF7A0FF204600F090
:108F600073F900203434A070607004F834091DE0F7
:108F700000BF94F83400032807D143463A462146FF
:108F80003046009500F015F800E02564204600F01A
:108F90004FFB16B12046FFF781FF04203434A07048
:108FA0000020607004F8340900E000BF00BFBDE895
:108FB000F883F0B50446059E086BCD8F0AE0C768BC
:108FC000A74204D1046142610383C66104E02030FA
:108FD0006F1EBDB2002DF2DC00BFF0BD70B50025E4
:108FE000074C03E005F12000C5B2241D20680028CD
:108FF000F8D02068F7F7C1F92844C5B2284670BDFB
:10900000C8070020002004E00021034A42F8201095
:10901000401C0028F8D07047C807002030B542092E
:1090200000F01F030121C3F11F04A140034C54F8B9
:1090300022400C43014D45F8224030BDC8070020B6
:1090400030B5420900F01F030121C3F11F04A14004
:10905000034C54F822408C43014D45F8224030BD6A
:10906000C807002000210AE001EB4102054B03EB99
:10907000820000220281026042604A1CD1B21029A3
:10908000F2D3704738D9002010B5044694F8370061
:10909000FFF7C4FF94F8370005490978884203D1E7
:1090A000204600F027F802E0204600F003F810BD4B
:1090B000D207002010B590F8373003EB43030C4C77
:1090C00004EB83010B893BB901230B810023C360AF
:1090D00003610860486009E00B895B1C0B810B6829
:1090E000C360002303610A681061086010BD0000BE
:1090F00038D9002010B590F8373003EB43030B4C00
:1091000004EB83010B893BB901230B810023C3606E
:1091100003610860486008E00B895B1C0B81002339
:10912000C3604A680261D060486010BD38D9002031
:109130002DE9F041054695F8370000EB4000124953
:1091400001EB80042F69EE6887B946B900202081C1
:109150002060606095F83700FFF772FF0EE020890D
:10916000401E208100203061266007E02089401EDB
:109170002081FE600EB9676000E037610020286141
:10918000E860BDE8F081000038D9002038B5044619
:109190000D4685B16B4602222946204600F06AF949
:1091A000BDF8000018B9032084F8360006E002205C
:1091B00084F8360002E0022084F836002046FFF7EB
:1091C000B7FF38BD0021034A1180034A11600180B6
:1091D00070470000DC070020D80700200022026052
:1091E00082604260C260026142618261C26114A217
:1091F0000262002242628262C2620264002106E0D0
:10920000002300F15C0242F821304A1CD1B200294F
:10921000F6D000223430026142600263C2620281F1
:109220004FF00042426100228261C26102624262EA
:109230000270427082701022C27034387047000091
:109240003F5461736B00000010B50446204600F0E7
:10925000EFF994F8360000F0040010B92046FFF74B
:1092600013FF10BD08B506480068FFF798FB00BF64
:109270006A46002103480068FFF7ACFCF8E70000ED
:10928000E8070020947A01082DE9F843044688464F
:1092900017461D464FF0000900BF00BFF7F762F800
:1092A000814600BF00BF0CB96748046827640020EE
:1092B000288094F83600082876D2DFE800F004050C
:1092C00050510607525300BF00BF00BF04200128C1
:1092D00004D0022813D0042833D122E0606CFF2888
:1092E0000CD100BF00BF4846F7F740F800BF00BFF1
:1092F00046F6C55028800020BDE8F88322E04FF6EE
:10930000FF71606C88420BD100BF00BF4846F7F781
:109310002DF800BF00BF46F6C55028800020EBE7BF
:1093200010E0606C401C58B900BF00BF4846F7F71A
:109330001DF800BF00BF46F6C55028800020DBE7BF
:1093400000E000BF00BF606C401C6064666C00BF42
:1093500000BF4846F7F70AF800BF00BF71E000BF42
:1093600000BF00BF94F83400072815D100231A4627
:10937000214618460097FFF7CAFD666C00BF00BF84
:109380004846F6F7F3FF00BF00BF08F4004000288E
:109390004AD1FFF7F5F947E00420012805D002285B
:1093A00013D0042833D122E03FE0606CFF280BD1BA
:1093B00000BF00BF4846F6F7D9FF00BF00BF46F622
:1093C000C5502880002097E722E04FF6FF71606CBF
:1093D00088420BD100BF00BF4846F6F7C7FF00BF69
:1093E00000BF46F6C5502880002085E710E0606C7D
:1093F000401C58B900BF00BF4846F6F7B7FF00BF92
:1094000000BF46F6C5502880002075E700E000BF89
:1094100000BF606C401C6064666C00BF00BF4846C3
:10942000F6F7A4FF00BF00BF0BE000BF00BF484637
:10943000F6F79CFF00BF00BF46F62D60288000268F
:1094400000BF00BF304657E7E8070020002108E0D2
:10945000064A02EBC100002202608280C2804A1CE0
:1094600091B2034A12889142F2DB704750D8002033
:10947000AC7A01082DE9F04F0C4616461D46042E25
:109480001ED1DFF8A091D9F80090A4EB0909A9F149
:10949000010313F5803F0DD94FF00009C0F84C903F
:1094A000C0F85090C0F81C9047F27E29A5F80090B3
:1094B000BDE8F08FC46403F10109C0F850903FE0AB
:1094C00084B3082E25D1D0F8489009EB0407DFF8C3
:1094D0005491D9F80090A7EB0909A9F10103A3421F
:1094E00001D2C76406E0DFF83C91D9F80090A144AE
:1094F000C0F84C90DFF82CA1D0F84C90DAF800A01E
:10950000A9EB0A09C0F85090D0F84C90C0F84890E8
:1095100016E0DFF81091D9F80090A144C0F84C9003
:1095200004650DE0FFE74FF00009C0F84C90C0F86B
:109530005090C0F81C9047F27E29A5F80090B7E73C
:10954000DFF8E4A0BAF800A0D0F84C90B9FBFAFB21
:109550000AFB1B991FFA89F8DFF8D09009EBC802C3
:10956000B2F80490B9F1000F0BD14FF00009C0F828
:109570001490C0F8189010604FF00109A2F8049000
:109580003EE0116834E0DFF89CA0D1F84C90DAF8A6
:1095900000A0A9EB0A09C1F85090D0F85090D1F87A
:1095A00050A0D1450ED9D1F81490B9F1000F01D0D7
:1095B00049691DE04FF00009C0F8149081614861CD
:1095C000002115E0D1F81890B9F1000F07D14FF044
:1095D0000009C0F8189041618861106007E0D1F877
:1095E00018C0C0F818C04161CCF81400886100218F
:1095F0000029C8D1B2F8049009F10109A2F8049039
:10960000B2F80690B2F804A0D14503DAB2F804909B
:10961000A2F80690C2614FF00009A5F8009000BFC3
:1096200046E70000E0070020AC7A010850D800208F
:1096300010B5C269BAB1002404651468844205D12A
:109640004169116039B100248C6104E0816943698A
:109650004B6103B19961002444618461C461C464B5
:109660009488641E948010BD2DE9F05F4FF0000BCC
:1096700000BF00BFF6F776FE834600BF00BF4FF085
:10968000000A50480068401C4E49086008460068BF
:109690004D490988B0FBF1F201FB12001FFA80F975
:1096A0004A4800EBC9073C68002678E0002C75D0DA
:1096B000D4F8148094F8360008286BD2DFE800F064
:1096C0000408051B0638074B00BF00BF00BF62E05F
:1096D0003C49E06C0968401A20653A49E06C096829
:1096E000884206D1002084F836002046FFF7ACFD02
:1096F00000E001264FE03349E06C0968401A20651C
:109700003049E06C0968884210D10020206420466E
:10971000FFF7C4FB2046FFF797FD00203434A0700C
:1097200003206070002004F8340900E0012632E0D4
:109730002449E06C0968401A20652249E06C0968F8
:10974000884206D1042084F836002046FFF770FFD7
:1097500000E001261FE01B49E06C0968401A206503
:109760001849E06C0968884210D100202064204626
:10977000FFF794FB2046FFF75BFF04203434A07012
:1097800003206070002004F8340900E0012602E0A4
:1097900004E0FFE700BF00BF444600E00126002EC2
:1097A00084D0CAF100050A480068A84201D20848DE
:1097B000056000BF00BF5846F6F7D8FD00BF00BFE8
:1097C000BDE8F09FE0070020AC7A010850D80020E7
:1097D000E40700201CB500BF0EE001AB6A46002183
:1097E0000846FFF7DDF8BDF8040028B90348007803
:1097F000012801D1FFF738FFEFE70000D107002073
:1098000010B58AB0044600201D4908601D49086053
:10981000FFF71CFE1C48006820B947F21220208088
:109820000AB010BD1948006819490968884203D276
:1098300047F213202080F3E7164800780F2803D35F
:1098400047F211202080EBE70B20002105910A460A
:10985000CDE9070406910D4800680F4909680A4BD5
:109860001B68CDE90131CDE903020A4800780023E5
:109870000A4A0BA100900F48FEF7FCFF00BFCFE79C
:10988000E0070020E40700209C7A0108A47A010880
:10989000907A0108987A0108A07A0108D597000803
:1098A00075432F4F532D494949205469636B205408
:1098B00061736B00F8D9002030B505460C461CB129
:1098C000284603F063FB02E0284604F03DFA30BD71
:1098D00010B5002409F0B8FC00F00104002C1FD1E1
:1098E00010A1012005F0FAF900BF00BF2046621C5C
:1098F000D4B208F0A1FC042CF8DB00240AE009F043
:10990000A3FC00F001040DA0F6F754FD4FF4FA702B
:1099100007F012FF002CF2D009A1012005F0DEF9BA
:1099200010BD0000C7EBBCECB2E9CDF8CFDFCAC771
:10993000B7F1C1ACBDD33F0D0A000000202E0000DE
:10994000CDF8CFDFD2D1C1ACBDD3A3A10D0A0000A9
:109950000FB438B5002400BF05A800900548009A50
:109960000499F6F715FD044600200090014838BC24
:109970005DF814FBB433012030B52DED068B91B0AA
:1099800004460D469FEDF80A8DED100A9FEDF60A8C
:109990008DED0F0A9FEDF40A8DED0E0A00200D905B
:1099A0000C900B900A90099009A80AA90BAA0CAB7D
:1099B000CDE90432CDE906100DA80EA90FAA10AB0F
:1099C000CDE90032CDE90210E84BE94AE9A1204691
:1099D000F6F7ACFEE648006842F20F71884215D0F7
:1099E000E3480068EC490860E048006848600120EE
:1099F00081F82500084690F82600B0B1042003F055
:109A0000F1FA0020E44981F826000EE0E348D0F89E
:109A1000A800B0F5007F04D0E048D0F8A8004028A6
:109A200003D10020DC4981F825000B98012842F081
:109A3000BB879DED100ADFEDDA0A30EE600AB1EE69
:109A4000400A10EE101A08460DF0F4FE41EC190B16
:109A50009FEDD40B53EC102B0DF0F6FB41EC180BE3
:109A60000DF0DAF8CC49C8609DED0F0ADFEDCF0AA2
:109A700030EE600AB1EE400A10EE101A08460DF002
:109A8000D9FE41EC190B9FEDC70B53EC102B0DF0D9
:109A9000DBFB41EC180B0DF0BFF8BF498860BF48F5
:109AA000B0F844004AF20101884219D1BA4840682E
:109AB00040F26A41884214D1B748006847F23051F9
:109AC00088420ED1B44890ED030AF1EE000A30EE60
:109AD000200A80ED030A9FEDB60AB04880ED170A10
:109AE000E6E1AD48406840F26A4188420BD1AA489D
:109AF000006847F6E011884205D19FEDAE0AA748FD
:109B000080ED170AD4E1A4484068E630E0B9A248E5
:109B1000006849F25011884216D19FED930A9F4880
:109B200080ED170A9C4890ED020AF0EE000A30EE34
:109B3000600A80ED020A90ED030AF1EE000A30EEB1
:109B4000600A80ED030AB3E193484068E630E0B96B
:109B50009148006842F6E061884216D1BFEE000AE3
:109B60008E4880ED170A8C4890ED020AD0ED050A68
:109B700030EE200A80ED020A90ED030AF2EE080AA8
:109B800030EE200A80ED030A92E183484068B0F588
:109B9000877F14D1804800684AF6705188420ED100
:109BA0007D4890ED030AF1EE000A30EE200A80EDC8
:109BB000030A9FED810A794880ED170A78E176481B
:109BC000406840F27E41884217D17348006845F6EC
:109BD0001011884211D1704890ED030AF1EE000A8D
:109BE00030EE200A80ED030A90ED020AF1EE040A3D
:109BF00030EE200A80ED020A5AE167484068B0F56D
:109C0000877F0BD16448006844F2A011884205D1D7
:109C10009FED6A0A614880ED170A49E15E48406895
:109C2000B0F58C6F0BD15C48006841F270718842CE
:109C300005D19FED600A594880ED170A38E1564872
:109C4000406840F26A4188420AD153480068B0F542
:109C5000965F05D19FED570A504880ED170A27E11E
:109C60004D48406843F22C31884214D14A4800687C
:109C700049F2907188420ED19FED510A474880ED1C
:109C8000170A454890ED030AF2EE000A30EE600A2A
:109C900080ED030A0CE14048406843F22C318842D1
:109CA00014D13D4800684BF24C3188420ED19FEDF3
:109CB000440A3A4880ED170A374890ED030AF2EE5D
:109CC0000C0A30EE200A80ED030AF1E032484068C9
:109CD00043F22C3188420AD12F480068B0F52F4F4B
:109CE00005D19FED380A2D4880ED170AE0E02A489B
:109CF000406843F22C31884214D12748006849F665
:109D00000E4188420ED19FED180A244880ED170AB3
:109D1000214890ED030AF3EE000A30EE200A80EDB0
:109D2000030AC5E01C4840681E30E0B91A480068C4
:109D30004BF68031884247D1B6EE000A174880EDD5
:109D4000170A154890ED020AF1EE000A30EE200ADB
:109D500080ED020A90ED030AF2EE040A30EE200ACA
:109D600080ED030AA4E02FE000000000901900201D
:109D70008C1900203C2564585925644028256678B4
:109D800025662925664025784025784025642D25BF
:109D9000642D25643E000000D43201205439022095
:109DA0000000C843333333333333CB3F0000964393
:109DB0009A99993ECDCC4CBECDCCCC3D9A9999BECA
:109DC000CDCCCCBE9A9999BFF7484068E630E0B94F
:109DD000F54800684CF64061884216D19FEDF30AC1
:109DE000F34880ED170AF04890ED020AF0EE080AF9
:109DF00030EE600A80ED020A90ED030AF1EE000AEF
:109E000030EE600A80ED030A52E0E748406840F215
:109E1000CA3188421CD1E44800684CF6406188424F
:109E200016D1B7EE080AE24880ED170ADE4890ED39
:109E3000030AF1EE000A30EE200A80ED030A90EDED
:109E4000020AF0EE000A30EE600A80ED020A2FE00E
:109E5000D5484068D74988420BD1D348006844F6BA
:109E60007C41884205D11FED400AD14880ED170A98
:109E70001EE0CD484068CF49884214D1CA480068E6
:109E800045F2221188420ED11FED340AC84880EDF8
:109E9000170AC54890ED020AF0EE000A30EE600A9B
:109EA00080ED020A04E01FED3E0AC14880ED170A6A
:109EB000BF48B0F844004AF20201884217D1BA48BC
:109EC0004068F52814D1B84800684AF21041884229
:109ED0000ED1B54890ED030AF1EE080A30EE600AA3
:109EE00080ED030A1FED4E0AB14880ED170AF0E13C
:109EF000AD48406840F26A41884214D1AA480068DF
:109F000047F6E01188420ED11FED570AA84880EDB0
:109F1000170AA54890ED030AF2EE000A30EE600A37
:109F200080ED030AD5E1A048406840F26A418842CA
:109F30000BD19D48006847F23051884205D11FED92
:109F4000760A9B4880ED170AC3E197484068E630DF
:109F5000E0B99548006849F25011884216D1B6EE32
:109F6000000A934880ED170A8F4890ED020AF1EE3F
:109F7000080A30EE600A80ED020A90ED030AF2EE64
:109F80000C0A30EE600A80ED030AA2E186484068C0
:109F9000E63058B98448006842F6E061884205D14D
:109FA0001FED8F0A824880ED170A92E17E484068D3
:109FB00040F27E41884214D17B48006845F26041FE
:109FC00088420ED11FED860A794880ED170A76483F
:109FD00090ED030AF2EE000A30EE600A80ED030A0B
:109FE00077E171484068B0F5877F1CD16E48006802
:109FF00044F2A011884216D11FED920A6C4880ED00
:10A00000170A694890ED020AF1EE000A30EE600A84
:10A0100080ED020A90ED030AF1EE000A30EE600ACC
:10A0200080ED030A55E16048406840F26A41884289
:10A0300013D15D480068B0F5965F0ED11FEDB60AEA
:10A040005B4880ED170A584890ED030AF2EE080AC3
:10A0500030EE600A80ED030A3BE153484068B0F5FA
:10A060008C6F14D15048006841F2707188420ED153
:10A070001FEDC30A4E4880ED170A4B4890ED030AC6
:10A08000F1EE080A30EE600A80ED030A21E146484D
:10A09000406843F22C31884214D1434800684BF2A7
:10A0A0004C3188420ED11FEDD00A414880ED170A8D
:10A0B0003D4890ED030AF1EE080A30EE200A80EDEB
:10A0C000030A06E13848406843F22C31884213D134
:10A0D00035480068B0F52F4F0ED1BFEE000A344866
:10A0E00080ED170A304890ED030AF1EE000A30EED9
:10A0F000600A80ED030AECE02B48406843F22C3103
:10A10000884214D12848006849F60E4188420ED191
:10A110001FEDEB0A264880ED170A234890ED030A4D
:10A12000F1EE000A30EE600A80ED030AD1E01E482D
:10A13000406843F22C31884214D11B48006849F230
:10A14000907188420ED11FEDF80A194880ED170A68
:10A15000154890ED030AF2EE0C0A30EE600A80ED2D
:10A16000030AB6E0104840681E30E0B90E480068A7
:10A170004BF6803188421FD11FEDF10A0C4880ED6B
:10A18000170A094890ED020AF1EE000A30EE600A63
:10A1900080ED020A90ED030AF2EE0C0A30EE200A7E
:10A1A00080ED030A95E007E0D4320120CDCCCC3F0E
:10A1B00054390220BAF5FFFFFD484068E630E0B9A7
:10A1C000FB4800684CF64061884216D1B6EE000AA2
:10A1D000F84880ED170AF64890ED020AF1EE080AF9
:10A1E00030EE600A80ED020A90ED030AF2EE000AFA
:10A1F00030EE600A80ED030A6BE0ED48406840F203
:10A20000CA3188421CD1EA4800684CF64061884255
:10A2100016D19FEDE90AE74880ED170AE44890ED72
:10A22000020AF1EE080A30EE600A80ED020A90EDB3
:10A23000030AF1EE080A30EE600A80ED030A48E0F6
:10A24000DB484068DD4988421CD1D948006844F6A3
:10A250007C41884216D19FEDDA0AD64880ED170A74
:10A26000D34890ED020AF1EE080A30EE600A80ED64
:10A27000020A90ED030AF2EE0C0A30EE600A80ED5D
:10A28000030A26E0CA484068CC4988421CD1C84825
:10A29000006845F22211884216D1BFEE000AC54877
:10A2A00080ED170AC24890ED020AF1EE080A30EE7E
:10A2B000600A80ED020A90ED030AF2EE080A30EE21
:10A2C000600A80ED030A04E0B6EE000AB94880EDAA
:10A2D000170AB848B0F844004AF2030188420ED188
:10A2E000B3484068F5280BD1B14800684AF21041E4
:10A2F000884205D1B6EE000AAE4880ED170A60E24A
:10A30000AB48406840F2CA31884211D1A848006881
:10A310004DF2A071884205D0A54800684DF6504125
:10A32000884205D19FEDA70AA24880ED170A48E2AE
:10A330009F48406840F2CA3188420AD19C48006870
:10A34000B0F5614F05D19FEDA00A9A4880ED170A3C
:10A3500037E29748406840F62A5188420BD194482A
:10A3600000684EF2B051884205D19FED960A91489F
:10A3700080ED170A25E28E484068B0F52F7F14D192
:10A380008B4800684DF2A071884204D0884800686C
:10A39000B0F5614F09D1864890ED020AF1EE040A4A
:10A3A00030EE600A80ED020A0BE28148406840F21C
:10A3B0006A4188420BD17E48006847F6E011884226
:10A3C00005D19FED820A7B4880ED170AF9E17848B4
:10A3D000406840F27E4188420FD17548006845F2DE
:10A3E0006041884209D1724890ED030AF3EE040AF5
:10A3F00030EE600A80ED030AE3E16D48406840F208
:10A400007E41884214D16A48006845F6101188429E
:10A410000ED1B6EE000A674880ED170A644890ED49
:10A42000030AF1EE000A30EE600A80ED030AC8E18B
:10A430005F484068B0F5877F14D15D48006844F2FA
:10A44000A01188420ED19FED620A5A4880ED170A8A
:10A45000574890ED030AF2EE0C0A30EE600A80EDE8
:10A46000030AAEE15248406840F2BE5188420BD127
:10A470004F48006844F2A011884205D19FED550A6B
:10A480004C4880ED170A9CE149484068E630E0B945
:10A490004748006849F25011884216D19FED490A99
:10A4A000444880ED170A424890ED020AF1EE080A8E
:10A4B00030EE600A80ED020A90ED030AF3EE080A1E
:10A4C00030EE600A80ED030A7BE139484068E630EF
:10A4D000E0B93748006842F6E061884216D19FED46
:10A4E0003A0A344880ED170A314890ED020AD0ED5F
:10A4F000050A30EE200A80ED020A90ED030AF2EE22
:10A500000C0A30EE600A80ED030A5AE128484068E0
:10A51000E630B8B92648006849F25011884211D196
:10A52000234890ED020AF1EE080A30EE600A80ED51
:10A53000020A90ED030AF0EE000A30EE600A80EDA8
:10A54000030A3EE11A48406843F22C31884214D194
:10A55000174800684BF24C3188420ED19FED190A22
:10A56000144880ED170A124890ED030AF0EE000A35
:10A5700030EE600A80ED030A23E10D48406843F2A3
:10A580002C31884228D10A480068B0F52F4F23D1DA
:10A59000BEEE000A074880ED170A054890ED030A51
:10A5A000F3EE020A30EE600A80ED030A09E10000D2
:10A5B000D4320120543902203333333FBAF5FFFF40
:10A5C000CDCC4CBF00000000CDCC4CBE85EB113F84
:10A5D000CDCC4C3E6666663FFD48406843F22C3168
:10A5E000884214D1FA48006849F60E4188420ED1DB
:10A5F0001FED0C0AF74880ED170AF54890ED030AA5
:10A60000F0EE080A30EE600A80ED030AD9E0F04867
:10A61000406843F22C31884214D1ED48006849F279
:10A62000907188420ED11FED190AEA4880ED170A91
:10A63000E74890ED030AF3EE040A30EE600A80ED7D
:10A64000030ABEE0E24840681E30E0B9E048006816
:10A650004BF68031884216D1B7EE080ADD4880ED0E
:10A66000170ADB4890ED020AF1EE000A30EE600AAC
:10A6700080ED020A90ED030AF1EE000A30EE600A66
:10A6800080ED030A9DE0D248406840F67A01884296
:10A690000AD1CF480068B0F5965F05D11FED330AA7
:10A6A000CC4880ED170A8CE0C9484068E630E0B934
:10A6B000C74800684CF64061884216D19FEDC60A33
:10A6C000C44880ED170AC24890ED020AF2EE000A73
:10A6D00030EE600A80ED020A90ED030AF3EE000A04
:10A6E00030EE600A80ED030A6BE0B948406840F242
:10A6F000CA3188421CD1B64800684CF64061884295
:10A7000016D1B7EE080AB34880ED170AB04890EDAD
:10A71000020AF2EE000A30EE600A80ED020A90EDC5
:10A72000030AF2EE0C0A30EE600A80ED030A48E0FC
:10A73000A7484068A94988421CD1A548006844F64A
:10A740007C41884216D19FEDA60AA24880ED170AE7
:10A750009F4890ED020AF1EE080A30EE600A80EDA3
:10A76000020A90ED030AF3EE000A30EE600A80ED73
:10A77000030A26E096484068984988421CD19448CC
:10A78000006845F22211884216D11FED720A9148E5
:10A7900080ED170A8E4890ED020AF2EE000A30EEC4
:10A7A000600A80ED020A90ED030AF3EE020A30EE31
:10A7B000600A80ED030A04E01FED7C0A854880ED05
:10A7C000170A8448B0F844004AF20401884217D1BD
:10A7D0007F484068F52814D17D4800684AF210414E
:10A7E00088420ED11FED860A7A4880ED170A784814
:10A7F00090ED030AF2EE000A30EE600A80ED030AE3
:10A8000060E273484068B0F5877F14D170480068F3
:10A810004AF6705188420ED19FED720A6D4880ED64
:10A82000170A6B4890ED030AF1EE000A30EE600A59
:10A8300080ED030A46E266484068E630E0B96448C5
:10A84000006849F25011884216D1B6EE000A6148FC
:10A8500080ED170A5E4890ED020AD0ED050A30EE51
:10A86000200A80ED020A90ED030AF3EE020A30EEB0
:10A87000600A80ED030A25E255484068E630E0B9F9
:10A880005348006842F6E061884216D1BEEE000AE5
:10A89000504880ED170A4E4890ED020AD0ED050AA7
:10A8A00030EE200A80ED020A90ED030AF1EE080A6C
:10A8B00030EE600A80ED030A04E245484068B0F5D6
:10A8C000877F14D14248006844F2A01188420ED11B
:10A8D0003F4890ED030AF2EE040A30EE600A80ED84
:10A8E000030A9FED410A3B4880ED170AEAE1384828
:10A8F000406840F26A41884214D13548006847F206
:10A90000305188420ED19FED390A324880ED170A46
:10A910002F4890ED030AF1EE000A30EE600A80ED58
:10A92000030ACFE12A48406840F67A0188420BD1F9
:10A930002748006845F61011884205D19FED290A85
:10A94000244880ED170ABDE12148406840F27E416D
:10A9500088420FD11E48006845F61011884209D17F
:10A960001B4890ED020AF2EE000A30EE200A80ED5C
:10A97000020AA7E11648406840F27E41884214D19D
:10A980001348006845F2604188420ED11FEDF00A7D
:10A99000104880ED170A0E4890ED030AF1EE000A08
:10A9A00030EE600A80ED030A8CE10948406840F609
:10A9B0007A0188421CD10648006841F270718842D1
:10A9C00016D19FED070A034880ED170A7AE10000CF
:10A9D000D432012054390220CDCC8C3FBAF5FFFF90
:10A9E0009A99993ECDCCCC3ECDCCCC3DCDCCCCBDF6
:10A9F000FE484068B0F58C6F14D1FC48006841F205
:10AA0000707188420ED11FED080AF94880ED170ACF
:10AA1000F64890ED030AF1EE080A30EE600A80ED88
:10AA2000030A4FE1F148406840F26A41884216D17A
:10AA3000EE480068B0F5965F11D1EC4890ED020A3F
:10AA4000F1EE080A30EE200A80ED020A90ED030ACA
:10AA5000F2EE080A30EE600A80ED030A32E1E348C4
:10AA6000406843F22C31884213D1E0480068B0F5C9
:10AA70002F4F0ED1BFEE080ADD4880ED170ADB48E4
:10AA800090ED030AF1EE080A30EE600A80ED030A49
:10AA900018E1D648406843F22C31884214D1D3489B
:10AAA000006849F60E4188420ED1BEEE000AD04839
:10AAB00080ED170ACD4890ED030AF2EE040A30EE5D
:10AAC000200A80ED030AFDE0C848406843F22C31BB
:10AAD000884214D1C548006849F2907188420ED16D
:10AAE000BEEE000AC24880ED170AC04890ED030A86
:10AAF000F3EE020A30EE600A80ED030AE2E0BB48A2
:10AB0000406843F22C31884214D1B84800684BF2B7
:10AB10004C3188420ED19FEDB70AB54880ED170A37
:10AB2000B24890ED030AF1EE000A30EE200A80ED03
:10AB3000030AC7E0AD4840681E30A0B9AB480068C2
:10AB40004BF6803188420ED19FEDAA0AA84880EDCD
:10AB5000170AA64890ED030AF2EE0C0A30EE200A1E
:10AB600080ED030AAEE0A148406842F6E061884209
:10AB70000AD19E480068B0F52F4F05D19FED9D0A80
:10AB80009B4880ED170A9DE098484068E630E0B9A0
:10AB9000964800684CF64061884216D1B7EE000A2C
:10ABA000934880ED170A914890ED020AF1EE000AF1
:10ABB00030EE600A80ED020A90ED030AF1EE080A19
:10ABC00030EE600A80ED030A7CE08848406840F27D
:10ABD000CA3188421CD1854800684CF640618842E1
:10ABE00016D1B7EE000A824880ED170A7F4890ED33
:10ABF000030AF1EE040A30EE600A80ED030A90EDDC
:10AC0000020AF0EE080A30EE600A80ED020A59E00E
:10AC100076484068784988421CD17448006844F6F8
:10AC20007C41884216D1BEEE000A714880ED170AB9
:10AC30006E4890ED020AF0EE000A30EE600A80EDF8
:10AC4000020A90ED030AF2EE080A30EE600A80ED87
:10AC5000030A37E065484068684988420BD1634879
:10AC6000006844F67C41884205D1B7EE000A60488E
:10AC700080ED170A26E05D4840685F4988421CD194
:10AC80005A48006845F22211884216D19FED5C0AAD
:10AC9000574880ED170A554890ED020AF0EE000A79
:10ACA00030EE600A80ED020A90ED030AF2EE080A27
:10ACB00030EE600A80ED030A04E0B6EE000A4C486C
:10ACC00080ED170A4A48B0F844004AF2050188426C
:10ACD00017D146484068F52814D1444800684AF224
:10ACE000104188420ED19FED470A414880ED170A76
:10ACF0003E4890ED030AF1EE000A30EE600A80ED66
:10AD0000030A26E23948406840F26A41884213D17A
:10AD100036480068B0F5965F0ED19FED3A0A344888
:10AD200080ED170A314890ED030AF1EE000A30EE8B
:10AD3000600A80ED030A0CE22C484068E630E0B976
:10AD40002A48006849F25011884216D19FED2E0A18
:10AD5000274880ED170A254890ED020AF1EE080A0F
:10AD600030EE600A80ED020A90ED030AF3EE020A6B
:10AD700030EE600A80ED030AEBE11C484068E630E3
:10AD8000E0B91A48006842F6E061884216D1B7EE91
:10AD9000080A174880ED170A144890ED020AD0ED12
:10ADA000050A30EE200A80ED020A90ED030AF1EE6A
:10ADB000040A30EE600A80ED030ACAE10B484068DD
:10ADC00040F26A41884226D10848006847F6E011FF
:10ADD000884220D19FED0B0A054880ED170A0348F1
:10ADE00090ED030AF0EE000A10E00000D4320120DA
:10ADF0005439022000000000BAF5FFFF6AFAFFFF95
:10AE0000CDCC4CBF3333B33FC3F5C83F30EE600AFF
:10AE100080ED030A9DE1FE48406840F26A418842A5
:10AE200014D1FB48006847F2305188420ED11FED23
:10AE30000B0AF84880ED170AF54890ED030AF0EE8A
:10AE4000000A30EE600A80ED030A82E1F0484068B3
:10AE500040F27E41884214D1ED48006845F6101159
:10AE600088420ED1B0EE000AEA4880ED170AE848A1
:10AE700090ED030AF0EE000A30EE600A80ED030A5E
:10AE800067E1E348406840F27E41884214D1E048DF
:10AE9000006845F2604188420ED19FEDDF0ADD482F
:10AEA00080ED170ADA4890ED030AF2EE040A30EE5C
:10AEB000600A80ED030A4CE1D5484068B0F5877F11
:10AEC00014D1D348006844F2A01188420ED1B7EEE5
:10AED000080AD04880ED170ACD4890ED030AF1EE3C
:10AEE000080A30EE600A80ED030A32E1C848406883
:10AEF000B0F58C6F14D1C648006841F27071884279
:10AF00000ED1B7EE080AC34880ED170AC04890ED8D
:10AF1000030AF1EE000A30EE600A80ED030A18E140
:10AF2000BB48406843F22C31884214D1B8480068CD
:10AF30004BF24C3188420ED1B0EE000AB54880ED9C
:10AF4000170AB34890ED030AF1EE080A30EE200A22
:10AF500080ED030AFDE0AE48406843F22C318842A0
:10AF600013D1AB480068B0F52F4F0ED1B7EE000AF1
:10AF7000A84880ED170AA64890ED030AF2EE040AED
:10AF800030EE600A80ED030AE3E0A148406843F236
:10AF90002C31884214D19E48006849F60E418842FF
:10AFA0000ED1B7EE080A9B4880ED170A984890ED3D
:10AFB000030AF1EE080A30EE200A80ED030AC8E029
:10AFC0009348406843F22C31884214D1904800687D
:10AFD00049F2907188420ED1B7EE000A8D4880ED9B
:10AFE000170A8B4890ED030AF3EE020A30EE600A6E
:10AFF00080ED030AADE0864840681E30E0B9844821
:10B0000000684BF68031884216D1B0EE000A8148C4
:10B0100080ED170A7E4890ED020AF1EE000A30EE4C
:10B02000600A80ED020A90ED030AF2EE040A30EEA7
:10B03000200A80ED030A8CE075484068E630E0B9EC
:10B04000734800684CF64061884216D1B0EE080A99
:10B05000704880ED170A6E4890ED020AF2EE000A81
:10B0600030EE600A80ED020A90ED030AF2EE000A6B
:10B0700030EE600A80ED030A6BE06548406840F2FC
:10B08000CA3188421CD1624800684CF6406188424F
:10B0900016D19FED620A5F4880ED170A5C4890ED7B
:10B0A000020AF1EE080A30EE600A80ED020A90ED25
:10B0B000030AF1EE080A30EE600A80ED030A48E068
:10B0C00053484068564988421CD15148006844F6AC
:10B0D0007C41884216D1B0EE000A4E4880ED170A36
:10B0E0004B4890ED020AF1EE080A30EE600A80ED5E
:10B0F000020A90ED030AF2EE080A30EE600A80EDD3
:10B10000030A26E042484068454988421CD140482D
:10B11000006845F22211884216D1B7EE080A3D4870
:10B1200080ED170A3A4890ED020AF1EE080A30EE77
:10B13000600A80ED020A90ED030AF2EE040A30EE96
:10B14000600A80ED030A04E01FEDD10A314880ED6A
:10B15000170A3048B0F844004AF20601884220D16C
:10B160002B484068B0F5877F1CD12948006844F21D
:10B17000A011884216D19FED2B0A264880ED170AB0
:10B18000234890ED030AF1EE000A30EE600A80EDEC
:10B19000030A90ED020AF1EE080A30EE600A80ED33
:10B1A000020AE2E11A48406840F26A4188420ED140
:10B1B00017480068B0F5965F09D1154890ED030A6D
:10B1C000F2EE040A30EE600A80ED030ACDE1104889
:10B1D0004068E63040BB0E48006849F25011884292
:10B1E00023D1B6EE000A0B4880ED170A084890ED0F
:10B1F000020AF7EE000A30EE600A80ED020A90EDD6
:10B20000030AF3EE000A30EE600A80ED030AACE1B7
:10B21000D4320120543902206666E63F9A9959409B
:10B22000BAF5FFFF6666663FFFE7FA484068E6301A
:10B2300058B9F848006842F6E061884205D1B6EE98
:10B24000000AF54880ED170A8FE1F2484068B0F532
:10B25000877F14D1EF4800684AF6705188420ED1BA
:10B26000EC4890ED030AF1EE000A30EE600A80ED42
:10B27000030AB6EE000AE84880ED170A75E1E548D2
:10B280004068F52814D1E34800684AF2104188422A
:10B290000ED19FEDE20AE04880ED170ADD4890EDFF
:10B2A000030AF1EE000A30EE600A80ED030A5CE169
:10B2B000D848406840F27E4188420FD1D5480068A6
:10B2C00045F26041884209D1D24890ED030AF2EE7E
:10B2D000020A30EE600A80ED030A46E1CD4840687C
:10B2E00040F27E41884214D1CA48006845F61011E8
:10B2F00088420ED19FEDC90AC74880ED170AC5489C
:10B3000090ED030AF1EE000A30EE600A80ED030AC8
:10B310002BE1C048406840F26A41884214D1BD48E0
:10B32000006847F2305188420ED19FEDBD0ABA48FD
:10B3300080ED170AB74890ED030AF2EE000A30EEEE
:10B34000600A80ED030A10E1B248406843F22C31F4
:10B35000884214D1AF4800684BF24C3188420ED17C
:10B360009FEDB00AAC4880ED170AAA4890ED030A99
:10B37000F2EE020A30EE200A80ED030AF5E0A5485D
:10B38000406843F22C31884213D1A2480068B0F5DE
:10B390002F4F0ED19FEDA40A9F4880ED170A9D48BC
:10B3A00090ED030AF2EE000A30EE600A80ED030A27
:10B3B000DBE09848406843F22C31884214D195482C
:10B3C000006849F60E4188420ED19FED960A9248D8
:10B3D00080ED170A8F4890ED030AF2EE040A30EE72
:10B3E000200A80ED030AC0E08A48406843F22C310D
:10B3F000884214D18748006849F2907188420ED182
:10B40000B6EE000A844880ED170A824890ED030AE0
:10B41000F2EE0C0A30EE600A80ED030AA5E07D48EA
:10B4200040681E30A0B97B4800684BF680318842E6
:10B430000ED11FED870A784880ED170A754890ED08
:10B44000030AF1EE000A30EE200A80ED030A8CE0D8
:10B4500070484068E630E0B96E4800684CF64061DC
:10B46000884216D19FED710A6B4880ED170A694832
:10B4700090ED030AF1EE080A30EE600A80ED030A4F
:10B4800090ED020AF1EE000A30EE600A80ED020A49
:10B490006BE06048406840F2CA3188421CD15D4888
:10B4A00000684CF64061884216D1B0EE000A5A4856
:10B4B00080ED170A574890ED030AF1EE080A30EEC6
:10B4C000600A80ED030A90ED020AF1EE000A30EE08
:10B4D000600A80ED020A48E04E48406854498842BC
:10B4E0001CD14C48006844F67C41884216D1B6EE27
:10B4F000000A494880ED170A464890ED020AF0EE2E
:10B50000000A30EE600A80ED020A90ED030AF1EEC7
:10B51000080A30EE600A80ED030A26E03D484068E4
:10B52000434988421CD13B48006845F222118842B9
:10B5300016D1BEEE000A384880ED170A354890ED66
:10B54000030AF2EE000A30EE600A80ED030A90ED85
:10B55000020AF0EE000A30EE600A80ED020A04E012
:10B56000B6EE000A2C4880ED170A2B48B0F84400CC
:10B570004AF20701884210D12648406840F27E41D5
:10B5800088420BD12348006845F26041884205D1CA
:10B59000B7EE080A204880ED170A01E21D4840680E
:10B5A00040F26A41884213D11A480068B0F5965FAC
:10B5B0000ED19FED1E0A184880ED170A154890ED30
:10B5C000030AF1EE000A30EE600A80ED030AE7E1BB
:10B5D00010484068E630E0B90E48006849F2501162
:10B5E000884227D1B6EE000A0B4880ED170A0948B9
:10B5F00090ED020AF0EE000A30EE600A80ED020AD9
:10B6000090ED030AF3EE000A30EE600A80ED030AC3
:10B61000C6E10FE0D432012054390220CDCC4C3F9A
:10B62000CDCCCC3ECDCC4CBE000000009A99D93F89
:10B63000BAF5FFFFFE484068E630E0B9FC48006814
:10B6400042F6E061884216D1B6EE000AF94880ED74
:10B65000170AF74890ED020AD0ED050A30EE200AED
:10B6600080ED020A90ED030AF0EE000A30EE600A67
:10B6700080ED030A94E1EE48406840F67A01884282
:10B680000BD1EB48006845F26041884205D1B7EE26
:10B69000080AE84880ED170A82E1E548406840F66C
:10B6A0007A0188420BD1E248006847F23051884263
:10B6B00005D1B7EE080ADF4880ED170A70E1DC48D3
:10B6C000406840F26A41884214D1D948006847F284
:10B6D000305188420ED1B7EE000AD64880ED170AE5
:10B6E000D34890ED030AF1EE000A30EE600A80EDD7
:10B6F000030A55E1CE48406840F2A55188420BD17B
:10B70000CB4800684AF21041884205D1B7EE080ADA
:10B71000C84880ED170A43E1C5484068B0F58C6F12
:10B7200014D1C348006841F2707188420ED1B7EE5F
:10B73000080AC04880ED170ABD4890ED030AF2EEF2
:10B74000000A30EE600A80ED030A29E1B84840683B
:10B7500043F22C31884214D1B54800684BF24C3189
:10B7600088420ED19FEDB40AB24880ED170AB04866
:10B7700090ED030AF1EE000A30EE200A80ED030A94
:10B780000EE1AB48406843F22C31884213D1A848FF
:10B790000068B0F52F4F0ED19FEDA80AA54880EDA7
:10B7A000170AA34890ED030AF1EE080A30EE600A8A
:10B7B00080ED030AF4E09E48406842F6E06188426A
:10B7C0000AD19B480068B0F52F4F05D1B7EE080AA3
:10B7D000984880ED170AE3E09548406843F22C3121
:10B7E000884214D19248006849F60E4188420ED131
:10B7F0001FED730A8F4880ED170A8D4890ED030AFC
:10B80000F2EE020A30EE200A80ED030AC8E0884812
:10B81000406843F22C31884214D18548006849F2CF
:10B82000907188420ED1B7EE000A824880ED170A67
:10B830007F4890ED030AF2EE0C0A30EE600A80EDCC
:10B84000030AADE07A4840681E30E0B978480068E5
:10B850004BF68031884216D1B7EE080A754880ED64
:10B86000170A734890ED020AF1EE000A30EE600A02
:10B8700080ED020A90ED030AF3EE000A30EE200A92
:10B8800080ED030A8CE06A484068E630E0B9684819
:10B8900000684CF64061884216D19FED690A654800
:10B8A00080ED170A624890ED030AF1EE080A30EEC7
:10B8B000600A80ED030A90ED020AF1EE000A30EE14
:10B8C000600A80ED020A6BE05948406840F2CA31D4
:10B8D00088421CD1564800684CF64061884216D117
:10B8E000B0EE040A534880ED170A514890ED020A61
:10B8F000F0EE080A30EE600A80ED020A90ED030ACD
:10B90000F1EE000A30EE600A80ED030A48E0484894
:10B9100040684C4988421CD14548006844F67C4147
:10B92000884216D19FED480A424880ED170A4048E8
:10B9300090ED020AF0EE000A30EE600A80ED020A95
:10B9400090ED030AF1EE000A30EE600A80ED030A82
:10B9500026E0374840683B4988421CD1344800689B
:10B9600045F22211884216D19FED380A314880ED08
:10B97000170A2F4890ED020AF1EE000A30EE600A35
:10B9800080ED020A90ED030AF2EE040A30EE600A3E
:10B9900080ED030A04E09FED2E0A264880ED170A89
:10B9A0002448B0F844004AF20801884213D12048E4
:10B9B000406840F26A4188420ED11D480068B0F5E7
:10B9C000965F09D11A4890ED030AF0EE000A30EEB6
:10B9D000600A80ED030A83E115484068B0F58C6F7A
:10B9E0000FD11348006841F27071884209D11048A4
:10B9F00090ED030AF0EE000A30EE600A80ED030AD3
:10BA00006EE10B484068E63078BB0948006849F2AF
:10BA1000501188422AD1B7EE000A064880ED170A75
:10BA2000034890ED020AF1EE000A30EE600A11E0E0
:10BA3000D4320120543902206666A63F9A9999BEF5
:10BA400033331340BAF5FFFF9A99993F6666663F14
:10BA5000CDCCAC3F80ED020A90ED030AF3EE000A74
:10BA600030EE600A80ED030A3AE1FFE7F7484068EC
:10BA7000E630E0B9F548006842F6E061884216D148
:10BA8000B6EE000AF24880ED170AF04890ED020A7F
:10BA9000D0ED050A30EE200A80ED020A90ED030A8F
:10BAA000F0EE000A30EE600A80ED030A18E1E74884
:10BAB000406843F22C31884214D1E44800684BF2CC
:10BAC0004C3188420ED1B7EE000AE14880ED170AEA
:10BAD000DE4890ED030AF1EE000A30EE200A80ED18
:10BAE000030AFDE0D948406843F22C31884213D163
:10BAF000D6480068B0F52F4F0ED1B6EE000AD448F4
:10BB000080ED170AD14890ED030AF2EE000A30EEFC
:10BB1000600A80ED030AE3E0CC48406843F22C3130
:10BB2000884214D1C948006849F60E4188420ED1B6
:10BB3000B7EE080AC64880ED170AC44890ED030A1C
:10BB4000F2EE000A30EE200A80ED030AC8E0BF489A
:10BB5000406843F22C31884214D1BC48006849F255
:10BB6000907188420ED19FEDBB0AB94880ED170A4B
:10BB7000B64890ED030AF2EE0C0A30EE600A80ED52
:10BB8000030AADE0B14840681E30E0B9AF48006834
:10BB90004BF68031884216D1B7EE080AAC4880EDEA
:10BBA000170AAA4890ED020AD0ED050A30EE200AE5
:10BBB00080ED020A90ED030AF2EE000A30EE200A50
:10BBC00080ED030A8CE0A1484068E630E0B99F4868
:10BBD00000684CF64061884216D19FED9F0A9C4850
:10BBE00080ED170A994890ED020AF2EE000A30EE55
:10BBF000600A80ED020A90ED030AF2EE000A30EED0
:10BC0000600A80ED030A6BE09048406840F2CA3158
:10BC100088421CD18D4800684CF64061884216D19C
:10BC2000B0EE040A8A4880ED170A884890ED020AAF
:10BC3000F2EE000A30EE600A80ED020A90ED030A8F
:10BC4000F1EE080A30EE600A80ED030A48E07F4812
:10BC50004068824988421CD17C48006844F67C4197
:10BC6000884216D19FED7E0A794880ED170A774801
:10BC700090ED020AF1EE000A30EE600A80ED020A51
:10BC800090ED030AF1EE080A30EE600A80ED030A37
:10BC900026E06E484068714988421CD16B480068B4
:10BCA00045F22211884216D1B6EE000A684880EDAE
:10BCB000170A664890ED020AF2EE000A30EE600ABA
:10BCC00080ED020A90ED030AF2EE040A30EE600AFB
:10BCD00080ED030A04E0B7EE000A5D4880ED170A24
:10BCE0005B48B0F844004AF20901884219D157482C
:10BCF000406840F27E41884214D15448006845F2C1
:10BD0000604188420ED1514890ED030AF0EE000ADE
:10BD100030EE600A80ED030A9FED520A4C4880ED38
:10BD2000170AA0E149484068E630E0B94748006892
:10BD300049F25011884216D1BFEE000A444880ED06
:10BD4000170A424890ED020AF1EE000A30EE600A4E
:10BD500080ED020A90ED030AF2EE080A30EE600A66
:10BD600080ED030A7FE139484068E63058B937482A
:10BD7000006842F6E061884205D1BFEE080A344807
:10BD800080ED170A6FE13148406840F2CA318842BD
:10BD90000BD12E48006849F25011884205D19FED21
:10BDA000320A2B4880ED170A5DE12848406840F2CE
:10BDB000CA3188420BD12548006842F6E0618842CA
:10BDC00005D19FED240A224880ED170A4BE11F4858
:10BDD0004068B0F5877F0BD11C48006844F2A01181
:10BDE000884205D1B6EE000A194880ED170A3AE1FB
:10BDF0001648406840F26A41884214D113480068EE
:10BE000047F2305188420ED1104890ED030AF0EE0F
:10BE1000000A30EE600A80ED030A9FED140A0C4818
:10BE200080ED170A1FE10948406840F26A418842E4
:10BE300020D10648006847F6E01188421AD19FEDEC
:10BE40000C0A034880ED170A0DE10000D4320120EE
:10BE50005439022000000000CDCC0C40BAF5FFFFA1
:10BE60003333333F9A9919BFCDCCCCBD333333BF75
:10BE7000CDCCCCBEF848406843F22C31884214D176
:10BE8000F548006849F2907188420ED1BFEE000A71
:10BE9000F24880ED170AF04890ED030AF3EE020A2B
:10BEA00030EE600A80ED030ADDE0EB48406843F2C3
:10BEB0002C31884214D1E84800684BF24C3188425A
:10BEC0000ED19FEDE70AE54880ED170AE24890EDB4
:10BED000030AF2EE040A30EE200A80ED030AC2E003
:10BEE000DD48406843F22C3188420AD1DA480068C4
:10BEF000B0F52F4F05D1B8EE080AD84880ED170AE3
:10BF0000B1E0D548406843F22C31884214D1D24880
:10BF1000006849F60E4188420ED1BFEE000ACF48B4
:10BF200080ED170ACC4890ED030AF2EE080A30EED5
:10BF3000200A80ED030A96E0C74840681E30A0B989
:10BF4000C54800684BF6803188420ED11FED3F0A8C
:10BF5000C24880ED170AC04890ED030AF2EE040AC9
:10BF600030EE200A80ED030A7DE0BB484068E630F1
:10BF7000A0B9B94800684CF6406188420ED19FEDE7
:10BF8000B90AB64880ED170AB34890ED020AF1EEFF
:10BF9000000A30EE600A80ED020A64E0AE484068B4
:10BFA00040F2CA31884214D1AB4800684CF6406177
:10BFB00088420ED19FEDAC0AA84880ED170AA6482A
:10BFC00090ED020AF0EE000A30EE600A80ED020AFF
:10BFD00049E0A1484068A549884214D19E480068BC
:10BFE00044F67C4188420ED19FEDA10A9B4880ED2A
:10BFF000170A994890ED020AF0EE000A30EE600A46
:10C0000080ED020A2FE094484068984988421CD18C
:10C010009148006845F22211884216D19FED940A9A
:10C020008E4880ED170A8C4890ED020AF0EE000A67
:10C0300030EE600A80ED020A90ED030AF0EE000A8D
:10C0400030EE600A80ED030A0DE0834890ED030AAC
:10C05000F0EE000A30EE600A80ED030A1FED7F0A61
:10C060007E4880ED170A7D48B0F844004AF210017E
:10C07000884213D17848406840F26A4188420ED124
:10C0800075480068B0F5965F09D1734890ED030AD2
:10C09000F1EE000A30EE600A80ED030A2BE26E48F2
:10C0A0004068E630E0B96C48006849F250118842B7
:10C0B00016D16A4890ED180A80ED170A664890ED8F
:10C0C000020AF1EE000A30EE600A80ED020A90EDFD
:10C0D000030AF2EE080A30EE600A80ED030A0AE273
:10C0E0005D484068E630E0B95B48006842F6E061D0
:10C0F000884216D1BEEE000A584880ED170A56480D
:10C1000090ED020AD0ED050A30EE200A80ED020A19
:10C1100090ED030AF0EE000A30EE600A80ED030AAB
:10C12000E9E14D48406840F2CA3188420BD14A48A3
:10C13000006842F6E061884205D19FED4D0A47480C
:10C1400080ED170AD7E144484068B0F58C6F14D1F0
:10C150004148006841F2707188420ED13E4890ED2E
:10C16000030AF1EE000A30EE600A80ED030A1FEDCB
:10C17000C30A3A4880ED170ABDE137484068B0F578
:10C18000877F0FD13448006844F2A011884209D15A
:10C19000314890ED030AF0EE080A30EE600A80EDB7
:10C1A000030AA8E12C48406840F27E41884214D13D
:10C1B0002948006845F2604188420ED1264890ED3A
:10C1C000030AF1EE000A30EE600A80ED030A9FEDEB
:10C1D000290A224880ED170A8DE11F48406840F681
:10C1E0007A0188420AD11C480068B0F5965F05D1F3
:10C1F000BFEE000A194880ED170A7CE11648406836
:10C2000040F67A0188420BD11348006845F61011B8
:10C21000884205D1BEEE000A104880ED170A6AE197
:10C220000D48406840F27E41884225D10A480068A6
:10C2300045F6101188421FD1074890ED030AF0EE31
:10C24000000A30EE600A80ED030ABFEE000A0348E0
:10C2500080ED170A4FE10000D4320120543902204A
:10C260003333B3BFCDCC4CBECDCC4C3EBAF5FFFF83
:10C270006666A6BFCDCC4CBFF948406840F26A4123
:10C2800088420FD1F648006847F23051884209D100
:10C29000F34890ED030AF1EE000A30EE600A80EDFB
:10C2A000030A28E1EE484068F5280FD1EC48006801
:10C2B0004AF21041884209D1E94890ED030AF1EEB3
:10C2C000040A30EE600A80ED030A14E1E448406895
:10C2D000B0F5B96F0BD1E24800684AF67051884258
:10C2E00005D1BEEE080ADF4880ED170A03E1DC48FD
:10C2F000406843F22C31884213D1D9480068B0F528
:10C300002F4F0ED1B8EE000AD64880ED170AD44858
:10C3100090ED030AF0EE080A30EE600A80ED030AA1
:10C32000E9E0CF48406843F22C3188421AD1CC482A
:10C33000006849F60E41884205D0C94800684BF2B2
:10C340004C3188420ED19FEDC80AC64880ED170ACD
:10C35000C34890ED030AF2EE080A30EE200A80EDA1
:10C36000030AC8E0BE48406843F22C31884214D129
:10C37000BB48006849F2907188420ED11FED430A14
:10C38000B84880ED170AB64890ED030AF2EE080AA5
:10C3900030EE600A80ED030AADE0B14840681E301F
:10C3A000E0B9AF4800684BF68031884216D19FED66
:10C3B000AF0AAC4880ED170AA94890ED020AF1EEE9
:10C3C000000A30EE600A80ED020A90ED030AF3EEF7
:10C3D000000A30EE200A80ED030A8CE0A048406895
:10C3E000E630E0B99E4800684CF64061884216D1BC
:10C3F0001FED630A9B4880ED170A994890ED020AE9
:10C40000F1EE080A30EE600A80ED020A90ED030AB0
:10C41000F1EE000A30EE600A80ED030A6BE090480E
:10C42000406840F2CA3188421CD18D4800684CF601
:10C430004061884216D1B6EE000A8A4880ED170A9C
:10C44000874890ED020AF1EE040A30EE600A80EDB2
:10C45000020A90ED030AF0EE000A30EE600A80ED69
:10C46000030A48E07E484068814988421CD17C48E4
:10C47000006844F67C41884216D1BFEE080A79482C
:10C4800080ED170A764890ED020AF1EE000A30EED0
:10C49000600A80ED020A90ED030AF1EE000A30EE28
:10C4A000600A80ED030A26E06D48406870498842C2
:10C4B0001CD16B48006845F22211884216D1BFEEAC
:10C4C000080A684880ED170A654890ED020AF1EE07
:10C4D000080A30EE600A80ED020A90ED030AF1EEE0
:10C4E000000A30EE600A80ED030A04E01FED9F0AA7
:10C4F0005C4880ED170A5B48B0F844004AF211012D
:10C50000884219D15648406840F27E41884214D191
:10C510005348006845F6101188420ED1504890EDFE
:10C52000020AF1EE0C0A30EE200A80ED020A9FEDBD
:10C53000510A4C4880ED170ADAE149484068E63074
:10C54000E0B94748006849F25011884216D1BFEE61
:10C55000000A444880ED170A414890ED020AD0EDE8
:10C56000050A30EE200A80ED020A90ED030AF1EE92
:10C57000080A30EE600A80ED030AB9E138484068E5
:10C58000E630E0B93648006842F6E061884216D1EC
:10C590009FED390A334880ED170A314890ED020AC1
:10C5A000D0ED050A30EE200A80ED020A90ED030A74
:10C5B000F1EE000A30EE200A80ED030A98E12848E7
:10C5C000406840F2CA3188420BD12548006842F6E3
:10C5D000E061884205D19FED290A224880ED170AC3
:10C5E00086E11F48406840F27E41884214D11C48D1
:10C5F000006845F2604188420ED1194890ED030A67
:10C60000F0EE000A30EE600A80ED030A9FED190A91
:10C61000144880ED170A6BE11148406840F2BE51A2
:10C6200088420BD10E48006844F2A011884205D11F
:10C630001FEDF40A0B4880ED170A59E108484068DD
:10C6400040F67A0188421BD105480068B0F5965F34
:10C6500016D1BEEE000A034880ED170A48E100003B
:10C66000D432012054390220CDCCCCBF00000000D0
:10C67000BAF5FFFFCDCCCCBD9A9919BF9A99993ED6
:10C68000CB48406840F26A41884213D1C8480068EC
:10C69000B0F5965F0ED1C64890ED030AF1EE000AA0
:10C6A00030EE600A80ED030A9FEDC20AC24880EDB9
:10C6B000170A1DE1BE484068B0F58C6F0FD1BC4829
:10C6C000006841F27071884209D1B94890ED020AC0
:10C6D000F1EE000A30EE600A80ED020A08E1B4488B
:10C6E000406843F22C31884214D1B14800684BF2C3
:10C6F0004C3188420ED19FEDB10AAF4880ED170A48
:10C70000AB4890ED030AF1EE080A30EE200A80ED06
:10C71000030AEDE0A648406843F22C31884213D169
:10C72000A3480068B0F52F4F0ED19FEDA50AA2488F
:10C7300080ED170A9E4890ED030AF1EE000A30EEF4
:10C74000200A80ED030AD3E09948406843F22C3177
:10C75000884214D19648006849F60E4188420ED1AD
:10C760001FED3E0A944880ED170A914890ED030AA8
:10C77000F2EE080A30EE200A80ED030AB8E08C4899
:10C78000406843F22C31884214D18948006849F24C
:10C79000907188420ED1BFEE080A874880ED170AD3
:10C7A000834890ED030AF2EE000A30EE600A80ED55
:10C7B000030A9DE07E4840681E30E0B97C4800686E
:10C7C0004BF68031884216D1B6EE000A7A4880EDE9
:10C7D000170A774890ED020AF1EE000A30EE200ABF
:10C7E00080ED020A90ED030AF3EE020A30EE200A11
:10C7F00080ED030A7CE06E484068E630E0B96C48A2
:10C8000000684CF64061884216D19FED6E0A6A4876
:10C8100080ED170A664890ED020AF0EE000A30EE4D
:10C82000600A80ED020A90ED030AF0EE000A30EE95
:10C83000200A80ED030A5BE05D48406840F2CA319F
:10C84000884214D15A4800684CF6406188420ED1A3
:10C850009FED5C0A584880ED170A554890ED030A91
:10C86000F1EE000A30EE200A80ED030A40E0504865
:10C8700040685549884214D14D48006844F67C41CF
:10C8800088420ED11FED830A4B4880ED170A4848B5
:10C8900090ED030AF0EE000A30EE600A80ED030A24
:10C8A00026E043484068484988421CD14048006817
:10C8B00045F22211884216D11FED940A3E4880EDC0
:10C8C000170A3B4890ED030AF0EE000A30EE600ACA
:10C8D00080ED030A90ED020AF0EE000A30EE600AE5
:10C8E00080ED020A04E01FED9D0A334880ED170A2F
:10C8F000314890ED170ADDED0E0A30EE200A10EEF9
:10C90000101A08460AF096FF41EC190B9FED2F0B09
:10C9100053EC102B0AF06EFA41EC180B0AF07CF97C
:10C92000234988619DED0E0A2A4880ED000A0B9884
:10C9300081F82400284801680068401C264A1060DD
:10C94000142931DD0020114608600E980AF072FFAC
:10C9500041EC180B164890ED030A10EE101A084629
:10C960000AF068FF41EC190B114890ED020A10EE35
:10C97000101A08460AF05EFF41EC1A0B0C4890F8BA
:10C980002500099A0B99CDE9061208908DED048BCC
:10C990008DED029B8DED00AB1048036810481149E6
:10C9A0000268012002F09AF911B0BDEC068B30BD8F
:10C9B000D43201209A9999BE54390220CDCC4CBE74
:10C9C0006666E6BFCDCCCC3FBAF5FFFF666666660D
:10C9D00066A64C407C190020881900209019002080
:10C9E0008C190020D87E010830B52DED068B91B052
:10C9F00004460D469FED590A8DED100A9FED570A2A
:10CA00008DED0F0A9FED550A8DED0E0A00200D9059
:10CA10000C900B900A90099009A80AA90BAA0CABDC
:10CA2000CDE90432CDE906100DA80EA90FAA10AB6E
:10CA3000CDE90032CDE90210494B4A4A4AA12046CD
:10CA4000F3F774FE0B9801287ED19DED100A4F4834
:10CA500080ED000A9DED0F0A4D4880ED000A414827
:10CA600000684C4908609DED100ADFED4B0A30EE7E
:10CA7000600AB1EE400A10EE101A08460AF0DAFE1B
:10CA800041EC190B9FED450B53EC102B0AF0DCFB2E
:10CA900041EC180B0AF0C0F83E49C8609DED0F0A42
:10CAA000DFED400A30EE600AB1EE400A10EE101AD7
:10CAB00008460AF0BFFE41EC190B9FED380B53EC12
:10CAC000102B0AF0C1FB41EC180B0AF0A5F8314914
:10CAD00088609DED0E0ADFED210A30EE200A08463F
:10CAE00080ED060A0B9881F824002F480168006841
:10CAF000401C2D4A106032292BDD002011460860B1
:10CB00000E980AF097FE41EC180B224890ED030AAC
:10CB100010EE101A08460AF08DFE41EC190B1D4864
:10CB200090ED020A10EE101A08460AF083FE41EC5E
:10CB30001A0B0B9806908DED048B8DED029B8DEDFD
:10CB400000AB0848194900E003E00268012002F048
:10CB5000C5F811B0BDEC068B30BD00000000000030
:10CB60009C190020981900203C25645859256440E0
:10CB70002825667825662925664025784025784051
:10CB800025642D25642D25643E00000080190020B9
:10CB900084190020003301200000C84333333333AD
:10CBA0003333CB3F00009643941900208C7E01085C
:10CBB00010B5F8F773F9064807F074FE04491E39FA
:10CBC00091F8240004F00AFE024807F0ABFA10BD09
:10CBD000723902205C3A022008B5016800919DED8F
:10CBE000000A08BD29B1064A12680243044B1A60C4
:10CBF00004E0034A12688243014B1A607047000048
:10CC00003038024029B1064A12680243044B1A60C8
:10CC100004E0034A12688243014B1A607047000027
:10CC20004038024029B1064A12680243044B1A6098
:10CC300004E0034A12688243014B1A607047000007
:10CC400044380240F0B500210022002402250026CD
:10CC50000223324F3F6807F00C0121B1042905D0AF
:10CC6000082937D105E02E4F076036E02D4F0760C9
:10CC700033E02A4F3F1F3F68C7F38056274F3F1FBF
:10CC80003F6807F03F036EB1264FB7FBF3F7DFF8BD
:10CC90008CC0ACF1040CDCF800C0CCF3881C07FBA2
:10CCA0000CF40CE01E4FB7FBF3F7DFF870C0ACF1EB
:10CCB000040CDCF800C0CCF3881C07FB0CF4174F05
:10CCC0003F1F3F68C7F301477F1C7D00B4FBF5F7AA
:10CCD000076002E0124F076000BF00BF0F4F3F68C0
:10CCE00007F0F0010909104F7A5C0768D7404760E8
:10CCF0000A4F3F6807F4E051890A0B4F7A5C476896
:10CD0000D7408760054F3F6807F46041490B064FE5
:10CD10007A5C4768D740C760F0BD00000838024021
:10CD20000024F40000127A000406002030B5034607
:10CD30000020054C234404E033F8015B0D54401CF3
:10CD40005B1C9042F8DB30BD00F8070870B5054663
:10CD50000024012D04D0022D05D0032D09D105E0BA
:10CD600000F092FF08E000F09FFF05E000F0AEFF4A
:10CD700002E000F089FF00BF00BF0220F8F7FEFAD2
:10CD80004FF480713648F8F79EFB012802D144F039
:10CD9000010401E024F0010480213148F8F793FBFD
:10CDA000012802D144F0020401E024F002044021F1
:10CDB0002B48F8F788FB012802D144F0040401E075
:10CDC00024F0040420212648F8F77DFB012802D135
:10CDD00044F0080401E024F0080410212048F8F78A
:10CDE00072FB012802D144F0100401E024F0100489
:10CDF00008211B48F8F767FB012802D144F0200402
:10CE000001E024F0200404211548F8F75CFB012818
:10CE100002D144F0400401E024F040044FF400410A
:10CE20001048F8F750FB012802D144F0800401E0DB
:10CE300024F08004012D04D0022D05D0032D09D14A
:10CE400005E000F019FF08E000F026FF05E000F023
:10CE500033FF02E000F010FF00BF00BF204670BDAE
:10CE600000180240000C0240014600200246012941
:10CE70000DDB08290BDC481EC2B2154800681041C2
:10CE800000F0010008B1012070470020FCE71029E4
:10CE90000CDCA1F10900C2B20D484068104100F05D
:10CEA000010008B10120EFE70020EDE718290CDCB4
:10CEB000A1F11100C2B206488068104100F00100E3
:10CEC00008B10120E0E70020DEE700BFDCE700005A
:10CED000E42B0120F0B503460C461546002200263F
:10CEE000012B01D1174911E0022B01D116490DE0A8
:10CEF000032B01D1154909E0042B01D1144905E0A8
:10CF0000062B01D1134901E00020F0BD002213E0FF
:10CF1000B1F80008B1F80278B84200D10EE0761CF2
:10CF2000B1F80208085CA054B1F80208401CC0F334
:10CF30000900A1F80208521CAA42E9D300BF3046FA
:10CF4000E3E7000058020120600A01206812012076
:10CF5000701A01207822012010B500240DE004EBA6
:10CF60008400074A02EBC0010648F3F713FD10B92D
:10CF7000002005490855601CC4B2312CEFDB10BD00
:10CF8000DC3301206C960120148801200021012847
:10CF90000BDB082809DC421ED1B2114A12680123BA
:10CFA0008B401A430E4B1A6018E010280ADCA0F1DF
:10CFB0000902D1B20A4A536801228A401343084A3F
:10CFC00053600BE0182809DCA0F11102D1B2044A29
:10CFD000926801238B401A43014B9A60704700000E
:10CFE000F02B01200349D1F8A8108143014AC2F86F
:10CFF000A81070475439022010B52DED0C8B044653
:10D00000E07A602809D1207B602806D1607B602807
:10D0100003D10120484948611EE0E07A60280CD124
:10D02000207B402809D1607B602806D1E07B062860
:10D0300003D10220404948610EE0E07A60280BD11C
:10D04000207B402808D1607B602805D1E07B0F2839
:10D0500002D1032038494861E07A432868D1207B17
:10D060006C2865D1607B602862D1A07C0206607C60
:10D0700002EB0042207C02EB0022E07B104400EE39
:10D08000100AB8EEC00A10EE101A08460AF0D2FBD9
:10D0900041EC1D0B9FED290B53EC102B09F0AAFE60
:10D0A00041EC1C0B9FED270B53EC102B0AF0CCF836
:10D0B00041EC1B0B9FED250B53EC102B0AF0C4F831
:10D0C00041EC1A0B9FED230B53EC102B09F092FE51
:10D0D00041EC190B9FED210B53EC102B09F08AFE4C
:10D0E00041EC180B09F098FD13494860084690ED93
:10D0F000010A10EE101A08460AF09CFB41EC190BCD
:10D10000B0EE490AF0EE690A02F08EFCB0EE408AF9
:10D11000F0EE608A9FED130B53EC102B51EC180BC3
:10D120000AF056F804D29FED110A034880ED010A77
:10D13000BDEC0C8B10BD00004433012066666666B2
:10D140006655A5400C022B8716D9E63FCDCCCCCC3A
:10D15000CCCCF03F00000000000000408716D9CE84
:10D16000F753F13F000000000000244000000000E1
:10D1700010B50446E07A60280CD1207B602809D1E4
:10D18000607B602806D101205C4908705CA101F039
:10D19000A5FD26E0E07A602810D1207B40280DD143
:10D1A000607B60280AD1E07B062807D10220534922
:10D1B000087059A1012001F091FD12E0E07A602889
:10D1C0000FD1207B40280CD1607B602809D1E07B07
:10D1D0000F2806D103204949087055A1012001F00C
:10D1E0007DFDE07A432867D1207B632864D1607B92
:10D1F000602861D1E17B207C41EA0021607C41EA2A
:10D200000041A07C41EA00604F4908604F48007827
:10D2100030B100204D4908704B4800684C49086007
:10D22000494909684A4A1268881A002801DB014600
:10D2300000E0414264293FDD4548006842490968F1
:10D24000401A00EE100AB8EEC00ADFED420A60EEA6
:10D25000200A9FED411A80EE810A2848D0ED030A8A
:10D2600030EE200A80ED030A90ED030ADFED3B0A61
:10D27000B4EEE00AF1EE10FA08DD90ED030ADFEDFE
:10D28000350A30EE600A80ED030A11E01B4890ED8C
:10D29000030ADFED330AB4EEE00AF1EE10FA07D22A
:10D2A00090ED030ADFED2B0A30EE200A80ED030A31
:10D2B0002548006826490860207B01280ED1607B44
:10D2C00026280BD1617C207C41EA002125488183FE
:10D2D000E17CA07C41EA00212248C1832148808B67
:10D2E00020B14FF4006000F0BDFC06E01D48008B4B
:10D2F00018B94FF40060FFF775FE10BD88330120A8
:10D30000D0FDD7AAC9E8D6C3CBD9B6C8C4A3CABD75
:10D31000B3C9B9A60D0A0000D0FDD7AAC9E8D6C383
:10D32000CAB9C4DC3036B3C9B9A60D0A0000000082
:10D33000D0FDD7AAC9E8D6C3CAB9C4DC3046B3C940
:10D34000B9A60D0A0000000098050020D9050020AC
:10D35000DC0500200000B44300401C4A00003443B8
:10D36000000034C36833012010B52DED0C8BFE484E
:10D37000B0F8520000EE100AF8EE400A9FEDFB1ADA
:10D3800080EE810AFA48D0ED000A30EE200AB0EEB5
:10D39000408AF848807D012826D0F648807D022802
:10D3A00022D0F548007838B9EF4890ED0C0AB5EE78
:10D3B000C00AF1EE10FA17D1EE48807DA0B9EA4814
:10D3C00090F8240004280FD0E74890F824000328A0
:10D3D0000AD0E5484079052806D0E3484079062878
:10D3E00002D00020E4490870E24890ED030AE348C7
:10D3F000D0ED000A30EE600AE14880ED000A90EDC1
:10D40000000ADFEDE00AB4EEE00AF1EE10FA07DD03
:10D4100090ED000ADFEDD50A30EE600A80ED000ADB
:10D42000D74890ED000ADFEDD80AB4EEE00AF1EE3D
:10D4300010FA07D290ED000ADFEDCC0A30EE200A98
:10D4400080ED000AC84890ED0C0A10EE101A08464C
:10D450000AF0F0F941EC1B0BC94800680AF0EAF940
:10D4600041EC1D0BB0EE4D0AF0EE6D0A02F0DCFA55
:10D47000B0EE40CAF0EE60CA53EC1B2B51EC1C0B13
:10D480000AF0EEF841EC1A0BB0EE4A0AF0EE6A0A26
:10D4900002F0CAFAB0EE409AF0EE609A51EC190B25
:10D4A00009F0BAFBB9490860B248807D02280FD064
:10D4B000B048807D03280BD0AE48807D042807D07B
:10D4C000AC48807D052803D0AA48807D06282FD14E
:10D4D000AE4890ED000AF3EE0E0AB4EEE00AF1EE6B
:10D4E00010FA03DDAA4880ED008A21E0A74890EDFC
:10D4F000000AF0EE080AB4EEE00AF1EE10FA11DDCF
:10D50000B0EE482AA348D0ED001AB3EE0E1AF0EEA2
:10D51000080A9E4890ED000A06F0DCFD9C4880ED6C
:10D52000000A05E09B4890ED000A994880ED000A4A
:10D530009048807D09287DD2DFE800F0051016882C
:10D54000FEFDFCFBFA009FED940A8A4880ED010A7B
:10D5500090ED030A894880ED000A5BE29FED8F0A97
:10D56000844880ED010A55E2894800680AF062F9B2
:10D5700041EC1B0B9FED8A0B53EC102B09F064FE62
:10D5800041EC1A0B9FED880B53EC102B09F032FC89
:10D5900041EC190B09F040FB764948607B4890ED5F
:10D5A000000AF1EE040AB4EEE00AF1EE10FA2ED20F
:10D5B000084690ED030AFAEE040AB4EEE00AF1EE32
:10D5C00010FA24DD90ED030AF2EE040AB4EEE00A4C
:10D5D000F1EE10FA1BD20120FFF746FC04460220B0
:10D5E000FFF742FC044034B39FED6B0A614880EDC5
:10D5F000010A00205F4988759FED670A084680EDA3
:10D60000030A9FED650A5D4880ED000A1DE05F4852
:10D6100090ED000A6648D0ED000AB4EEE00AF1EEA3
:10D6200010FA12D20120FFF71FFC30B90220FFF7D9
:10D630001BFC01E0EDE108E038B19FED570A4D48D1
:10D6400080ED010A00204B498875E3E1504890EDD8
:10D65000000AB1EE400A10EE100A0AF0EBF841ECB5
:10D660001B0B9FED4F0B53EC102B09F0EDFD41EC24
:10D670001A0B9FED4D0B53EC102B09F0BBFB41EC4B
:10D68000190B09F0C9FA3B494860404890ED000A7F
:10D69000F1EE040AB4EEE00AF1EE10FA2ED20846DA
:10D6A00090ED030AFAEE040AB4EEE00AF1EE10FA85
:10D6B00024DD90ED030AF2EE040AB4EEE00AF1EE86
:10D6C00010FA1BD20120FFF7CFFB04460220FFF720
:10D6D000CBFB04408CB39FED300A264880ED010A55
:10D6E0000020244988759FED2C0A084680ED030A26
:10D6F0009FED290A214880ED000A21E0234890EDA2
:10D70000000A2B48D0ED000AB4EEE00AF1EE10FA60
:10D7100016D20120FFF7A8FB18B90220FFF7A4FBDF
:10D7200058B19FED1D0A134880ED010A002005E065
:10D730006EE167E1FFE092E003E001E00D498875EA
:10D7400068E1134800680AF075F841EC1B0B9FED87
:10D75000140B53EC102B09F077FD41EC1A0B9FEDE5
:10D76000120B53EC102B25E0543902200000B44377
:10D77000FC1E002088330120341F0020241F0020BD
:10D780002C1F002000003443000034C3281F002059
:10D79000081F0020001F0020000000000024F4C823
:10D7A000CDCCCCAC6A6E59410000000000000040B6
:10D7B000041F002009F01EFB41EC190B09F02CFAA4
:10D7C0009D4948609D4890ED000AF1EE040AB4EED0
:10D7D000E00AF1EE10FA2ED2084690ED030AFAEEB6
:10D7E000040AB4EEE00AF1EE10FA24DD90ED030A2B
:10D7F000F2EE040AB4EEE00AF1EE10FA1BD20120B8
:10D80000FFF732FB04460220FFF72EFB04402CB347
:10D810001FED1F0A884880ED010A0020864988759F
:10D820001FED230A084680ED030A1FED250A8448F0
:10D8300080ED000A12E0814890ED000A8148D0EDA9
:10D84000000AB4EEE00AF1EE10FA07D21FED2E0A3C
:10D85000794880ED010A002077498875DAE07A4836
:10D8600090ED000AB1EE400A10EE100A09F0E2FF56
:10D8700041EC190B1FED360B53EC102B09F0E4FCB7
:10D8800041EC1B0B1FED380B53EC102B09F0B2FAD7
:10D8900041EC1A0B09F0C0F967494860674890ED00
:10D8A000000AF2EE040AB4EEE00AF1EE10FA2ED20B
:10D8B000084690ED030AFAEE040AB4EEE00AF1EE2F
:10D8C00010FA24DD90ED030AF2EE040AB4EEE00A49
:10D8D000F1EE10FA1BD20120FFF7C6FA044602202F
:10D8E000FFF7C2FA04402CB31FED550A524880EDF1
:10D8F000010A0020504988751FED590A084680ED3D
:10D90000030A1FED5B0A4E4880ED000A12E04B4807
:10D9100090ED000A4B48D0ED000AB4EEE00AF1EEBB
:10D9200010FA07D21FED640A434880ED010A002077
:10D93000414988756EE04448006809F07BFF41EC7E
:10D940001B0B1FED690B53EC102B09F07DFC41EC18
:10D950001A0B1FED6B0B53EC102B09F04BFA41EC3B
:10D96000190B09F059F934494860344890ED000A20
:10D97000F2EE040AB4EEE00AF1EE10FA2ED20846F6
:10D9800090ED030AFAEE040AB4EEE00AF1EE10FAA2
:10D9900024DD90ED030AF2EE040AB4EEE00AF1EEA3
:10D9A00010FA1BD20120FFF75FFA04460220FFF7AE
:10D9B0005BFA04402CB31FED880A1F4880ED010A72
:10D9C00000201D4988751FED8C0A084680ED030A6A
:10D9D0001FED8F0A1A4880ED000A12E0174890EDFB
:10D9E000000A1848D0ED000AB4EEE00AF1EE10FA91
:10D9F00007D21FED970A104880ED010A00200E495A
:10DA0000887507E09FED110A0B4880ED010A01E0DF
:10DA100000E000BF00BF0E4890F8BD0048B10648C6
:10DA2000807D18B900200449886102E00120024984
:10DA30008861BDEC0C8B10BD88330120281F0020AD
:10DA4000241F0020041F0020081F0020005043490D
:10DA50005439022021B1028842F04002028004E0E1
:10DA600002884FF6BF731A400280704702460020BA
:10DA700013890B400BB1012000E0002070470146E4
:10DA8000888970478181704710B50022028802F4AE
:10DA900041520B884C8823438C882343CC882343F2
:10DAA0000C8923434C8923438C892343CC8923430A
:10DAB0001A430280838B4FF2FF74234083830B8AC7
:10DAC000038210BD7047000010B5124890F834076B
:10DAD00080B1012819D11048F7F774FE00B110BDCC
:10DAE00014210E48F3F70DF80D4A0EA10B48F2F77A
:10DAF0006DFC0BE00848F7F765FE00B1EFE70A4858
:10DB0000007908B1F5F7E4FE00E000BF00BF00BFF8
:10DB1000E5E70000F81B022048C901206C960120AF
:10DB200038CF0120257300005439022070B5044617
:10DB30000D46012D04D0022D05D0032D09D105E09D
:10DB400000F0CEF808E000F0DBF805E000F0E8F8BF
:10DB500002E000F0C5F800BF00BF04F0010028B1EA
:10DB60004FF480513C48F7F7B9FC04E04FF4805182
:10DB70003948F7F7B1FC04F0020028B14FF4005126
:10DB80003548F7F7ABFC04E04FF400513248F7F7A3
:10DB9000A3FC04F0040028B14FF480412E48F7F7AD
:10DBA0009DFC04E04FF480412B48F7F795FC04F00E
:10DBB000080028B14FF400412748F7F78FFC04E034
:10DBC0004FF400412448F7F787FC04F0100020B11F
:10DBD00001212248F7F782FC03E001211F48F7F7F3
:10DBE0007BFC04F0200020B102211C48F7F776FCF2
:10DBF00003E002211948F7F76FFC04F0400020B160
:10DC000080211748F7F76AFC03E080211448F7F7F2
:10DC100063FC04F0800028B14FF480711048F7F7DE
:10DC20005DFC04E04FF480710D48F7F755FC012DC1
:10DC300004D0022D05D0032D09D105E000F058F8DD
:10DC400008E000F065F805E000F074F802E000F08C
:10DC50004FF800BF00BF70BD001402400018024022
:10DC6000001002400349D1F8A8100143014AC2F84C
:10DC7000A81070475439022010B502210148F7F767
:10DC80002DFC10BD0010024010B502210148F7F72D
:10DC900023FC10BD0010024010B501210148F7F728
:10DCA0001DFC10BD0010024010B501210148F7F71E
:10DCB00013FC10BD0010024010B54FF40071024873
:10DCC000F7F70CFC10BD00000004024010B54FF443
:10DCD00000710248F7F700FC10BD0000000402408C
:10DCE00010B501210148F7F7F9FB10BD000402400F
:10DCF00010B501210148F7F7EFFB10BD0004024009
:10DD000010B502210148F7F7E9FB10BD00040240FD
:10DD100010B502210148F7F7DFFB10BD00040240F7
:10DD200010B54FF400610248F7F7D8FB10BD0000B2
:10DD30000014024010B54FF400610248F7F7CCFB25
:10DD400010BD000000140240002101280BDB082850
:10DD500009DC421ED1B2114A126801238B409A435A
:10DD60000E4B1A6018E010280ADCA0F10902D1B2AB
:10DD70000A4A536801228A409343084A53600BE0E1
:10DD8000182809DCA0F11102D1B2044A92680123DB
:10DD90008B409A43014B9A6070470000F02B0120A2
:10DDA00010B54FF480710248F7F796FB10BD0000E4
:10DDB0000008024010B54FF480710248F7F78EFB5F
:10DDC00010BD0000000802400CB50020019000903A
:10DDD0003448006840F480303249086000BF314860
:10DDE000006800F4003000900198401C01900098F9
:10DDF00018B90198B0F5A04FF1D12A48006800F495
:10DE0000003010B10120009001E000200090009847
:10DE1000012846D123484030006840F08050214915
:10DE2000403108602048006840F440401E490860C6
:10DE30001C48083000681B49083108600846006823
:10DE400040F4004008600846006840F4A0500860B4
:10DE50001648091F0860081F006840F08070091FFD
:10DE6000086000BF0F48006800F000700028F9D07B
:10DE700040F205700E4908600A480830006820F03A
:10DE800003000849083108600846006840F00200B5
:10DE9000086000BF03480830006800F00C00082844
:10DEA000F8D10CBD00380240007000400854400713
:10DEB000003C024010B507F06BFC08F09BFA08F03C
:10DEC000FFFA0A490A4807F00BFB0A490A4807F01B
:10DED000F3FA07F07DFCFBF7FBFC08F071F808F0A3
:10DEE000BFF80649064808F0BCFD10BD8D64010866
:10DEF000596401084525010855250108920D0020A7
:10DF00008E0D00209FED0A0A0A4981ED000A9FED5F
:10DF1000080A094981ED000A9FED050A074981EDCC
:10DF2000010A9FED030A064981ED010A70470000CE
:10DF3000000000002C33012044330120683301200D
:10DF400088330120DFED050A0548C0ED000ADFED4A
:10DF5000030A0448C0ED000A7047000000000000FA
:10DF60002C3301204433012010B528480078B8B183
:10DF700000202649087000240FE004EB8401244AA5
:10DF800002EBC1002821F2F7BCFD00202149085511
:10DF9000343141F82400601CC4B2312CEDDB33E095
:10DFA00000242FE01B48005D50B31B48D0F804014B
:10DFB0001A490968401A40F2DC51884220D31648B9
:10DFC000D0F80401154908604FF4AF611448F2F726
:10DFD00098FD04EBC40000EB0412124800EB0211A0
:10DFE0004FF4C8720E48F2F75AFD4FF4AF620C4975
:10DFF000062001F04DF800200649343141F8240094
:10E00000601CC4B2312CCDDB10BD00000C280020F8
:10E01000DC3301201488012054390220102800200C
:10E02000F4900120843B012010B51548006840F4AD
:10E030007000134908601348006840F0010011495E
:10E04000086000200F49083108600E4800680E493A
:10E0500008400C4908600D48091D0860081F006849
:10E0600020F48020091F0860002006490C31086058
:10E07000FFF7AAFE4FF0006001498039086010BD2B
:10E0800088ED00E000380240FFFFF6FE103000246B
:10E0900010B5002400BF00BFF2F764F9044600BFCA
:10E0A00000BFFAF7F1FA00BF00BF2046F2F75EF9B1
:10E0B00000BF00BF0121054800F072F818B101212E
:10E0C000024800F067F8FAF7F5FA10BD00040040C6
:10E0D00010B5002400BF00BFF2F744F9044600BFAA
:10E0E00000BFFAF7D1FA00BF00BF2046F2F73EF9B1
:10E0F00000BF00BF0121054800F052F818B101210E
:10E10000024800F047F8FAF7D5FA10BD00080040C1
:10E1100010B5002400BF00BFF2F724F9044600BF89
:10E1200000BFFAF7B1FA00BF00BF2046F2F71EF9B0
:10E1300000BF00BF0121064800F032F828B10121DC
:10E14000034800F027F806F0DDFFFAF7B3FA10BD38
:10E15000000C004010B5002400BF00BFF2F702F928
:10E16000044600BF00BFFAF78FFA00BF00BF204689
:10E17000F2F7FCF800BF00BF0121054800F010F8DD
:10E1800018B10121024800F005F8FAF793FA10BD22
:10E1900000140040CA43028270470146486A704733
:10E1A00030B50246002000230024158A05EA010349
:10E1B000958905EA010413B10CB1012000E00020AB
:10E1C00030BD000010B52DED060B2DED0A8B9DED39
:10E1D0000B0ADDED0E0A30EE600A10EE101A08464A
:10E1E00009F028FB41EC1C0B9FED201BB0EE4C0A04
:10E1F000F0EE6C0A01F08CFCB0EE40AAF0EE60AAE2
:10E200009DED0A0ADDED0D0A30EE600A10EE101ADF
:10E21000084609F00FFB41EC1C0B9FED141BB0EE00
:10E220004C0AF0EE6C0A01F073FCB0EE40BAF0EE6E
:10E2300060BA53EC1A2B51EC1B0B08F01FFD41EC9C
:10E24000190BB0EE490AF0EE690A02F0EDFAB0EEF1
:10E25000408AF0EE608A51EC180B08F0DDFC00EE0D
:10E26000100ABDEC0A8B06B010BD000000000000D3
:10E270000000004008B5014608880090BDF8000085
:10E2800008BD0146086870472DE9F04100260027C7
:10E2900000BF00BFF2F766F8074600BF00BFFAF7FD
:10E2A000F3F900BF00BF3846F2F760F800BF00BFC7
:10E2B00040F225516A4800F00DFCE0B101266848A3
:10E2C00000F0C2FCC4B26748B0F80008401CC0F3BC
:10E2D00009006449B1F8021888420CD06148B0F8CE
:10E2E000000860490C540846B0F80008401CC0F310
:10E2F0000900A1F8000840F22771594800F0EAFB34
:10E3000038B35848B0F804085649B1F8061888429E
:10E3100012D05448B0F80658B0F80608401CC0F3B4
:10E3200009005049A1F8060801F58060445D2146C6
:10E330004B4800F08EFC51E0002240F22771484823
:10E3400000F0F2FB012240F22661454800F0ECFBB0
:10E3500044E040F22661424800F0BCFB08B341486B
:10E36000B0F804083F49B1F80618884212D03D4879
:10E37000B0F80658B0F80608401CC0F30900394947
:10E38000A1F8060801F58060445D2146344800F09C
:10E3900060FC23E0002240F22661314800F0C4FB1B
:10E3A0001CE0DEB92E4800F04FFCC4B22D48B0F896
:10E3B0000008401CC0F309002A49B1F8021888423D
:10E3C0000CD02848B0F8000826490C540846B0F88C
:10E3D0000008401CC0F30900A1F800083C2C06D13D
:10E3E00000202149086001202049086008E03E2CF7
:10E3F00006D11E480068012802D102201B4908608E
:10E40000194800686E2804DD002018490860164984
:10E41000086016480068012808D1134801680068A0
:10E42000401C114A10601248445415E00F4800681F
:10E43000022811D10C4801680068401C0A4A10608B
:10E440000B4844540020094908600120094981F81B
:10E450002500642081F82700FAF72CF9BDE8F08147
:10E46000004C0040701A01204C110020481100207F
:10E47000242B0120003301202DE9F041002640F239
:10E480002551564800F026FB074600BF00BFF1F7B4
:10E4900069FF064600BF00BFFAF7F6F800BF00BFED
:10E4A0003046F1F763FF00BF00BF40F225514B48F3
:10E4B00000F010FBD8B1494800F0C6FBC5B248488F
:10E4C000B0F80008401CC0F309004549B1F8021833
:10E4D00088420CD04248B0F8000841490D54084623
:10E4E000B0F80008401CC0F30900A1F8000840F291
:10E4F00027713A4800F0EEFA38B33948B0F804080A
:10E500003749B1F80618884212D03548B0F80648A5
:10E51000B0F80608401CC0F309003149A1F806080C
:10E5200001F58060055D29462C4800F092FB50E023
:10E53000002240F22771294800F0F6FA012240F249
:10E540002661264800F0F0FA43E040F226612348B5
:10E5500000F0C0FA08B32248B0F804082049B1F826
:10E560000618884212D01E48B0F80648B0F80608CF
:10E57000401CC0F309001A49A1F8060801F58060A3
:10E58000055D2946154800F064FB22E0002240F2B8
:10E590002661124800F0C8FA1BE0104800F054FB56
:10E5A000C5B20F48B0F80008401CC0F309000C4980
:10E5B000B1F8021888420CD00948B0F800080849A0
:10E5C0000D540846B0F80008401CC0F30900A1F83B
:10E5D0000008FAF76FF8BDE8F08100000010014074
:10E5E000580201202DE9F0410026002700BF00BF9E
:10E5F000F1F7B8FE064600BF00BFFAF745F800BFC6
:10E6000000BF3046F1F7B2FE00BF00BF40F2255117
:10E610004E4800F05FFAE0B101274C4800F014FBCF
:10E62000C5B24B48B0F80008401CC0F30900484987
:10E63000B1F8021888420CD04548B0F800084449A7
:10E640000D540846B0F80008401CC0F30900A1F8BA
:10E65000000840F227713D4800F03CFA38B33C48CE
:10E66000B0F804083A49B1F80618884212D0384880
:10E67000B0F80648B0F80608401CC0F30900344959
:10E68000A1F8060801F58060055D29462F4800F0D5
:10E69000E0FA51E0002240F227712C4800F044FAE1
:10E6A000012240F22661294800F03EFA44E040F29F
:10E6B0002661264800F00EFA08B32548B0F8040891
:10E6C0002349B1F80618884212D02148B0F806480C
:10E6D000B0F80608401CC0F309001D49A1F806085F
:10E6E00001F58060055D2946184800F0B2FA23E084
:10E6F000002240F22661154800F016FA1CE0DFB94E
:10E70000124800F0A1FAC5B21148B0F80008401C48
:10E71000C0F309000E49B1F8021888420CD00C4829
:10E72000B0F800080A490D540846B0F80008401C2B
:10E73000C0F30900A1F800082946064803F06CF967
:10E7400005490870F9F7B6FFBDE8F08100440040C4
:10E75000600A0120FC2B0120401600202DE9F04129
:10E760000026002700BF00BFF1F7FCFD074600BFF1
:10E7700000BFF9F789FF00BF00BF3846F1F7F6FD8B
:10E7800000BF00BF40F225516A4800F0A3F9E0B194
:10E790000126684800F058FAC4B26748B0F800088B
:10E7A000401CC0F309006449B1F8021888420CD03B
:10E7B0006148B0F8000860490C540846B0F80008F9
:10E7C000401CC0F30900A1F8000840F22771594825
:10E7D00000F080F938B35848B0F804085649B1F849
:10E7E0000618884212D05448B0F80658B0F8060807
:10E7F000401CC0F309005049A1F8060801F58060EB
:10E80000445D21464B4800F024FA51E0002240F2DA
:10E810002771484800F088F9012240F226614548F6
:10E8200000F082F944E040F22661424800F052F9DB
:10E8300008B34148B0F804083F49B1F806188842C7
:10E8400012D03D48B0F80658B0F80608401CC0F396
:10E8500009003949A1F8060801F58060445D2146A8
:10E86000344800F0F6F923E0002240F226613148F6
:10E8700000F05AF91CE0DEB92E4800F0E5F9C4B208
:10E880002D48B0F80008401CC0F309002A49B1F82F
:10E89000021888420CD02848B0F8000826490C54C9
:10E8A0000846B0F80008401CC0F30900A1F80008B1
:10E8B0003C2C06D100202149086001202049086035
:10E8C00008E03E2C06D11E480068012802D1022033
:10E8D0001B490860194800686E2804DD00201849AB
:10E8E00008601649086016480068012808D11348D6
:10E8F00001680068401C114A10601248445415E039
:10E900000F480068022811D10C4801680068401CBB
:10E910000A4A10600B48445400200949086001204D
:10E92000094981F82500642081F82700F9F7C2FE23
:10E93000BDE8F0810048004068120120401100202D
:10E940003C110020AC2A0120D43201202DE9F041F5
:10E950000026002700BF00BFF1F704FD074600BFF7
:10E9600000BFF9F791FE00BF00BF3846F1F7FEFC8B
:10E9700000BF00BF40F225514E4800F0ABF8E0B1B7
:10E9800001264C4800F060F9C5B24B48B0F80008C9
:10E99000401CC0F309004849B1F8021888420CD065
:10E9A0004548B0F8000844490D540846B0F800083E
:10E9B000401CC0F30900A1F8000840F227713D484F
:10E9C00000F088F848B33C48B0F804083A49B1F878
:10E9D0000618884214D03848B0F80648B0F806083F
:10E9E000401CC0F309003449A1F8060801F5806015
:10E9F000055DFFF7DFF929462E4800F02AF955E0BA
:10EA0000002240F227712B4800F08EF8012240F2DC
:10EA10002661284800F088F848E040F22661254841
:10EA200000F058F828B32448B0F804082249B1F897
:10EA30000618884214D02048B0F80648B0F80608F6
:10EA4000401CC0F309001C49A1F8060801F58060CC
:10EA5000055DFFF7AFF92946164800F0FAF825E002
:10EA6000002240F22661134800F05EF8FFF798F9A3
:10EA70001CE0DEB90F4800F0E7F8C5B20E48B0F868
:10EA80000008401CC0F309000B49B1F80218884285
:10EA90000CD00948B0F8000807490D540846B0F8F2
:10EAA0000008401CC0F30900A1F80008F9F702FEB5
:10EAB000BDE8F081001401407822012021B1828953
:10EAC00042F40052828104E082894DF6FF731A40BD
:10EAD0008281704770B50246002400230025002083
:10EAE00040F66A16B14200D100BFC1F3421501F0F1
:10EAF0001F03012606FA03F3012D02D19689334044
:10EB000006E0022D02D1168A334001E0968A334096
:10EB10000C12012606FA04F41688344013B10CB125
:10EB2000012000E0002070BDF0B50346002400265F
:10EB30000025002040F66A17B94200D100BF1846F0
:10EB4000C1F3421401F01F06012707FA06F5012C54
:10EB500001D10C3004E0022C01D1103000E014305F
:10EB60001AB107682F43076002E00768AF430760E8
:10EB7000F0BD00002DE9FF4705460E460024A146E2
:10EB800000BFA046B08900B100BF2C8A24F44054D5
:10EB9000F08804432C82AC8941F20C608443B08835
:10EBA00031890843718908430443AC81AC8A24F459
:10EBB0004074B0890443AC826846FEF743F82048AD
:10EBC000854202D01F48854202D1DDF80C9001E059
:10EBD000DDF80890A88900F4004040B109EBC900B5
:10EBE00000EB091031684900B0FBF1F707E009EBD1
:10EBF000C90000EB091031688900B0FBF1F764200F
:10EC0000B7FBF0F004012009642101FB1078A8890A
:10EC100000F4004040B1322000EBC800B0FBF1F03E
:10EC200000F00700044308E0322000EB08106421E4
:10EC3000B0FBF1F000F00F0004432C81BDE8FF872A
:10EC4000001001400014014001468888C0F308000C
:10EC50007047C1F3080282807047000030B5ADF202
:10EC6000D47D4FF4FA6201A90620FEF733F9054678
:10EC70005DB32A4601A9012000F00AFA002422E02F
:10EC8000144890F8880D50B901A9085D1249F6F7AB
:10EC90005DF9042803D101210E4880F8881D0D4834
:10ECA00090F8880D70B1F6F731FA08B9FEF70CFF4D
:10ECB0000021084880F8881D90F83407012801D108
:10ECC000FEF74AF9641CAC42DAD3FFF74DF90DF2B6
:10ECD000D47D30BDF81B022048C901200FB430B5E7
:10ECE000ADF2044D04460DF58360CDF8000468468E
:10ECF000DDF80024DDF81414F1F74AFB6846F1F75B
:10ED00005EFE05462A466946204600F0C1F900200D
:10ED1000CDF800040DF2044D30BC5DF814FB00008A
:10ED200030B5BDB078221FA90320FEF7D3F8054601
:10ED3000002D4ED0002444E01FA8005D3C2806D1E1
:10ED400000202E49086001202D4908600AE01FA814
:10ED5000005D3E2806D12A480068012802D1022021
:10ED600027490860254800686E2804DD00202449F2
:10ED70000860224908602248006801280AD11FA8BB
:10ED8000015D1E4802680068401C1C4B186001A809
:10ED9000815415E01A480068022811D11FA8015DAE
:10EDA000164802680068401C144B186001A8815482
:10EDB0001846016801A8FAF7DFFD00201049086035
:10EDC000641CAC42B8D30F48D0F804010E49086067
:10EDD00011E00C48D0F804010B490968401AB0F55D
:10EDE0007A7F08D90748D0F8040107490860002055
:10EDF000064981F825003DB030BD0000A41900206F
:10EE0000A019002054390220A8190020D432012072
:10EE100010B50120FDF79AFF064908600220FDF7B2
:10EE200095FF044948600320FDF790FF0149886081
:10EE300010BD0000E42B012010B532240A490878E7
:10EE40000121FEF773FE084908790221FEF76EFEE4
:10EE50000549087A0321FEF769FE00BF201EA4F1D0
:10EE60000104FBD110BD0000F02B012000BFFEE724
:10EE700070B504460F49C86880470E494869804705
:10EE80000C48016A0F2088470A48016AC4F307202A
:10EE90008847E0B2074A116A88470649C86980472F
:10EEA0000546044988698047024908698047284621
:10EEB00070BD0000C80D00202DE9F04105460E464A
:10EEC000174600241349C86880471249486980479B
:10EED0001048016A0F2088472A19C2F307200D4AFB
:10EEE000116A88472A19D0B20A4A116A884700BFB6
:10EEF00005E00849C86980473055601C84B2BC42AF
:10EF0000F7DB044988698047024908698047BDE802
:10EF1000F0810000C80D002070B504460D460F4971
:10EF2000C86880470D49486980470C48016AF0204D
:10EF300088470A48016AC4F307208847E0B2074AB5
:10EF4000116A88470548016A284688470349886945
:10EF5000804702490869804770BD0000C80D002045
:10EF60002DE9F04105460E46174600241349C868AE
:10EF700080471249486980471048016AF020884755
:10EF80002A19C2F307200D4A116A88472A19D0B2FC
:10EF90000A4A116A884700BF05E0305D074A116AD6
:10EFA0008847601C84B2BC42F7DB0449886980470B
:10EFB000024908698047BDE8F0810000C80D0020C3
:10EFC0000020014908607047082C004040F0800193
:10EFD000014A116070470000002C004001200149E7
:10EFE00008607047A4800542F8B506460C461546F1
:10EFF0000121C802FDF706FE1048007830400F4995
:10F000000870284600F024F8204600F02DF80B4840
:10F010000078FFF7DBFF00208DF800008DF801007D
:10F020008DF8020001208DF803006846F9F75AFABE
:10F03000FFF7C6FFFFF7D2FFF8BD0000F412002073
:10F0400000F07F01014A116070470000002C004071
:10F050000021044A126822F4C0710143014A116080
:10F0600070470000042C004008B5002100910749BA
:10F07000096821F07F01009100F07F01009A11439F
:10F080000091024A0099116008BD0000042C004064
:10F090002DE9F047054689469246012D02D1274CBD
:10F0A000274E15E0022D02D1264C274E10E0032DED
:10F0B00002D1264C264E0BE0042D02D1254C264EC3
:10F0C00006E0062D02D1254C254E01E0BDE8F08773
:10F0D000B4F80408B4F80618884202D14FF00108C9
:10F0E00001E04FF00008002719E0B4F80408401CC4
:10F0F000C0F30900B4F8061888420ED019F80710BA
:10F10000B4F8042804F580608154B4F80408401C65
:10F11000C0F30900A4F8040800E002E07F1C574592
:10F12000E3D300BFB8F1000F05D0012240F22771F0
:10F130003046FFF7F9FC00BFC8E700005802012085
:10F1400000100140600A01200044004068120120C4
:10F1500000480040701A0120004C00407822012035
:10F16000001401401CB501215A20FDF73BFD4FF46E
:10F17000FE70009002208DF8050001208DF8070038
:10F1800000208DF806008DF8040069461148F6F756
:10F190002FF94FF40040009069460F48F6F728F920
:10F1A0000320009002208DF8050001208DF8070053
:10F1B00000208DF8060001208DF8040069460748FC
:10F1C000F6F716F94FF40070009069460448F6F718
:10F1D0000FF91CBD00180240000C02400010024054
:10F1E0000004024010B51820FDF73EFE80F001013A
:10F1F000A1480170A14880F88010B0F844004AF29C
:10F200000701884204D100219C4880F8811009E060
:10F210001720FDF729FE80F00101974841709748BB
:10F2200080F881101620FDF71FFE80F00101924842
:10F230008170924880F882100620FDF715FE8E49F5
:10F2400088718E4981F87C000220FDF70DFE8B4904
:10F2500081F890000120FDF707FE884981F89100B0
:10F260000520FDF701FE84490871844981F87F007B
:10F270000420FDF7F9FD80490873804981F8920068
:10F280000320FDF7F1FD7C4948737C4981F8930028
:10F290000E20FDF7E9FD7A4908700F20FDF7E4FD27
:10F2A000784908701020FDF7DFFD7749087077482E
:10F2B000007818BB72480078012824D16F48007983
:10F2C00008B9012000E000206C4908710846007967
:10F2D000A8B100210320FAF7EFFA684890F89000EF
:10F2E000664991F89110084020B14FF48060FDF715
:10F2F00079FE08E04FF48060FEF7B4FC03E00121E2
:10F300000320FAF7D9FA5D48007920B164215B48FF
:10F31000A0F85A1003E096215848A0F85A1058480F
:10F3200000785A49087055480079002875D1584925
:10F33000524881670C20FDF797FD504981F88600FF
:10F340000D20FDF791FD4D4981F887004D4800786B
:10F35000012810D14F48007868B9084690F88D0010
:10F3600048B9084690F88C0008B9012100E0002156
:10F37000424880F88C1044480078012810D1464853
:10F38000007868B93D4890F88C0048B93B4890F83F
:10F390008D0008B9012100E00021384880F88D1067
:10F3A000384800783B490870374800783A49087077
:10F3B000324890F8860018B10120304988710EE07B
:10F3C0002E4890F8870038B12C4890F8930018B96F
:10F3D00002202A49887102E000202849887108200B
:10F3E000FDF742FD254981F888000920FDF73CFD25
:10F3F000224981F889000A20FDF736FD1F4981F86E
:10F400008A000B20FDF730FD1C4981F88B0008466F
:10F4100090F8880010B1012048711AE0174890F860
:10F42000890018B102201549487112E0134890F87C
:10F430008A0018B10320114948710AE00F4890F87A
:10F440008B0018B104200D49487102E000200B49DF
:10F4500048710A4890F87D0018B10121074880F8EA
:10F46000AC10064890F8930020B19FED0C0A0C48B0
:10F4700080ED030A10BD00002C390220543902200F
:10F48000351F0020371F0020381F0020361F0020A6
:10F490009F860100391F00203A1F00200000000055
:10F4A000683301201CB501217220FDF79BFB4FF44E
:10F4B0007040009002208DF8050001208DF80700B3
:10F4C00000208DF8060001208DF8040069460F48E1
:10F4D000F5F78EFF0320009069460D48F5F788FF89
:10F4E0004FF4C070009069460A48F5F781FF032089
:10F4F000009069460848F5F77BFF4FF400600090E4
:10F5000069460248F5F774FF1CBD00000014024074
:10F5100000180240001002400004024010B54148AB
:10F5200001680068401C3F4A1060B1F57A7F78DDC1
:10F5300006F062F9FFF7F4FBF5F7BCFE3A48D0F8A5
:10F5400004013A490968401A092806D93648D0F812
:10F5500004013649086006F023FB3348D0F8040163
:10F5600033490968401A0B2806D90023082231497B
:10F5700040F20360F4F74EFB2B48D0F804012E490B
:10F580000968401A0F2820D92C48006830B10023A0
:10F5900008222B4940F20360F4F73CFB2248D0F8E4
:10F5A000040125490968401A11280ED91E48D0F8CF
:10F5B0000401214908602348006830B10023082273
:10F5C0001F4940F20460F4F725FB1748D0F8040106
:10F5D0001D490968401A0D280BD91348D0F80401B9
:10F5E0001949086000230822124940F20460F4F728
:10F5F00011FB0D48007978B90B4890F88C000A4946
:10F6000091F88D10084320B12B200749487203E080
:10F6100007E0012004494872034A917B507AF8F7C9
:10F620002DFF10BDF805002054390220E805002008
:10F63000EC0500208C050020F0050020FC050020D2
:10F640006405002000060020F405002010B5754870
:10F65000B0F844004AF20101884204D14FF4F87036
:10F660007149086076E06F48B0F844004AF2020140
:10F67000884204D14FF415706B4908606AE069480C
:10F68000B0F844004AF20301884204D14FF42E70CE
:10F69000654908605EE06348B0F844004AF204013E
:10F6A000884204D14FF4F8705F49086052E05D4829
:10F6B000B0F844004AF20601884204D140F22B20FF
:10F6C0005949086046E05748B0F844004AF205013D
:10F6D000884204D14FF41570534908603AE051480C
:10F6E000B0F844004AF20701884204D14FF4F870A0
:10F6F0004D4908602EE04B48B0F844004AF208013A
:10F70000884204D14FF42E704749086022E04548F2
:10F71000B0F844004AF20901884204D14FF4157050
:10F720004149086016E03F48B0F844004AF2100131
:10F73000884204D14FF4F8703B4908600AE0394828
:10F74000B0F844004AF21101884203D140F28F2000
:10F750003549086005F058FB3349098888B205F03F
:10F76000D9FE3048407948B92E4890F82400032843
:10F7700004D02C4890F82400042802D10320294901
:10F7800088832848007B78B90120264908730846F9
:10F79000D0F80401254908604FF40050FDF722FC21
:10F7A00001210220FAF788F81E48D0F804011F4909
:10F7B0000968401A47F23051884229D3194890F815
:10F7C000A80000F0800018BB4FF40050FEF74AFA82
:10F7D000C820F8F7CDFE164908701248D0F8040189
:10F7E00014490968401A42F21071884204D30D4846
:10F7F000D0F804010F4908600D48007820B10121BC
:10F800000220FAF759F803E000210220FAF754F831
:10F810000449087FF6F719FFFFF720FAF3F7A2FC77
:10F8200010BD00005439022064030020680300204A
:10F83000700300206C03002003B40198410000987D
:10F8400050EAC12018BF04204A0D18BF40F0010043
:10F8500040F2FF72B2EB515F08BF40F00200012896
:10F8600008BF052002B0704730B52DED048B81B084
:10F87000B0EE408AF0EE608A6A4651EC180B03F055
:10F8800083FA00989FED329B7E300090002821DCA7
:10F8900053EC192B51EC180B07F004FC1AD0002183
:10F8A00040F608004FF00000044651EC180B07F03A
:10F8B000B3F908EE100A40F6080004EA00014FF020
:10F8C0000000B5EEC08AF1EE10FA04BF0220F1F795
:10F8D00054F92DE00098FF2830DB002108464FF056
:10F8E000000000F4400553EC192B51EC180B07F005
:10F8F000A9FD8CBF002401240220F1F73EF99FED01
:10F90000168A4DB1002C0CBF4FF400004FF480005C
:10F91000A84218BF9FED118A042108464FF000004D
:10F92000002C01BFB1EE480A01B0BDEC048B30BD24
:10F93000B0EE480A01B0BDEC048B30BD51EC180BA1
:10F9400007F06AF901B000EE100ABDEC048B30BD7F
:10F9500000000000000000000000807FFFFF7F7FAC
:10F9600010B52F499FED2C1B2DED020B84B005988F
:10F9700020F000408842D8BF9DED040B2DDD2949C1
:10F98000884209D1049840B94FF00100F1F7F5F829
:10F9900001F086FD06B010BD05DB9DED040B01F006
:10F9A0006BFD06B010BD68469DED040B00F0BCFF7A
:10F9B00010F0030004BF9DED021B9DED000B0CD069
:10F9C00001280ED09DED021B9DED000B022817D0E3
:10F9D000012001F0F9FA06B010BD01F0C1F906B03E
:10F9E00010BD9DED021B9DED000B012001F0ECFA16
:10F9F00051EC100B07F004F906B041EC100B10BDF0
:10FA000001F0AEF951EC100B07F0FAF806B041EC3A
:10FA1000100B10BD000000000000000000000000FE
:10FA2000FB21E93F0000F07F2DED020B019820F053
:10FA3000004001909DED000B02B0704700000000F7
:10FA400030B540F2FF742DED048BF0EE608A18EEB5
:10FA5000901A85B0B0EE408A9FED2B9B05468DED48
:10FA6000008B34EA115147D053EC192B51EC180B91
:10FA700007F018FB40D02A4651EC180B07F08EFF18
:10FA800041EC180B18EE900A8DED008B34EA105003
:10FA90001CD053EC192B51EC180B07F003FB2BD1A6
:10FAA0000220F1F76AF801F01BFD10EE901A18EE33
:10FAB000900A8DED020B8DED008B61F31E0003901B
:10FAC0009DED020B05B0BDEC048B30BD0220F1F7BB
:10FAD00054F801F0F5FC10EE901A18EE900A8DED36
:10FAE000020B8DED008B61F31E0003909DED020B68
:10FAF00005B0BDEC048B30BD05B0B0EE480AF0EEA9
:10FB0000680ABDEC048B30BD00000000000000005E
:10FB10002DE9F04D2DED040B2DED0E8B96B0DDE9AA
:10FB20002550279CDDF890A025F0004624F00048E1
:10FB3000BAF1000F14BF0121002101EB4502FC497D
:10FB400053184A1093422AD3002814BF01230023DC
:10FB500003EB44030B44F7498B4220D358EA0001DE
:10FB60009FEDF59B76D0DFF8D8B35D4503D1BAF1B0
:10FB7000000F05D188E0BAF1000F08BF002100D0C6
:10FB8000012101EB450111F5001F08D8002814BF21
:10FB90000121002101EB440111F5001F0BD99DED5E
:10FBA000261B9DED240B16B0BDEC0E8B04B0BDE8FA
:10FBB000F04D01F06BBC0027002DBCBFE14988452A
:10FBC00021DAE1498845A8BF02271CDAC3451ADCBF
:10FBD000DE4901EB2851142908DDC1F1340220FA75
:10FBE00002F101FA02F282420DD108E058B9C1F1E6
:10FBF000140228FA02F101FA02F2424503D101F09F
:10FC00000101C1F1020756EA0A0124D1002C22DACF
:10FC1000002D18BF022F01D0012F0AD00220F0F7CB
:10FC2000ACFF16B0BDEC0E8B04B0BDE8F04D01F09A
:10FC30000BBC0220F0F7A1FF01F006FC51EC100B09
:10FC400006F0DEFF41EC100B16B0BDEC0E8B04B0DD
:10FC5000BDE8F08D18E09FEDBEAB9FEDBF8B002897
:10FC600071D1B848804522D105F1804010F580104F
:10FC700008BFBAF1000F07D0B3450ADC002CA8BFBB
:10FC80009DED260BE0DA0DE0B0EE490AF0EE690AD0
:10FC9000DAE7002C06DA9DED260B51EC100B06F08E
:10FCA000AFFF6FE0AE48784490ED000BCCE7D8454D
:10FCB0004DD1002C48DA2EB186423AD1BAF1000F6C
:10FCC00042D126E0BAF1000F13D00220F0F755FF21
:10FCD00001F0F6FB8DED020B9DED240B8DED000B7D
:10FCE00010EE900A039961F31E0003909DED020B44
:10FCF000AAE78DED02AB9DED240B1AEE901A10EEE3
:10FD0000900A8DED000B61F31E0003909DED020B38
:10FD10009AE78DED028B9DED240B18EE901A10EEF4
:10FD2000900A8DED000B61F31E0003909DED020B18
:10FD30008AE709DA9DED240B51EC190B53EC102BDB
:10FD400007F058F81EE020E09DED240B7CE786428A
:10FD50001BDAB4F1804F0DD0A4F10050B0F1FF5088
:10FD600013D1002D11DB9DED240B51EC100B06F08F
:10FD7000D5FB07E09DED240B53EC102B51EC100B41
:10FD800000F0C2BC41EC100B5EE79DED240B51EC82
:10FD9000100B02F0E9FFBAF1000FCDE90E0142D1DC
:10FDA0009FED710B46B3A6F1E040B0F17F600CD03F
:10FDB0005E4538D1002D00DAA7B3022F0CBF012019
:10FDC0004FF0FF3007F0D9F9DCE7002D01DD002C02
:10FDD0000DDA002D01DD002C1FDB002D16DA002CC2
:10FDE00014DB012F08BF9FED620B3FF42DAFB0EE87
:10FDF0004A0AF0EE6A0A27E7022F18BF002D0CD03E
:10FE0000012F0AD1002DFFF61FAF06E0002DB8BF6D
:10FE1000002C08DA012F3FF417AFB0EE480AF0EEDD
:10FE2000680A11E71BE0012000EBE57050EA0701CA
:10FE300015D0791EB0EE498AF0EE698A084308BFF2
:10FE40009FED4D8B4E480025804570DD4D494E4855
:10FE5000884514DDB0420DDB002C19DB2FE00120BA
:10FE6000F0F78BFE16B0BDEC0E8B04B0BDE8F04D84
:10FE700001F016BBB34502DC002C09DC1FE0864212
:10FE800002DA002C1BDA03E05E452BDD002C16DDC8
:10FE90000220F0F772FE01F013FB8DED020B53EC24
:10FEA0001A2B51EC180B07F0CFF9CDE9000103999B
:10FEB000019861F31E0003909DED020BC4E6022041
:10FEC000F0F75BFE01F00CFB10EE901A18EE900AB2
:10FED0008DED020B8DED008B61F31E0003909DED07
:10FEE000020BB1E69DED0E0B53EC192B51EC100BF0
:10FEF00007F0B6FB9FED260BCDE9080153EC102B64
:10FF00009DED080B51EC100B07F09EF99FED221BA5
:10FF100053EC112B07F0CCFA9DED081B53EC112B81
:10FF200007F092F99FED1E1B53EC112B3CE08CE087
:10FF3000FFFF1F00FFFF0F00000000000000F03F68
:10FF40000000F03F0000F07F0000404301FCFFFF95
:10FF5000000000000000F07F000000000000000032
:10FF60002E7F000000000000000000000000008064
:10FF7000000000000000F0FF000000000000F0BFE3
:10FF80000000E0410000F043FFFFEF3F00000000F1
:10FF9000000000000000D03F555555555555D53F40
:10FFA000000000000000E03F07F082FA9DED080B22
:10FFB00041EC1A0B53EC102B51EC100B07F044F9E9
:10FFC00053EC1A2B07F040F941EC1A0B9FEDFE0B96
:10FFD00053EC102B9DED080B51EC100B07F034F98E
:10FFE00041EC1B0B9FEDFA0B51EC1A0B53EC102B51
:10FFF00007F02AF941EC1A0B9FEDF70B53EC102B8D
:020000040801F1
:100000009DED080B51EC100B07F01EF953EC1A2B69
:1000100007F026FB41EC1A0B51EC1B0B53EC1A2B8F
:1000200006F02CFE0690CDE906519DED060B53EC33
:100030001B2B51EC100B07F013FB53EC1A2B07F0A2
:1000400037FA41EC100B00F0A1B90020B6F5801F83
:100050000EDA9FEDE30B53EC102B9DED0E0B51ECE4
:10006000100B07F0F1F8CDE90E016FF034000E46E9
:1000700000EB2650A0F2FF37C6F31300DA4940F038
:100080007F6646F040568842D8BF002408DDD74935
:100090008142C8BF012403DC0024A6F580167F1C22
:1000A000D348784400EBC4000F9690ED00CB9DED53
:1000B0000E0B53EC1C2B51EC100B07F0D1FA9DEDFD
:1000C0000E0B41EC1B0B53EC1C2B51EC100B06F0F0
:1000D000D5FD41EC100B51EC190B53EC102B06F035
:1000E00089FE41EC1D0B51EC1B0B53EC1D2B07F053
:1000F000ABF841EC1A0BBF488DED10AB784410956E
:1001000090ED000B4FF0005040EA660000EB844099
:100110008DED080B00F5002009909DED080B53ECC8
:100120001C2B51EC100B07F09BFA9DED0E1B53ECB2
:10013000112B07F0BDF941EC100B53EC102B9DED8A
:10014000100B51EC100B07F07FF89DED080B41EC04
:100150001C0B53EC102B9DED100B51EC100B07F00A
:1001600073F853EC1B2B07F0A3F953EC1C2B07F08F
:1001700077FA53EC1D2B07F067F841EC1C0B53EC9E
:100180001A2B51EC1A0B07F05FF841EC1B0B9A4845
:100190000621B0EE4B0AF0EE6B0A784400F098FEB0
:1001A000B0EE401AF0EE601AB0EE41DAF0EE61DA2D
:1001B00053EC1B2B51EC1B0B07F046F853EC1D2B9B
:1001C00007F042F89DED100B41EC1B0B53EC1A2B82
:1001D00051EC100B06F052FD53EC1C2B07F034F8D9
:1001E00053EC1B2B06F04AFD9DED100B41EC1B0B55
:1001F00053EC102B51EC100B07F026F841EC1D0BC3
:100200009FED7FEB53EC1E2B06F038FD53EC1B2BC0
:1002100006F034FD0890CDE908519DED080B53EC34
:100220001E2B51EC100B07F01BFA53EC1D2B07F0A3
:1002300017FA53EC1B2B07F03BF99DED080B41EC33
:100240001D0B53EC102B9DED100B51EC100B06F019
:10025000FBFF41EC1B0B53EC1A2B51EC1D0B06F072
:10026000F3FF9DED080B41EC1A0B53EC102B51ECF6
:100270001C0B06F0E9FF53EC1A2B06F0FFFC41ECD7
:100280001A0B51EC1B0B53EC1A2B06F0F7FC0C90DD
:10029000CDE90C519DED0C0B53EC1B2B51EC100BCD
:1002A00007F0DEF953EC1A2B07F002F941EC1B0BB7
:1002B0009FED550B53EC102B9DED0C0B51EC100BDF
:1002C00006F0C2FF41EC1A0B9FED510B51EC1B0BDA
:1002D00053EC102B06F0B8FF41EC1B0B9FED4E0BBF
:1002E00053EC102B9DED0C0B51EC100B06F0ACFFFA
:1002F00053EC1B2B06F0C2FC41EC100B4848784431
:1003000000EBC40090ED001B51EC100B53EC112BD3
:1003100006F0B4FC41EC1B0B384606F02EFFCDE98D
:10032000080153EC1B2B51EC1A0B06F0A7FC41EC17
:10033000100B3C48784400EBC40090ED00CB51EC2E
:10034000100B53EC1C2B06F099FC9DED081B53EC95
:10035000112B06F093FC0690CDE906519DED080B9C
:1003600053EC102B9DED060B51EC100B07F078F9B8
:1003700053EC1C2B07F074F953EC1A2B07F070F9AF
:1003800053EC1B2B07F094F841EC100B9DED261B52
:1003900053EC102B8DED001B00959DED260B51ECC1
:1003A000100B06F051FF9DED000B41EC1A0B53ECC6
:1003B000102B9DED260B51EC100B07F051F99DED24
:1003C000061B53EC112B2FE0000000604715F73F90
:1003D000FE822B654715F73F44DF5DF80BAE543EB8
:1003E00000000000000040438E9803007AB60B0026
:1003F000727A0000D87A0000AA790000000000009C
:100400000000000000000840000000E009C7EE3FC7
:10041000FD033ADC09C7EE3FF5015B14E02F3EBE59
:1004200036780000F077000006F00EFF53EC1A2B30
:1004300006F024FC9DED060B41EC1A0B53EC102B3F
:100440009DED000B51EC100B06F0FEFECDE90C010A
:100450009DED0C0B51EC1A0B53EC102B06F00EFC1F
:10046000CDE902010C46AA498C422FDB611A0843F0
:1004700018D19DED0C0B53EC102B9DED020B51ECA4
:10048000100B07F0EDF841EC1B0B9FEDA30B51ECAB
:100490001A0B53EC102B06F0F1FB53EC1B2B06F060
:1004A000D1FF2DD20220F0F768FB01F009F810EE21
:1004B000901A18EE900A8DED020B8DED008B61F312
:1004C0001E0003909DED020BFFF7BEBB944A24F083
:1004D0000041914214D39349214408437FF4EFAC87
:1004E0009DED0C0B53EC102B9DED020B51EC100B02
:1004F00007F0B6F853EC1A2B06F0A4FF7FF6DFAC3A
:1005000024F000408849894A002601EB20518242AC
:100510002BDA481C4FF4801121FA00F02044844A61
:10052000C0F30A517A44A1F2FF3192ED000B814AE7
:100530008DED080BCA4020EA0202C0F3130040F41C
:100540008010C1F1140120FA01F60992002CB8BF05
:1005500076429DED080B53EC102B9DED0C0B51ECEE
:10056000100B07F07DF8CDE90C019DED0C0B51EC63
:100570001A0B53EC102B06F081FB9FED6F0B0890CC
:10058000CDE9085153EC102B9DED080B51EC100BED
:1005900006F05AFE41EC1B0B9FED690B53EC102B40
:1005A0009DED080B51EC100B06F04EFE9DED0C0B73
:1005B00041EC1C0B53EC102B9DED080B51EC100B78
:1005C00007F04EF853EC1A2B06F072FF9FED5E1BFE
:1005D00053EC112B06F038FE53EC1C2B06F04EFBAF
:1005E00041EC1A0B51EC1B0B53EC1A2B06F046FB9B
:1005F000CDE902019DED020B53EC1B2B51EC100BCE
:1006000007F02EF853EC1A2B06F052FF9DED020B6B
:1006100041EC1A0B53EC102B51EC100B06F014FEAE
:10062000CDE908014A489DED080B0521784400F00A
:100630004FFC9DED081B51EC100B53EC112B06F0F9
:1006400003FE9DED021B53EC112B06F031FFCDE9AB
:1006500006019DED020B53EC1A2B51EC100B06F02A
:10066000F3FD53EC1A2B06F009FB9FED3B0B41EC1D
:100670001A0B53EC102B9DED060B51EC100B06F0F2
:10068000EFFF9DED060B41EC1B0B53EC102B9DED8A
:10069000020B51EC100B06F0D7FD53EC1B2B06F0B0
:1006A000A9FB53EC1A2B06F0DBFF9DED021B53EC6C
:1006B000112B06F0D5FF53EC192B06F0F9FECDE90E
:1006C000020101EB065001150029C8BF039015DC9B
:1006D0009DED020B324651EC100B07F05FF9FFF76E
:1006E000ABF8042808BF00F0FBFE32469DED020B7C
:1006F00051EC100B07F052F9CDE902019DED020B10
:1007000051EC180B53EC102B06F09EFDFFF73ABB93
:100710000000904000000000FE822B654715973CCA
:1007200000CC904000346F3F01FCFFFF0000E03F31
:10073000B0760000FFFF0F0000000000432EE63FF0
:10074000396CA80C615C20BEEF39FAFE422EE63F00
:10075000487500000000000000000000000000409C
:1007600010B52F499FED2C1B2DED020B84B0059881
:1007700020F000408842DCBF00209DED040B32DDFC
:100780002849884209D1049840B94FF00100F0F798
:10079000F4F900F085FE06B010BD05DB9DED040BFD
:1007A00000F06AFE06B010BD68469DED040B00F037
:1007B000BBF810F0030011D0012818D09DED021BEA
:1007C0009DED000B02281AD000F0CAFA51EC100B74
:1007D00006F016FA06B041EC100B10BD9DED021BA1
:1007E0009DED000B012000F0EFFB06B010BD9DED6C
:1007F000021B9DED000B00F0B3FA06B010BD012006
:1008000000F0E2FB51EC100B06F0FAF906B041ECF7
:10081000100B10BD000000000000000000000000F0
:10082000FB21E93F0000F07F00B52DED048BB0EE19
:10083000409AF0EE609A83B051EC190B06F044FE3A
:1008400041EC180B18EE100A18EE901A8DED008B83
:10085000002818BF0120084320F00040C0F17F604D
:1008600000F1E040C00F14D019EE101A19EE900AF2
:100870008DED009B002918BF0121084320F00040A6
:10088000C0F17F6000F1E040C00F04BF0120F0F72D
:1008900074F9B0EE480A03B0F0EE680ABDEC048BC0
:1008A00000BD00000000000010B51D499FED1A1B9F
:1008B0002DED020B84B0059820F000408842DCBF8B
:1008C00001209DED040B21DD1649884209D10498D1
:1008D00040B94FF00100F0F750F900F0E1FD06B02B
:1008E00010BD05DB9DED040B00F0C6FD06B010BD8C
:1008F00068469DED040B00F017F800F0010001219F
:10090000A1EB40009DED021B9DED000B00F0F4FB00
:1009100006B010BD00000000000000000000000054
:10092000FB21E93F0000F07F2DE9F14F04462DED5A
:10093000020B2DED088B8AB09FEDE70B80ED020BCB
:10094000139EE74826F0004585420ADC9DED120B18
:10095000002084ED000B0AB0BDEC088B03B0BDE8AD
:10096000F08FE0489FEDE0AB9FEDE1BBA84247DD93
:10097000E14F9FEDE39B9FEDE48B9DED120B53EC5C
:100980001A2B51EC100B002E1CDD06F069FE41EC19
:10099000100BBD4208D053EC1B2B51EC100B06F092
:1009A0005FFEC4E900010BE053EC192B51EC100B76
:1009B00006F056FE53EC182B06F052FEC4E9000177
:1009C0000120C8E706F05AF941EC100BBD4208D0EF
:1009D00053EC1B2B51EC100B06F050F9C4E900014D
:1009E0000BE053EC192B51EC100B06F047F953ECCC
:1009F000182B06F043F9C4E900014FF0FF30AAE7D5
:100A0000C348A84279DB9DED120B51EC100B02F0AC
:100A1000ABF941EC180B9FEDC00B53EC102B06F01B
:100A200013FC9FEDBF1B53EC112B06F027F906F0CA
:100A300075FB074606F0A1FB41EC190B53EC1A2B92
:100A400006F002FC53EC182B06F032FD41EC180BBB
:100A500053EC1B2B51EC190B06F0F6FBDFF8C8A288
:100A600041EC100B4FEA15580125FA4453EC102BBA
:100A700051EC180B06F0F4FD032DC4E900013DD044
:100A8000C1F30A5005EB4511A8EB00001139814272
:100A900034DA0AEB051BB0EE48AA9BED000BF0EE32
:100AA00068AA53EC102B51EC190B06F0CDFB41EC6E
:100AB0001B0B51EC1A0B53EC1B2B06F0D1FD41EC38
:100AC000180B51EC1A0B53EC182B06F0C9FD53EC24
:100AD0001B2B06F0C5FD9BED020B41EC1A0B53ECF2
:100AE000102B51EC190B06F0AFFB53EC1A2B06F050
:100AF000B7FD41EC100B6D1CB8E70EE0002EA8BF4F
:100B00003846BFF628AF94ED000B51EC100B06F001
:100B100077F8C4E9000178421DE7C6F3130040F4FA
:100B2000801EC6F30A50A0F2F530471100F01F05F1
:100B3000C5F12000DDF848B008900020069007902D
:100B40000520EC467949002D07EB0002794408BFE7
:100B500051F8221009D051F8223001EB8201AB404C
:100B60004A68089922FA01F11943A1FB0E26A1FB5C
:100B70000B131A449A4234BF0123002303EB0608E7
:100B80000CEB8003D3E901A60E448E4234BF012151
:100B9000002192448A4411B1924502D903E0924562
:100BA00001D2012100E00021C3E901A641444CF833
:100BB0002010011EA0F10100C4DC029800F10050D9
:100BC000850F0298DDE903678000DDF8148006F0E8
:100BD000D4FA41EC1A0B304606F0E6FA9FED541BAE
:100BE00053EC112B06F030FB41EC1B0B384606F0A2
:100BF000DBFA9FED511B53EC112B06F025FB41EC6A
:100C0000180B404606F0D0FA9FED4D1B53EC112B0C
:100C100006F01AFB41EC190B51EC180B53EC192B95
:100C200006F02CF853EC1B2B06F028F853EC1A2B8B
:100C300006F024F8CDE90801002008909DED080B8E
:100C400053EC1A2B51EC100B06F00AFD53EC1B2B46
:100C500006F006FD53EC182B06F002FD53EC192BA1
:100C600006F026FC9FED381B53EC112B06F0ECFA36
:100C70009FED370B41EC180B53EC102B9DED080B3F
:100C800051EC100B06F0E0FA53EC182B05F0F6FFD0
:100C90009FED310B41EC180B53EC102B9DED080B25
:100CA00051EC100B06F0D0FA53EC182B05F0E6FFD0
:100CB00041EC100B139810F0004F06D06D4251EC30
:100CC000100B05F09DFF41EC100B284684ED000B46
:100CD00041E60000000000000000000000000000ED
:100CE000FB21E93F7CD9024000004054FB21F93F41
:100CF0003163621A61B4D03DFB21F93F000000006E
:100D00000000601A61B4D03D7370032E8A19A33BB2
:100D1000FB2139410000000083C8C96D305FE43F0A
:100D2000000000000000E03F72710000C070000091
:100D3000000000000000103E000000000000103C19
:100D4000000000000000103A182D4454FB21F93D2A
:100D50003326A611460B113C00000054FB21F93D3F
:100D600010B52DED040B2DED088B82B0B0EE419A3D
:100D7000F0EE619A0B9820F000449FED4BABB4F17C
:100D8000795F11DA9DED0A0B51EC100B06F0C6F9F4
:100D9000002801BFB0EE4A0AF0EE6A0A02B0BDECCC
:100DA000088B04BF04B010BD9DED0A0B53EC102B53
:100DB00051EC100B06F048FA41EC180B3C480621A8
:100DC000B0EE480AF0EE680A784400F081F853EC7F
:100DD000182B51EC100B06F037FA9DED0A0B41EC85
:100DE0001B0B53EC192B51EC100B06F02DFA41ECB8
:100DF000190B53EC1B2B51EC180B06F025FA53EC96
:100E0000192B06F02DFC9FED2C0B41EC190B53EC2C
:100E1000102B51EC180B06F017FA41EC100B284878
:100E2000844210DA53EC192B51EC100B06F018FC2D
:100E300053EC1A2B06F03CFB41EC100B02B0BDEC5E
:100E4000088B04B010BD1F48A042BCBF9FED1E1B05
:100E50008DED001B06DBA4F5001001900020009032
:100E60009DED001B51EC100B53EC112B06F0F8FB21
:100E70009DED000B41EC180B53EC102B51EC1A0BB1
:100E800006F0EEFB41EC1A0B53EC192B51EC180B4E
:100E900006F0E6FB53EC1A2B06F00AFB41EC100BB4
:100EA000CCE7000000000000000000000000F03F60
:100EB000DC6D000000000000000000000000E03FCA
:100EC0003333D33F0000E93F000000000000D23F71
:100ED00070B504462DED028B4D1E00EBC500B0EE43
:100EE000408AF0EE608A90ED000B35F0060017D0D6
:100EF00053EC182B51EC100B06F0A6F941EC100B3B
:100F00006D1E04EBC50090ED001B51EC100B53EC73
:100F1000112B05F0B3FE41EC100B35F00600E7D1C4
:100F2000022D36D0042D1CD0062D1CBFBDEC028B2B
:100F300070BD53EC182B51EC100B06F085F994EDB5
:100F40000A1B53EC112B05F099FE53EC182B06F0FD
:100F50007BF994ED081B53EC112B05F08FFE41EC4F
:100F6000100B53EC182B51EC100B06F06DF994EDAF
:100F7000061B53EC112B05F081FE53EC182B06F0E9
:100F800063F994ED040B53EC102B05F077FE41EC64
:100F9000100B53EC182B51EC100B06F055F994ED97
:100FA000021B53EC112B05F069FE53EC182B06F0D5
:100FB0004BF994ED001B53EC112B05F05FFEBDECDB
:100FC000028B41EC100B70BD31B504462DED040BC6
:100FD0002DED0A8BB0EE41BAF0EE61BA0B989DEDA3
:100FE0000A0B20F00040B0F1795F0DDA51EC100BE4
:100FF000FEF722FC042808BF00F072FA9DED0A0BF0
:10100000BDEC0A8B05B030BD53EC102B51EC100B2E
:1010100006F01AF941EC180B9DED0A0B53EC182B56
:1010200051EC100B06F010F941EC190B2C48B0EE06
:10103000480AF0EE680A05217844FFF749FF9FED62
:101040002ACBB0EE40AAF0EE60AA9CB353EC1C2B66
:1010500051EC190B06F0F8F841EC1C0B53EC1A2B71
:1010600051EC190B06F0F0F89FED210B41EC190B38
:1010700053EC102B51EC1B0B06F0E6F853EC192B3C
:1010800006F0EEFA53EC182B06F0DEF853EC1B2BAF
:1010900006F0E6FA53EC1C2B06F0E2FA9DED0A1B73
:1010A00053EC112B06F004FABDEC0A8B05B041ECB1
:1010B000100B30BDFFE753EC1A2B51EC180B06F068
:1010C000C3F853EC1C2B05F0D9FD53EC192B06F09B
:1010D000BBF89DED0A1B53EC112B05F0CFFDE3E7A8
:1010E0006C6C000000000000495555555555C5BFB2
:1010F000000000000000E03FF1B506462DED040BB6
:10110000BD482DED0C8B8AB0B0EE418AF0EE618ABD
:10111000179D25F000449FEDBABB9FEDBBCB8442E9
:1011200008DA9DED160B51EC100B05F0F7FF0028C7
:1011300000F0E980B64FA74231DC002D0DDA9DEDBD
:10114000160B51EC100B05F05BFDCDE9160151ECCF
:10115000180B05F055FD41EC180B9FEDAF0B53EC50
:10116000102B9DED160B51EC100B06F0A1F953EC72
:10117000182B9FEDAB0BCDE9040151EC100B06F0E1
:101180006FFA41EC100B53EC102B9DED040B51EC5E
:10119000100B05F073FD9FEDA48BCDE916019DEDBD
:1011A000160B53EC102B51EC100B06F04DF8CDE95B
:1011B00004019DED040B53EC102B51EC100B06F0C9
:1011C00043F841EC190B9A480621B0EE490AF0EEBB
:1011D000690A7844FFF77CFE9648B0EE40DAF0EEFC
:1011E00060DAB0EE490AF0EE690A06217844FFF7AA
:1011F0006FFE9DED041B51EC100B53EC112B06F010
:1012000023F89DED040B41EC1A0B53EC102B9DEDD4
:10121000160B51EC100B06F017F841EC190B53ECC0
:101220001A2B51EC1D0B05F029FD53EC192B06F080
:101230000BF853EC182B05F021FD9DED041B53EC2E
:10124000112B06F001F853EC182B05F017FD41ECBB
:10125000180B9FED790B51EC190B53EC102B05F08B
:10126000F3FF53EC182B05F009FD41EC190B9DED34
:10127000160B53EC192B51EC100B05F0FFFC41EC55
:10128000180BA74269DC304605F077FF41EC1A0BDA
:1012900051EC180B53EC1A2B05F0F0FC41EC1B0B36
:1012A00053EC182B51EC180B05F0CEFF53EC1B2B15
:1012B00005F0A0FD53EC192B06F0D2F99DED161B9D
:1012C00053EC112B06F0F4F89FED5D1B53EC112B42
:1012D00005F0BAFF53EC1A2B06F0EAF841EC180BB4
:1012E000022000EAA570C0F1010005F046FF53ECB2
:1012F000182B05F0A9FF00BF41EC100B0AB0BDECA4
:101300000C8B05B0F0BD711C1698214308430CD01E
:101310009DED160B012E1CBF53EC102B51EC1C0B3A
:1013200010D000BF05F066FDE6E79DED160B51EC11
:10133000100B01F019FD41EC100B51EC1B0B53ECA1
:10134000102BEFE751EC100BFEF776FA042808BFDC
:1013500000F0C6F89DED160BD0E7012E04BFB0EEED
:10136000480AF0EE680AC9D08DED048B002404947D
:101370009DED040B53EC102B9DED160B51EC100B57
:1013800006F096F853EC192B06F092F841EC190B85
:1013900053EC182B51EC1C0B05F02CFD41EC180BF9
:1013A0008DED008B00949DED040B53EC102B9DED07
:1013B000000B51EC100B05F047FF53EC1B2B05F015
:1013C0005DFC9DED000B41EC1A0B53EC192B51EC1D
:1013D000100B05F039FF53EC1A2B05F04FFC53ECC2
:1013E000182B05F031FF9DED001B53EC112B05F080
:1013F00045FC81E7000000000000303E00000000D6
:10140000000000000000F03F000000000000F0BFFE
:101410002894E53F00000000182D4454FB21E93FCB
:10142000075C143326A6813C000000000000000089
:10143000FA6A0000106B0000635555555555D53FAD
:1014400000000000000000409FED070B10B553ECBA
:10145000102B9FED070B51EC100B05F0CBFC41EC72
:10146000100B10BD00000000000000000000000094
:10147000000000000000F03F10B553EC102B51ECC1
:10148000100B05F0FBFB41EC100B10BD10B553EC3D
:10149000112B51EC100B05F0F1FB41EC100B10BDC2
:1014A0009FED050B10B553EC102B51EC100B05F014
:1014B000A1FC41EC100B10BD00000000000000007A
:1014C0009FED050B10B553EC102B51EC100B05F0F4
:1014D000BBFE41EC100B10BD0000000000000070CE
:1014E0009FED050B10B553EC102B51EC100B05F0D4
:1014F000ABFE41EC100B10BD00000000000000101E
:1015000010B5044691ED000BFEF7AEF984ED000A2C
:1015100010BD10B5044690ED000B0846FEF790FA9A
:1015200084ED000B10BD30380A2801D2012070472D
:101530000020704700BF704710B504460121062007
:10154000F8F7BAF94BF69E702040002872D004F4E8
:10155000805040B14FF47A710320F5F775F81020F0
:101560007349487285E004F4807038B1002103208B
:10157000F5F76AF803206E4948727AE004F40050E7
:1015800040B14FF47A710420F5F75EF80020684905
:1015900048726EE004F4806040B14FF47A71042028
:1015A000F5F752F810206249487262E004F0080032
:1015B00040B14FF47A710420F5F746F804205C49F5
:1015C000487256E004F4004040B14FF47A710420B0
:1015D000F5F73AF80420564948724AE004F08000D2
:1015E00028B14FF47A710420F5F72EF841E004F4A5
:1015F000006040B14FF47A710320F5F725F8072019
:101600004B49487235E004F0020038B10021062051
:10161000F5F71AF80A20464948722AE004F0040057
:1016200090B1444890F8250028B164210220F5F7D4
:101630000BF805E022E04FF47A710220F5F704F888
:1016400002203B49487214E004F4007060B14FF48A
:101650007A710120F4F7F8FF002035494872B2EEA4
:10166000040AFCF76FFC04E04FF4FA710320F4F76E
:10167000EBFF3220FCF746FC002010BD44F2610075
:10168000204098B304F4804040B14FF47A710720B1
:10169000F4F7DAFF0620264948722DE004F0200016
:1016A00028B14FF47A710620F4F7CEFF24E004F05D
:1016B000010038B100210520F4F7C6FF05201C49C0
:1016C000487219E004F0400088B100210220F4F7CC
:1016D000BBFF0020164948720121154880F8BD1053
:1016E000B2EE040AFCF72EFC0120C6E709E04FF435
:1016F000FA710320F4F7A8FF0520FCF703FC002093
:10170000BBE70C4890F8250020B164210120F4F7D4
:101710009BFF04E04FF47A710120F4F795FF082055
:101720000349487201210620F8F7C6F80120A4E712
:1017300054390220D432012010B504464FF47A7196
:1017400004FB01F000F002F810BD00002DE9F041AB
:101750000446F3F761F80746002507480068074983
:10176000B0FBF1F000FB04F602E0F3F755F8C51BFF
:10177000B542FAD3BDE8F081B007002040420F0027
:1017800008B56846F7F77EFA08BD10B54FF47A70D1
:10179000FFF7D2FF4FF44070F6F7E0FE4FF4E13070
:1017A00004F002FFFDF7DEFCFDF77CFE00210420C3
:1017B000F2F7BAFA00210420F2F71CF9F4F73EFF21
:1017C00002F0EAFA6420FFF7B7FF10BD10B54FF43E
:1017D000C0727E217F20FDF707FC10BD10B50446C6
:1017E000072C05D0082C03D0092C01D00A2C2FD1AE
:1017F0007D4890ED024AD0ED013A90ED003A7B48E9
:10180000D0ED022A90ED012AD0ED001A784890ED33
:10181000021AD0ED010A90ED000AF3F761FE754857
:1018200080ED000AC0ED010A80ED021AD0ED022A17
:1018300090ED012AD0ED001A6F4890ED021AD0ED1C
:10184000010A90ED000AFCF7BDFC6C4880ED080A27
:10185000674908316948001D01F0FCFC072C74D26F
:10186000DFE804F0040574A2A9B0B700B9E060494C
:1018700008316248001D01F0EDFC6148D0ED022AFC
:1018800090ED012AD0ED001A5E4890ED021AD0EDDD
:10189000010A90ED000AF3F79DFA584880ED090A15
:1018A00090ED091AF0EE410A514890ED021AB0EE9F
:1018B000410AF3F761FA514880ED000A524890ED71
:1018C000000ADFED520AB4EEE00AF1EE10FA06DB90
:1018D00018224A4938314E48EFF7E1F81FE04A48EC
:1018E00090ED000ADFED490AB4EEE00AF1EE10FADD
:1018F0000FD290ED000ADFED470AB4EEE00AF1EEF8
:1019000010FA06DB18223D4950314148EFF7C7F87D
:1019100005E01822394968313D48EFF7C0F83748EB
:10192000D0ED040A3848B0F84A0000EE100AB8EECC
:10193000400AF4EEC00AF1EE10FA05D218222F493F
:1019400080313348EFF7ABF84BE049E028490831E4
:101950002A48001D01F07EFC2948D0ED022A90EDB6
:10196000012AD0ED001A274890ED021AD0ED010AA5
:1019700090ED000AF3F72EFA204880ED090A90ED69
:10198000091AF0EE410A1A4890ED021AB0EE410A27
:10199000F3F7F2F9194880ED000A182200F150011E
:1019A0001B48EFF77CF81CE0114908311348001D73
:1019B00001F050FC15E00E4908311048001D01F0FF
:1019C00049FC0EE00A4908310C48001D01F042FCB8
:1019D00007E0074908310948001D01F03BFC00E021
:1019E00000BF00BF10BD0000543B0220483B022056
:1019F000243B0220603B02203C3B0220743A022040
:101A0000183B02200C3B0220543902200000FA430C
:101A10005C3A02200000484370B504460D46206839
:101A200058B9294604F1080004F0AFFD08B90020B8
:101A300070BD022020600020FAE72168481C206069
:101A400004F108004554206806280BD104F10A006F
:101A5000FCF710FC6060B0F5FD7F03DD0020206026
:101A6000401EE5E7D4E90010801D814201DA002024
:101A7000DEE700202060204600F074FDD8E70A462B
:101A80000271130A4371130C8371130EC3717047F3
:101A9000A84890ED000ADFEDA80A60EE200AA748EA
:101AA00090ED081A80EE810AF0EE000A80EE201A0E
:101AB000A34880ED001A9F4890F824000B286FD2AD
:101AC000DFE800F006113B5F6F7E8D9CBDDEFE00FF
:101AD0009FED9C0A9C4880ED000A9FED9A0A9B4866
:101AE00080ED000A23E1934890ED000AB5EEC00AAC
:101AF000F1EE10FA0AD19FED930A934880ED000AA7
:101B00009FED900A914880ED000A15E0894890ED1C
:101B1000000A8A48D0ED0A0A30EE200A8A4880ED91
:101B2000000A844890ED000A8448D0ED0A0A30EE9D
:101B3000600A864880ED000AF9E07E4890ED000AD0
:101B4000B5EEC00AF1EE10FA0AD19FED7E0A7E488A
:101B500080ED000A9FED7B0A7C4880ED000A0FE0D3
:101B6000744890ED000AB1EE400A774880ED000A13
:101B7000704890ED000AB1EE400A744880ED000A0A
:101B8000D5E06C4890ED000AB1EE400A6E4880ED59
:101B9000000A684890ED000A6C4880ED000AC6E033
:101BA000BAE0644890ED000A674880ED000A614899
:101BB00090ED000AB1EE400A644880ED000AB6E0FC
:101BC0005C4890ED000AB1EE400A5F4880ED000AE3
:101BD000584890ED000A5D4880ED000AA7E055489E
:101BE00090ED000A584880ED000A524890ED000A36
:101BF000B1EE400A554880ED000A98E04D4890ED5E
